:020000040000FA
:1000000080080120C1CF0100B79D040095CF0100F9
:1000100095CF010095CF010095CF010000000000B1
:1000200000000000000000000000000061C70100A7
:1000300095CF010000000000D1C6010095CF01005E
:10004000D1C801002DC70400D1C80100D1C80100EA
:10005000D1C80100D1C80100D1C80100D1C8010038
:10006000F5C60400D1C80100D1C8010013C70400BF
:10007000D1C80100D1C80100D1C80100D1C8010018
:10008000D1C80100D1C80100D1C80100D1C8010008
:10009000D1C80100D1C80100D1C80100D1C80100F8
:1000A000D1C80100D1C80100D1C80100D1C80100E8
:1000B000D1C80100D1C80100D1C80100D1C80100D8
:1000C000D1C80100D1C80100D1C80100D1C80100C8
:1000D000D1C80100D1C80100D1C80100D1C80100B8
:1000E000D1C80100D1C80100D1C80100D1C80100A8
:1000F000D1C80100D1C80100D1C80100D1C8010098
:1001000001F0FF01102A2BDB10F0070F08D010F8C8
:10011000013B013A8B422DD010F0070F42B3F6D1CC
:10012000F0B441EA012141EA014122F007047FF0E5
:1001300000070023F0E80256083C85EA010586EA3C
:10014000010685FA47F5A3FA87F586FA47F6A5FA78
:1001500087F68EB9EED1F0BC01F0FF0102F0070284
:1001600032B110F8013B013A83EA010313B1F8D12F
:100170000020704701387047002D06BF3546033810
:10018000073815F0010F07D1013015F4807F02BF49
:10019000013015F4C03F0130F0BC0138704700BF9A
:1001A00053B94AB9002908BF00281CBF4FF0FF31DE
:1001B0004FF0FF3000F00CB8ADF1080C6DE904CE43
:1001C0000EF030FFDDF804E0DDE9022304B07047F3
:1001D000704700BF2DE9F14F03F11C0402EB840CC2
:1001E0004FEA930B8A68CB680868496800F046F9C3
:1001F0003CE9F0006040694072407B400BF1060E24
:100200004EE083EA134480EA134582EA134746BA74
:1002100096EA3444604000F00F1684EA063420F079
:100220000F1684EA161054BA94EA0106724002F0DE
:100230000F1486EA043622F00F1486EA14124CBA20
:100240006540694001F00F1485EA043521F00F1470
:1002500085EA14115CBA67407B4003F00F1487EA0B
:10026000043723F00F1487EA141344BA44404DBAFC
:100270004D4056BA56405FBA5F4087EA174886EA53
:10028000174B84EA17464FEA38488BEA1B4485EA45
:100290001B4788EA1B4580EA3440694072407B4036
:1002A00000F0703400F0803500F00F3040EA440078
:1002B00040EAD50080EA900404F0332480EA840008
:1002C000604001F0703401F0803501F00F3141EAF7
:1002D000440141EAD50181EA910404F0332481EA22
:1002E0008401614002F0703402F0803502F00F3278
:1002F00042EA440242EAD50282EA920404F033243C
:1003000082EA8402624003F0703403F0803503F027
:100310000F3343EA440343EAD50383EA930404F02A
:10032000332483EA84036340C943DB4381EA000446
:1003300083EA044686EA020183EA014382EA3345FE
:1003400083EA14435C4084EA00077FEA040A8AEAED
:10035000024A8AEA010B87EA11488AEA374A80EAA8
:10036000060181EA1A418AEA030A04EA0A004540C2
:1003700088EA040707EA0B0041408AEA0B0608EA0C
:10038000060084EA34428AEA3A4602EA0603584002
:100390004540414087EA37438BEA3B4003EA000986
:1003A00085EA090582EA0309464006EA0906714022
:1003B00085EA010005EA3546464006EA314181EA10
:1003C000304181EA364606EA304686EA3546344010
:1003D0000F4086EA010508EA050886EA3640024031
:1003E00088EA020881EA314213405C4080EA020355
:1003F00009EA030987EA0907674088EA040806EA68
:100400000A0601EA0B018AEA0B0425408AEA3A440B
:10041000204045408BEA3B4B02EA0B02564084EAFF
:100420000B04234059406E40694087EA364080EA19
:10043000384080EA060380EA104481EA134585EAE1
:10044000344585EA17427D4082EA354180EA05401D
:100450003CE9F0006040694072407B40BEF1010E13
:100460003FF6CFAE20BC00F05FF828606960AA605C
:10047000EB60BDE8F08F00BF00F000BA80EA101416
:1004800004F0F01480EA0410604081EA111404F0D2
:10049000F01481EA0411614082EA121404F0F014AD
:1004A00082EA0412624083EA131404F0F01483EA2F
:1004B0000413634080EA102404F47F4480EA04209B
:1004C000604081EA112404F47F4481EA0421614000
:1004D00082EA122404F47F4482EA0422624083EA1E
:1004E000132404F47F4483EA0423634081EA500424
:1004F00004F0553480EA4400614083EA520404F079
:10050000553482EA4402634082EA900404F03334B2
:1005100080EA8400624083EA910404F0333481EA83
:1005200084016340704700BF82EA900404F03334D2
:1005300080EA8400624083EA910404F0333481EA63
:100540008401634081EA500404F0553480EA440099
:10055000614083EA520404F0553482EA4402634065
:1005600080EA102404F47F4480EA0420604081EA99
:10057000112404F47F4481EA0421614082EA1224B8
:1005800004F47F4482EA0422624083EA132404F4E0
:100590007F4483EA0423634080EA101404F0F014DB
:1005A00080EA0410604081EA111404F0F01481EA3A
:1005B0000411614082EA121404F0F01482EA041279
:1005C000624083EA131404F0F01483EA04136340D6
:1005D000704700BF2DE9F14F94464FEA930B8A68AC
:1005E000CB6808684968FFF749FF0BF1060E33E056
:1005F00083EA134480EA134582EA134746BA96EA2F
:100600003444604000F00F1684EA063420F00F16E0
:1006100084EA161054BA94EA0106724002F00F14EC
:1006200086EA043622F00F1486EA14124CBA6540AA
:10063000694001F00F1485EA043521F00F1485EAB2
:1006400014115CBA67407B4003F00F1487EA04374B
:1006500023F00F1487EA1413BCE8F00060406940EF
:1006600072407B4000F0E03400F0103500F00F30B5
:1006700040EA540040EAC50080EA900404F03324C4
:1006800080EA8400604001F0E03401F0103501F0B0
:100690000F3141EA540141EAC50181EA910404F0B5
:1006A000332481EA8401614002F0E03402F0103525
:1006B00002F00F3242EA540242EAC50282EA920490
:1006C00004F0332482EA8402624003F0E03403F051
:1006D000103503F00F3343EA540343EAC50383EABA
:1006E000930404F0332483EA8403634081EA3247AD
:1006F00087EA134581EA354690EA060484EA034B0B
:1007000082EA1B4280EA044484EA054483EA144AEC
:1007100085EA14448BEA044B84EA374481EA0B41AE
:1007200081EA164104EA0A00454082EA04082BEAFD
:10073000080041408AEA0B0602EA060084EA3443D4
:100740008AEA3A4603EA060778404540414088EA8B
:1007500038478BEA3B4007EA000985EA090583EA46
:100760000709464006EA0906714085EA010005EAE4
:100770003546464006EA314181EA304181EA364653
:1007800006EA304686EA3546344008EA010886EA39
:1007900001052A4086EA364003405A4081EA314347
:1007A0001F407C4080EA030709EA070988EA090834
:1007B000544088EA020806EA0A0601EA0B018AEABE
:1007C0000B0215408AEA3A42104045408BEA3B4012
:1007D00003405E404240174079404D404E40E44364
:1007E000F64386EA18435D4085EA054083EA1343F1
:1007F00086EA034183EA384284EA114383EA0443E8
:100800005FEA3343BEF1010E3FF6F2AE1ED4BCE800
:10081000F0006040694072407B4020BCFFF784FEDE
:1008200028606960AA60EB60BDE8F08F2DE9E041C7
:100830004FF2F00280EA1031114080EA0130484066
:1008400041088208C3084FF0000E4FE700F0113056
:1008500001F0113102F0113203F0113340EA41008E
:1008600040EA820040EAC3004FF2F00280EA103111
:10087000114080EA01304840BDE8E0812DE9F04FA9
:1008800002F11C050646074600EB850851F8040BEB
:10089000043A46F8040BF9D14FF0010CFFF7C6FFFC
:1008A0005FEA302080EA0C001ECF41404A405340AE
:1008B0005C401EC62000464517D04FEA4C0C1CF485
:1008C000807F18BFACF1E50C2C2DE7D03C2D06D174
:1008D000FFF7ACFF06CF41404A4006C6100006CFE6
:1008E00041404A4006C61000D8E736E90F00FFF73E
:1008F000C5FD043D86E80F00F7D1BDE8F08F00BFCD
:1009000070B491E87800B2E802105B1854EB0C0464
:10091000B2E802104D4156EB0C0680E878008041A9
:10092000013070BC704700BF70B491E87800B2E845
:1009300002105B1A74EB0C04B2E802108D4176EBE6
:100940000C0680E878008041404270BC704700BFD0
:100950002DE9F00791E80017C0CAA8FB063440F85B
:10096000043BA9FB0615E8FB6741EAFB665140F82A
:10097000044BA9FB0743ECFB661344CAE8FB625433
:10098000EAFB6714ECFB673440F8045BA9FB0275D3
:10099000EAFB6235ECFB6245E8FB6617E9FB66376C
:1009A000EAFB6647ECFB6657BAC0BDE8F007704744
:1009B0002DE9F00391E8F803B2E802105B1854EB5C
:1009C0000C04B2E802104D4156EB0C0692E80610FA
:1009D0004F4158EB020859EB0C0980E8F8038041BD
:1009E0000130BDE8F00370472DE9F00391E8F8030A
:1009F000B2E802105B1A74EB0C04B2E802108D41ED
:100A000076EB0C0692E806108F4178EB020879EB42
:100A10000C0980E8F80380414042BDE8F0037047CC
:100A20002DE9F003524290E83800B1E88003174006
:100A3000DB1918EA020854EB080419EA020955EB1D
:100A4000090538C090E8780091E8820311404B41D5
:100A500017407C4118EA020855EB080519EA02091B
:100A600056EB090678C080410130BDE8F0037047BD
:100A70002DE9F003524290E83800B1E880031740B6
:100A8000DB1B18EA020874EB080419EA020975EB8B
:100A9000090538C090E8780091E8820311408B4145
:100AA0001740BC4118EA020875EB080519EA02096B
:100AB00076EB090678C080414042BDE8F0037047FC
:100AC0002DE9F00152424FF0030890E8300091E820
:100AD000C000A31B1340E41AF618EB1B1340ED1AD9
:100AE000FF1830C0C0C1B8F10108EED104680E682B
:100AF000A31B1340E41AF61804600E60BDE8F00171
:100B0000704700BF00B592EC070AB1E8005E07EE3F
:100B1000101A56EC102A58EC117AA9FB0250AAFBC5
:100B20000234E9FB6603EBFB624340EC145AAAFB78
:100B30000605ECFB6235E9FB6740E9FB6830EEFB3C
:100B40006250AAFB0721EAFB6851EBFB680112EE39
:100B5000108AEBFB6632ECFB6652EAFB6802EBFBA9
:100B6000681243EC154AA9FB084312EE908AE9FB90
:100B70006803EAFB6813EBFB6823EBFB6754EEFBAF
:100B8000660413EE108AE9FB6814EAFB6824EBFBA9
:100B9000683406EE105A17EE109A99E8000CACFB78
:100BA000076511EE909AECFB6915EEFB6925EAFBEF
:100BB0006935EBFB694510EE109AEAFB6906EBFB21
:100BC000691612EE109AECFB6926EEFB6936EAFB19
:100BD0006946EBFB695610EE909AAAFB0987EBFB7E
:100BE000692712EE909AECFB6937EEFB6947EAFB46
:100BF0006957EBFB696711EE109AEEFB6918EAFB87
:100C00006928EBFB693813EE109AECFB6948EEFBA0
:100C10006958EAFB6968EBFB697800BD2DE9F04F84
:100C200007EE900AFFF76EFF17EE909AA9EC054ABF
:100C300089E8FF01BDE8F08F00B591E8805FA7FB70
:100C40000750A7FB0834E7FB6803E7FB694340EC68
:100C5000145AA7FB0905E7FB6A35E8FB6840E7FB88
:100C60006A30E7FB6B50A8FB0921E7FB6B51E7FB00
:100C70006C01E8FB6932E8FB6A52E7FB6C02E7FBB8
:100C80006E1243EC154AA8FB0A43E8FB6B03E7FB33
:100C90006E13E8FB6E23E9FB6954E8FB6B04E8FB89
:100CA0006C14E8FB6E24E9FB6E3406EE105AA9FBC7
:100CB0000A65E8FB6C15E9FB6C25E9FB6E35EAFB80
:100CC0006E45E9FB6A06E9FB6B16E9FB6C26EAFB5D
:100CD0006C36EAFB6E46EBFB6E56A9FB0B87EAFB14
:100CE0006B27EAFB6C37EBFB6C47EBFB6E57ECFBBF
:100CF0006E67EAFB6A18EAFB6B28EBFB6B38EBFBD1
:100D00006C48ECFB6C58ECFB6E68EEFB6E7800BD3B
:100D10002DE9F04F07EE900AFFF78EFF17EE909A3D
:100D2000A9EC054A89E8FF01BDE8F08F2DE9F0073D
:100D300091E8F807B2E802105B1854EB0C04B2E833
:100D400002104D4156EB0C06B2E802104F4158EB31
:100D50000C08B2E8021059EB01095AEB0C0A80E8C2
:100D6000F80780410130BDE8F00770472DE9F00732
:100D700091E8F807B2E802105B1A74EB0C04B2E8D1
:100D800002108D4176EB0C06B2E802108F4178EB31
:100D90000C08B2E8021079EB01097AEB0C0A80E842
:100DA000F80780414042BDE8F00770472DE9F007A1
:100DB000524290E87800B1E880071740DB1918EA42
:100DC000020854EB080419EA020955EB09051AEA6E
:100DD000020A56EB0A0678C090E87800B1E880076E
:100DE00017407B4118EA020854EB080419EA02098B
:100DF00055EB09051AEA020A56EB0A0678C080414B
:100E00000130BDE8F00770472DE9F007524290E845
:100E10007800B1E880071740DB1B18EA020874EB82
:100E2000080419EA020975EB09051AEA020A76EBC9
:100E30000A0678C090E87800B1E880071740BB4107
:100E400018EA020874EB080419EA020975EB0905AF
:100E50001AEA020A76EB0A0678C080414042BDE8F1
:100E6000F00770472DE9F00152424FF0040890E876
:100E7000300091E8C000A31B1340E41AF618EB1BE6
:100E80001340ED1AFF1830C0C0C1B8F10108EED10F
:100E9000BDE8F001704700BF00B592EC080AB1E868
:100EA000805707EE101A53EC102A56EC114AA7FB94
:100EB0000251A8FB020BE7FB6310E9FB62B041ECB7
:100EC000145AA8FB0351EAFB6201E7FB64B5E7FB98
:100ED0006605E8FB661505EE10BAA9FB03B6EAFB4A
:100EE0006316ECFB6356E8FB640BE9FB641BEAFB4F
:100EF000645BECFB646B05EE900AACFB023012EE17
:100F0000104AEEFB6250E9FB6460EAFB64B0E7FB69
:100F10006431E8FB645112EE904AE8FB6461E9FB3E
:100F200064B1EAFB640106EE103AA7FB043213EE4B
:100F3000104AE7FB6462E8FB64B2E9FB6402EAFB87
:100F4000641211EE904AE9FB6453EAFB646313EE0A
:100F5000904AE7FB64B3E8FB6403E9FB6413EAFB34
:100F6000642306EE905A17EE109A99E8000610EEE8
:100F7000108AA9FB0854EAFB68B412EE108AECFB55
:100F80006804EEFB6814E9FB6824EAFB683410EEA1
:100F9000908AEEFB6865E9FB68B5EAFB680512EE2E
:100FA000908AECFB6815EEFB6825E9FB6835EAFBE7
:100FB000684507EE106A11EE108AAEFB0876E9FB71
:100FC0006806EAFB681613EE108AECFB6826EEFB57
:100FD0006836E9FB6846EAFB685611EE908AECFB3E
:100FE00068B7EEFB6807E9FB6817EAFB682713EEB2
:100FF000908AECFB6837EEFB6847E9FB6857EAFB31
:10100000686700BD2DE9F04F07EE900AFFF744FF37
:1010100017EE908A07EE90BAA8EC084A88E8FF001D
:10102000BDE8F08F00B591E89857A3FB0352A3FBEE
:101030000401E3FB6420E3FB671042EC145AA3FBBA
:101040000752E3FB6802E4FB6415E3FB6805E3FB7E
:101050006925A4FB07B6E3FB6926E3FB6A56E4FBBC
:10106000670BE4FB682BE3FB6A5BE3FB6C6B40EC18
:10107000151AA4FB0810E4FB6950E3FB6C60E3FB6A
:101080006EB0E7FB6721E4FB6951E4FB6A61E3FBB7
:101090006EB1E4FB6E0106EE102AA7FB0832E4FBFA
:1010A0006A62E4FB6CB2E4FB6E02E7FB6E12E7FBE4
:1010B0006853E7FB6963E4FB6CB3E7FB6C03E7FB96
:1010C0006E13E8FB6E2306EE905AA7FB0954E7FB6C
:1010D0006AB4E7FB6C04E8FB6C14E8FB6E24E9FBE4
:1010E0006E34E8FB6865E7FB6AB5E8FB6A05E8FB78
:1010F0006C15E9FB6C25E9FB6E35EAFB6E4507EEE6
:10110000106AA8FB0976E8FB6A06E9FB6A16E9FBA8
:101110006C26EAFB6C36EAFB6E46ECFB6E56E8FB8F
:1011200069B7E9FB6907E9FB6A17EAFB6A27EAFB8B
:101130006C37ECFB6C47ECFB6E57EEFB6E6700BD4B
:101140002DE9F04F07EE900AFFF76CFF17EE908A3B
:1011500007EE90BAA8EC084A88E8FF00BDE8F08FD7
:101160002DE9F14FFEC8F0EC030A90E8005F4FF064
:101170000A0003EE100A10EE900ADB199CEA030C39
:1011800018EB3C4897EA080713EB375393EA3C4CBB
:1011900018EB3C6898EA375724189EEA040E19EBBE
:1011A0003E4990EA090014EB305494EA3E4E19EBA4
:1011B0003E6999EA305049EC128A59EC118A491972
:1011C0009AEA010A18EB3A4895EA080511EB3551FD
:1011D00091EA3A4A18EB3A6898EA355592199BEA2F
:1011E000020B19EB3B4996EA090612EB365292EADA
:1011F0003B4B19EB3B6999EA365613EB706393EA64
:101200003B6B18EB3B4898EA706013EB305393EA62
:101210003B4B5FEA3B6B18EB0B0898EA30505FEAF8
:10122000706014EB756494EA3C6C19EB3C4999EAE4
:10123000756514EB355494EA3C4C5FEA3C6C19EB51
:101240000C0999EA35555FEA756549EC118A59EC44
:10125000128A11EB766191EA3E6E18EB3E4898EAED
:10126000766611EB365191EA3E4E5FEA3E6E18EB20
:101270000E0898EA36565FEA766612EB776292EAD3
:101280003A6A19EB3A4999EA776712EB375292EAD0
:101290003A4A5FEA3A6A19EB0A0999EA37575FEA6C
:1012A000776700EE900A13EE100A01387FF461AF01
:1012B00001BCFEC0E0EC030AA0E8005FBDE8F08FCF
:1012C00030B44FF0000310F8014B11F8015B013A04
:1012D00084EA050443EA0403F5D1A3F101034FEACC
:1012E000D37030BC704700BF4FF0000310F8012BE3
:1012F000013943EA0203F9D1A3F101034FEAD370A4
:10130000704700BF30B411F8014B12F8015B6C401C
:1013100000F8014B013BF6D130BC704702EAE371A3
:101320004FEA430002EAE07C9CEA4101404102EAC4
:10133000E07C9CEA4101404102EAE07C9CEA4101F8
:10134000404102EAE07C9CEA4101404102EAE07C43
:101350009CEA4101404102EAE07C9CEA41014041B3
:1013600002EAE07C9CEA4101404102EAE07C9CEA1E
:101370004101404102EAE07C9CEA4101404102EA2D
:10138000E07C9CEA4101404102EAE07C9CEA4101A8
:10139000404102EAE07C9CEA4101404102EAE07CF3
:1013A0009CEA4101404102EAE07C9CEA4101404163
:1013B00002EAE07C9CEA4101404102EAE07C9CEACE
:1013C0004101404102EAE07C9CEA4101404102EADD
:1013D000E07C9CEA4101404102EAE07C9CEA410158
:1013E000404102EAE07C9CEA4101404102EAE07CA3
:1013F0009CEA4101404102EAE07C9CEA4101404113
:1014000002EAE07C9CEA4101404102EAE07C9CEA7D
:101410004101404102EAE07C9CEA4101404102EA8C
:10142000E07C9CEA4101404102EAE07C9CEA410107
:10143000404102EAE07C9CEA4101404102EAE07C52
:101440009CEA4101404102EAE07C9CEA41014041C2
:1014500002EAE07C9CEA4101404149184041704762
:101460002DE9F34FD0F80080D1F80090D0F804A017
:10147000D1F804B098FA88F899FA89F99AFA8AFAB0
:101480009BFA8BFB42464B46FFF748FF04000D00DA
:1014900052465B46FFF742FF45400F0095EA0106C2
:1014A000654082EA080283EA0903FFF737FF4540F7
:1014B0004E4003BC01B4F0B484688D68C668CF6840
:1014C00024BA2DBA36BA3FBA88EA040089EA05017F
:1014D0008AEA060A8BEA070B03B422002B00FFF707
:1014E0001DFF8046894632003B00FFF717FF89EA5F
:1014F00000090F0089EA010689EA080962406B4089
:10150000FFF70CFF89EA000971403846FCBC4C40EB
:1015100084EA510485EAC17584EA910485EA8175FB
:1015200084EAD11485EA4165454085EA500586EA9A
:10153000C07685EA900586EA807685EAD01586EA47
:10154000406688EA060889EA070988EA040689EA03
:101550000507FFF7E3FE464047404F4088EA010891
:1015600082EA0A0283EA0B03FFF7D8FE474088EAC3
:10157000010852465B46FFF7D1FE474088EA000863
:1015800088EA010889EA010994EA080484EA58040F
:1015900085EAC87584EA980485EA887584EAD814CF
:1015A00085EA486595EA090585EA590586EAC97616
:1015B00085EA990586EA897685EAD91586EA496633
:1015C00001BC24BA04602DBA456036BA86603FBAC1
:1015D000C760BDE8F08F00BF30B40168426883681F
:1015E000C46809BA12BA1BBA24BACD1705F0870528
:1015F00095EA44045B415241494109BA016012BA7B
:1016000042601BBA836024BAC46030BC704700BF1C
:101610002DE9F00391E8F803B2E802105B1854EBEF
:101620000C04B2E802104D4156EB0C0692E806108D
:101630004F4158EB020859EB0C098941013B74F109
:10164000000475F1000576F1FF3677F1FF3778F188
:10165000FF3879F1FF3951F1000113EBD17354F1E7
:10166000000455F100054E414F4158EB010859EB7C
:10167000010980E8F803BDE8F00370472DE9F003A5
:1016800091E8F803B2E802105B1A74EB0C04B2E8BC
:1016900002108D4176EB0C0692E806108F4178EB34
:1016A000020879EB0C09894113EBD17354F1000462
:1016B00055F100054E414F4158EB010859EB010926
:1016C00080E8F803BDE8F003704700BF2DE9F04F54
:1016D00007EE900AFFF716FA5AEC359AB9EB0509AE
:1016E0007AEB060AB84171EB080172F1000273F15E
:1016F000000374F100046BEB0B0B491972417B4141
:1017000054EB08044BF1000557EC146A15EE108AEF
:10171000BEEB0E0E59EB02095AEB030A6041694118
:101720005EF1000E96419F4178EB040879EB0509C4
:101730007AF1000A70F1000B71F1000C6EF1010EEC
:1017400016EBDE7657F1000758F1000859EB0E0949
:101750005AEB0E0A5BEB0E0B5CEB0E0C17EE900ACD
:1017600080E8C01FBDE8F08F2DE9F04F07EE900A2A
:10177000FFF762FAB0E700BF2DE9F00791E8F8073C
:10178000B2E802105B1854EB0C04B2E802104D41B1
:1017900056EB0C06B2E802104F4158EB0C08B2E8C9
:1017A000021059EB01095AEB0C0A8941B3F1FF33DE
:1017B00074F1FF3475F1FF3576F1000677F100071B
:1017C00078F1000879F101097AF1FF3A51F100014D
:1017D0005B184C414D4156F1000657F1000758F196
:1017E000000859EBD1795AEB010A80E8F807BDE807
:1017F000F00770472DE9F00791E8F807B2E802100A
:101800005B1A74EB0C04B2E802108D4176EB0C0607
:10181000B2E802108F4178EB0C08B2E8021079EBC5
:1018200001097AEB0C0A89415B184C414D4156F194
:10183000000657F1000758F1000859EBD1795AEB2F
:10184000010A80E8F807BDE8F007704718EB0408C4
:1018500059EB05095AEB060A5BEB070B5FF0000C2E
:101860004CF1000C18EB050859EB06095AEB070A76
:101870005BEB070B50EB0C005FF0000C51EB0C0125
:1018800052EB0C0263414CF1000CB8EB070879F104
:1018900000097AF1000A7BEB040BA841B141A24197
:1018A000B3416CF1000CBBEB050BB041B941AA414F
:1018B000BB416CF1000C6FEAEC74B8EB040879EBF7
:1018C00004097AEB040A7BF1000B70F1000071F15E
:1018D000000172EBD472A3416CF1000C18EBEC78B0
:1018E00059EBEC795AEBEC7A5BF1000B50F1000408
:1018F00051F1000552EBDC7653EBEC774CF1000C28
:1019000018EBEC7059EBEC715AEBEC725BF10003E5
:1019100054F1000455F1000556EBDC7657EBEC77FB
:10192000704700BF2DE9F04F07EE900AFFF7B4FAB9
:1019300059EC168A17EE10AAFFF788FF59EC148AA3
:101940005BEC15AAFFF782FF17EE908A88E8FF008C
:10195000BDE8F08F2DE9F04F07EE900AFFF762FB2C
:1019600059EC168A17EE10AAFFF770FF59EC148A8B
:101970005BEC15AAFFF76AFF17EE908A88E8FF0074
:10198000BDE8F08F2DE9F00791E8F807B2E8021002
:101990005B1854EB0C04B2E802104D4156EB0C06F8
:1019A000B2E802104F4158EB0C08B2E8021059EBB4
:1019B00001095AEB0C0A4FF0260261EB010122EA01
:1019C00001015B1854F1000455F1000556F10006C1
:1019D00057F1000758F1000859F100095AF1000ABF
:1019E00061EB010122EA01010B4480E8F807BDE840
:1019F000F00770472DE9F00791E8F807B2E8021008
:101A00005B1A74EB0C04B2E802108D4176EB0C0605
:101A1000B2E802108F4178EB0C08B2E8021079EBC3
:101A200001097AEB0C0A4FF0260261EB010102EA90
:101A300001015B1A74F1000475F1000576F10006EE
:101A400077F1000778F1000879F100097AF1000ACE
:101A500061EB010102EA0101A3EB010380E8F80751
:101A6000BDE8F007704700BF2DE9F04F07EE900A80
:101A7000FFF712FA4FF0260C59EC148A4FF0000AC7
:101A8000E0FB0C8AE1FB6C9A51EC150AE2FB6CA0BE
:101A9000E3FB6C0153EC162AE4FB6C12E5FB6C23B0
:101AA0005EEC174AE6FB6C34E7FB6CB40CFB04F409
:101AB00018EB040459F100055AF1000650F1000733
:101AC00051F1000852F1000953F1000A5BF1000BDB
:101AD00060EB00002CEA000004448EE8F00FBDE843
:101AE000F08F00BF2DE9F04F07EE900AFFF79AFA4A
:101AF000C0E700BF2DE9F00391E8F8134FF4EE3191
:101B0000BF390022E3FB6123E4FB6134E5FB61455F
:101B1000E6FB6156E7FB6167E8FB6178E9FB6189F9
:101B2000ECFB619C4FF0260101FB0CFC12EB0C025C
:101B300053F1000354F1000455F1000556F100067D
:101B400057F1000758F1000859F100096CEB0C0C33
:101B500021EA0C010A4480E8FC03BDE8F003704769
:101B60002DE9F00390E8F8134FEAEC7202F013024B
:101B70002CF0004C02F11301591854F1000155F1F9
:101B8000000156F1000157F1000158F1000159F12F
:101B900000015CF100014FEAE17101F01301114411
:101BA0005B1854F1000455F1000556F1000657F199
:101BB000000758F1000859F100094CF1000C2CF015
:101BC000004C80E8F813BDE8F00370472DE9F14FB1
:101BD000F8C892E8005E19EB03095AEB040A5BEBC4
:101BE000050B5CEB060C4EEB070E91E8E001A9FB40
:101BF0000502AAFB0543E9FB6624EAFB6634A9FB60
:101C00000765E9FB6845B1E80003EBFB6836ECFBD0
:101C10006846EEFB6856ABFB0987ECFB6957EEFBA9
:101C2000696791E80202EAFB6148EBFB6158ECFB53
:101C30006168EEFB61784FF00001EAFB0951EBFBB4
:101C40006961ECFB6971EEFB69814FF4A03C4FEADE
:101C5000154949EA06495FF0000AE9FB0C0A4FEA18
:101C6000164646EA0746E6FB6C2A4FEA174747EA5C
:101C70000847E7FB6C3A4FEA184848EA0148E8FB96
:101C80006C4AADB25544AF0805F0030507EB870772
:101C9000C01952F1000153F1000254F1000345F163
:101CA000000420BC1FC5BDE8F08F00BF30B490E831
:101CB0003C10511D53F1000154F1000155F1000198
:101CC0004CF100014FEA9101494201F0050152181F
:101CD00053F1000354F1000455F100054CF1000CE0
:101CE0000CF0030C80E83C1030BC70472DE9F04F3D
:101CF00090E8F00F00F140004FF0040E59E0F0B40E
:101D0000826BC36B04680525242687593C444FEA3F
:101D1000724787EAF24787EA92273C4442684FEAD3
:101D2000F21787EAB24787EAD2073C4440F8044BEF
:101D3000032D08BF6FF01B0687593A444FEA7347DB
:101D400087EAF34787EA93273A4443684FEAF31751
:101D500087EAB34787EAD3073A4440F8042B875908
:101D60003B444FEA744787EAF44787EA94273B44A9
:101D700044684FEAF41787EAB44787EAD4073B443C
:101D800040F8043B013DC0D1A0F13C00076A3C444F
:101D90004FEA724787EAF24787EA92273C44026893
:101DA0004FEAF21787EAB24787EAD2073C44C46396
:101DB000F0BC4FF0020288EA781C8CEAF84C0BEB7E
:101DC000BC1C8AEA090303EA080383EA0A039C4469
:101DD00050F8043B9C4451F8043B9C44674444EA5B
:101DE000050B0BEA060B04EA05034BEA030BE3447D
:101DF00084EAF42383EA34530BEBB30B87EA771CB2
:101E00008CEAF74C0AEBBC1C89EA080303EA0703D7
:101E100083EA09039C4450F8043B9C4451F8043B7A
:101E20009C4466444BEA040A0AEA050A0BEA0403E6
:101E30004AEA030AE2448BEAFB2383EA3B530AEBB8
:101E4000B30A86EA761C8CEAF64C09EBBC1C88EADD
:101E5000070303EA060383EA08039C4450F8043BA3
:101E60009C4451F8043B9C4465444AEA0B0909EA46
:101E700004090AEA0B0349EA0309E1448AEAFA235E
:101E800083EA3A5309EBB30985EA751C8CEAF54CF1
:101E900008EBBC1C87EA060303EA050383EA070391
:101EA0009C4450F8043B9C4451F8043B9C446444DB
:101EB00049EA0A0808EA0B0809EA0A0348EA03089B
:101EC000E04489EAF92383EA395308EBB30884EA4A
:101ED000741C8CEAF44C07EBBC1C86EA050303EA8D
:101EE000040383EA06039C4450F8043B9C4451F8E5
:101EF000043B9C44E34448EA090707EA0A0708EA66
:101F0000090347EA0307674488EAF82383EA38535A
:101F100007EBB3078BEA7B1C8CEAFB4C06EBBC1C83
:101F200085EA040303EA0B0383EA05039C4450F8A3
:101F3000043B9C4451F8043B9C44E24447EA0806B5
:101F400006EA090607EA080346EA0306664487EA42
:101F5000F72383EA375306EBB3068AEA7A1C8CEA46
:101F6000FA4C05EBBC1C84EA0B0303EA0A0383EA80
:101F700004039C4450F8043B9C4451F8043B9C44AB
:101F8000E14446EA070505EA080506EA070345EACB
:101F90000305654486EAF62383EA365305EBB30569
:101FA00089EA791C8CEAF94C04EBBC1C8BEA0A0325
:101FB00003EA090383EA0B039C4450F8043B9C4466
:101FC00051F8043B9C44E04445EA060404EA070453
:101FD00005EA060344EA0304644485EAF52383EA38
:101FE000355304EBB304013A7FF4E5AEA0F14000B1
:101FF000BEF1010E7FF483AEA0F1400C9CE80F000F
:10200000001949199219DB19ACE80F009CE80F0080
:102010004044494452445B44ACE80F00BDE8F08FB3
:102020002DE90050ACF1400204EE90CAB2EC020A75
:10203000C0CAB2EC021AB2E80003B2EC022AB2E85B
:10204000000CB2EC023AB2E8005055EC124A84EAB5
:10205000D46080EA451085EAD56181EA441180EABE
:10206000141080EA057081EA151181EA04711CEBF5
:10207000903C4EEB913E1CEB814C4EEB804E53EC72
:10208000132A82EA0A0083EA0B01204029405040CB
:1020900059401CEB000C5EEB010E51EC140AD0E928
:1020A00000451CEB040C5EEB050ED1E900451CEB72
:1020B000040C5EEB050E18EB0C0859EB0E09D0E989
:1020C000024512196B41D1E9024512196B4155ECD9
:1020D000124A8AEA04008BEA050110EA080011EAB4
:1020E000090190EA0A0091EA0B0112184B4188EAB3
:1020F000D86080EA491089EAD96181EA481180EA0A
:10210000181080EA097081EA191181EA087112EB4E
:10211000903243EB913312EB814243EB804343EC2B
:10212000132A53EC102A55EC114A82EAD22080EA95
:10213000435083EAD32181EA425180EA921080EA37
:10214000836081EA931181EA82611CEB107C4EEB83
:10215000117E1CEB011C4EEB001E82EA0601324090
:1021600001EA040050401CEB000C01EA0C00504056
:1021700083EA07023B4012EA050159405EEB010E7B
:1021800002EA0E01594053EC132AA4185D4145ECB4
:10219000114A12184B418CEADC2080EA4E508EEA3C
:1021A000DE2181EA4C5180EA9C1080EA8E6081EA4F
:1021B0009E1181EA8C6112EB107243EB117312EBEA
:1021C000011243EB001343EC132A84EAD46080EA43
:1021D000451085EAD56181EA441180EA141080EA4D
:1021E000057081EA151181EA04711AEB903A4BEB04
:1021F000913B1AEB814A4BEB804B53EC122A82EA5B
:10220000080083EA090120402940504059401AEB58
:10221000000A5BEB010B51EC140AD0E904451AEB00
:10222000040A5BEB050BD1E904451AEB040A5BEBEE
:10223000050B16EB0A0657EB0B07D0E906451219FA
:102240006B41D1E9064512196B4155EC114A88EAF8
:10225000040089EA05013040394090EA080091EA1B
:10226000090112184B4186EAD66080EA471087EAD6
:10227000D76181EA461180EA161080EA077081EA88
:10228000171181EA067112EB903243EB913312EB96
:10229000814243EB804343EC122A53EC132A55EC62
:1022A000104A82EAD22080EA435083EAD32181EAAD
:1022B000425180EA921080EA836081EA931181EAB8
:1022C00082611AEB107A4BEB117B1AEB011A4BEB84
:1022D000001B82EA0C0112EA0C0201EA04005040E1
:1022E0001AEB000A01EA0A00504083EA0E0213EAE0
:1022F0000E0312EA050159405BEB010B02EA0B01E8
:10230000594053EC122AA4185D4145EC104A1218AA
:102310004B418AEADA2080EA4B508BEADB2181EAE2
:102320004A5180EA9A1080EA8B6081EA9B1181EA27
:102330008A6112EB107243EB117312EB011243EB43
:10234000001343EC122A84EAD46080EA451085EA3F
:10235000D56181EA441180EA141080EA057081EAAF
:10236000151181EA047118EB903849EB913918EB9B
:10237000814849EB804953EC112A82EA060083EA3E
:102380000701204029405040594018EB000859EB04
:10239000010951EC140AD0E9084518EB040859EB7F
:1023A0000509D1E9084518EB040859EB05091CEBB0
:1023B000080C5EEB090ED0E90A4512196B41D1E910
:1023C0000A4512196B4155EC104A86EA040087EA67
:1023D000050110EA0C0011EA0E0170407940121854
:1023E0004B418CEADC6080EA4E108EEADE6181EAC5
:1023F0004C1180EA1C1080EA0E7081EA1E1181EAFD
:102400000C7112EB903243EB913312EB814243EBB0
:10241000804343EC112A53EC122A55EC134A82EA0A
:10242000D22080EA435083EAD32181EA425180EAF4
:10243000921080EA836081EA931181EA826118EB4D
:10244000107849EB117918EB011849EB001982EA71
:102450000A0112EA0A0201EA0400504018EB0008DF
:1024600001EA0800504083EA0B0213EA0B0312EA68
:102470000501594059EB010902EA0901594053ECA1
:10248000112AA4185D4145EC134A12184B4188EA01
:10249000D82080EA495089EAD92181EA485180EA66
:1024A000981080EA896081EA991181EA886112EBCB
:1024B000107243EB117312EB011243EB001343EC68
:1024C000112A84EAD46080EA451085EAD56181EA60
:1024D000441180EA141080EA057081EA151181EA3E
:1024E000047116EB903647EB913716EB814647EBBC
:1024F000804753EC102A82EA0C0083EA0E01204048
:1025000029405040594036184F4151EC140AD0E947
:102510000C4536196F41D1E90C4536196F411AEB5C
:10252000060A5BEB070BD0E90E4512196B41D1E9A6
:102530000E4512196B4155EC134A8CEA04008EEAE1
:10254000050110EA0A0011EA0B0190EA0C0091EA79
:102550000E0112184B418AEADA6080EA4B108BEACE
:10256000DB6181EA4A1180EA1A1080EA0B7081EA85
:102570001B1181EA0A7112EB903243EB913312EB9B
:10258000814243EB804343EC102A53EC112A55EC73
:10259000124A82EAD22080EA435083EAD32181EAB8
:1025A000425180EA921080EA836081EA931181EAC5
:1025B000826116EB107647EB117716EB011647EBAD
:1025C000001782EA080112EA080201EA04005040FA
:1025D000361801EA0600504083EA090213EA0903AB
:1025E00012EA050159404F4102EA0701594053ECF4
:1025F000102AA4185D4145EC124A12184B4186EA94
:10260000D62080EA475087EAD72181EA465180EAFE
:10261000961080EA876081EA971181EA866112EB61
:10262000107243EB117312EB011243EB001343ECF6
:10263000102A84EAD46080EA451085EAD56181EAEF
:10264000441180EA141080EA057081EA151181EACC
:1026500004711CEB903C4EEB913E1CEB814C4EEB1D
:10266000804E53EC132A82EA0A0083EA0B012040D1
:102670002940504059401CEB000C5EEB010E51EC20
:10268000140AD0E910451CEB040C5EEB050ED1E9F1
:1026900010451CEB040C5EEB050E18EB0C0859EB17
:1026A0000E09D0E9124512196B41D1E912451219F0
:1026B0006B4155EC124A8AEA04008BEA050110EAE4
:1026C000080011EA090190EA0A0091EA0B011218C8
:1026D0004B4188EAD86080EA491089EAD96181EAE9
:1026E000481180EA181080EA097081EA191181EA1C
:1026F000087112EB903243EB913312EB814243EBC2
:10270000804343EC132A53EC102A55EC114A82EA19
:10271000D22080EA435083EAD32181EA425180EA01
:10272000921080EA836081EA931181EA82611CEB56
:10273000107C4EEB117E1CEB011C4EEB001E82EA5E
:102740000601324001EA040050401CEB000C01EA93
:102750000C00504083EA07023B4012EA0501594051
:102760005EEB010E02EA0E01594053EC132AA41845
:102770005D4145EC114A12184B418CEADC2080EA9D
:102780004E508EEADE2181EA4C5180EA9C1080EAAC
:102790008E6081EA9E1181EA8C6112EB107243EB2C
:1027A000117312EB011243EB001343EC132A84EA7A
:1027B000D46080EA451085EAD56181EA441180EA57
:1027C000141080EA057081EA151181EA04711AEB90
:1027D000903A4BEB913B1AEB814A4BEB804B53EC1D
:1027E000122A82EA080083EA090120402940504069
:1027F00059401AEB000A5BEB010B51EC140AD0E9CB
:1028000014451AEB040A5BEB050BD1E914451AEBEE
:10281000040A5BEB050B16EB0A0657EB0B07D0E936
:10282000164512196B41D1E9164512196B4155EC49
:10283000114A88EA040089EA05013040394090EAEB
:10284000080091EA090112184B4186EAD66080EA35
:10285000471087EAD76181EA461180EA161080EABC
:10286000077081EA171181EA067112EB903243EB8F
:10287000913312EB814243EB804343EC122A53EC39
:10288000132A55EC104A82EAD22080EA435083EAA8
:10289000D32181EA425180EA921080EA836081EA82
:1028A000931181EA82611AEB107A4BEB117B1AEBE0
:1028B000011A4BEB001B82EA0C0112EA0C0201EA3E
:1028C000040050401AEB000A01EA0A00504083EA73
:1028D0000E0213EA0E0312EA050159405BEB010BED
:1028E00002EA0B01594053EC122AA4185D4145EC51
:1028F000104A12184B418AEADA2080EA4B508BEAE0
:10290000DB2181EA4A5180EA9A1080EA8B6081EAF1
:102910009B1181EA8A6112EB107243EB117312EB87
:10292000011243EB001343EC122A84EAD46080EADC
:10293000451085EAD56181EA441180EA141080EAE5
:10294000057081EA151181EA047118EB903849EBA2
:10295000913918EB814849EB804953EC112A82EAFE
:10296000060083EA0701204029405040594018EBF7
:10297000000859EB010951EC140AD0E9184518EB8D
:10298000040859EB0509D1E9184518EB040859EB7F
:1029900005091CEB080C5EEB090ED0E91A4512196B
:1029A0006B41D1E91A4512196B4155EC104A86EA80
:1029B000040087EA050110EA0C0011EA0E017040DC
:1029C000794012184B418CEADC6080EA4E108EEAA6
:1029D000DE6181EA4C1180EA1C1080EA0E7081EA07
:1029E0001E1181EA0C7112EB903243EB913312EB22
:1029F000814243EB804343EC112A53EC122A55ECFD
:102A0000134A82EAD22080EA435083EAD32181EA42
:102A1000425180EA921080EA836081EA931181EA50
:102A2000826118EB107849EB117918EB011849EB2A
:102A3000001982EA0A0112EA0A0201EA040050407F
:102A400018EB000801EA0800504083EA0B0213EA81
:102A50000B0312EA0501594059EB010902EA090189
:102A6000594053EC112AA4185D4145EC134A121841
:102A70004B4188EAD82080EA495089EAD92181EA85
:102A8000485180EA981080EA896081EA991181EAC8
:102A9000886112EB107243EB117312EB011243EBDE
:102AA000001343EC112A84EAD46080EA451085EAD9
:102AB000D56181EA441180EA141080EA057081EA48
:102AC000151181EA047116EB903647EB913716EB3E
:102AD000814647EB804753EC102A82EA0C0083EAD8
:102AE0000E01204029405040594036184F4151ECCA
:102AF000140AD0E91C4536196F41D1E91C45361935
:102B00006F411AEB060A5BEB070BD0E91E45121961
:102B10006B41D1E91E4512196B4155EC134A8CEA01
:102B200004008EEA050110EA0A0011EA0B0190EA9E
:102B30000C0091EA0E0112184B418AEADA6080EA31
:102B40004B108BEADB6181EA4A1180EA1A1080EAB5
:102B50000B7081EA1B1181EA0A7112EB903243EB90
:102B6000913312EB814243EB804343EC102A53EC48
:102B7000112A55EC124A82EAD22080EA435083EAB5
:102B8000D32181EA425180EA921080EA836081EA8F
:102B9000931181EA826116EB107647EB117716EB01
:102BA000011647EB001782EA080112EA080201EA5F
:102BB00004005040361801EA0600504083EA09023A
:102BC00013EA090312EA050159404F4102EA0701DD
:102BD000594053EC102AA4185D4145EC124A1218D2
:102BE0004B4186EAD62080EA475087EAD72181EA1E
:102BF000465180EA961080EA876081EA971181EA5F
:102C0000866112EB107243EB117312EB011243EB6E
:102C1000001343EC102A51EC140A803004EE100A21
:102C2000A1F14001A1EC020AC0C1A1EC021AA1E885
:102C30000003A1EC022AA1E8000CA1EC023AA1E8F1
:102C40000050BDE8009000BF00B59CE8F00FDCE943
:102C50001201DCE91C23241845EB01054FEA560E4E
:102C60008EEAC77E8EEA162E8EEA076E8EEAD61E92
:102C70008EEA476E14EB0E044FEA570E8EEAC67EBC
:102C80008EEA172E8EEA066E8EEAD71E45EB0E05EB
:102C90004FEAD24E8EEA433E8EEAC20E8EEA537E51
:102CA0008EEA921E8EEA836E14EB0E044FEAD34E28
:102CB0008EEA423E8EEAC30E8EEA527E8EEA931E62
:102CC00045EB0E05DCE91401DCE91E23361847EB61
:102CD00001074FEA580E8EEAC97E8EEA182E8EEA58
:102CE000096E8EEAD81E8EEA496E16EB0E064FEA82
:102CF000590E8EEAC87E8EEA192E8EEA086E8EEA8A
:102D0000D91E47EB0E074FEAD24E8EEA433E8EEABB
:102D1000C20E8EEA537E8EEA921E8EEA836E16EB08
:102D20000E064FEAD34E8EEA423E8EEAC30E8EEA7C
:102D3000527E8EEA931E47EB0E07DCE9160118EB74
:102D4000000849EB01094FEA5A0E8EEACB7E8EEA63
:102D50001A2E8EEA0B6E8EEADA1E8EEA4B6E18EB96
:102D60000E084FEA5B0E8EEACA7E8EEA1B2E8EEAB2
:102D70000A6E8EEADB1E49EB0E094FEAD44E8EEA4C
:102D8000453E8EEAC40E8EEA557E8EEA941E8EEA89
:102D9000856E18EB0E084FEAD54E8EEA443E8EEA59
:102DA000C50E8EEA547E8EEA951E49EB0E09DCE9CB
:102DB0001801DCE908231AEB000A4BEB010B4FEA80
:102DC000520E8EEAC37E8EEA122E8EEA036E8EEAD1
:102DD000D21E8EEA436E1AEB0E0A4FEA530E8EEAAB
:102DE000C27E8EEA132E8EEA026E8EEAD31E4BEB63
:102DF0000E0B4FEAD64E8EEA473E8EEAC60E8EEA9C
:102E0000577E8EEA961E8EEA876E1AEB0E0A4FEAFE
:102E1000D74E8EEA463E8EEAC70E8EEA567E8EEA80
:102E2000971E4BEB0E0BACE8F00FDCE91201DCE96E
:102E30000267121843EB01034FEA560E8EEAC77E73
:102E40008EEA162E8EEA076E8EEAD61E8EEA476E40
:102E500012EB0E024FEA570E8EEAC67E8EEA172E4E
:102E60008EEA066E8EEAD71E43EB0E034FEAD84E6B
:102E70008EEA493E8EEAC80E8EEA597E8EEA981E88
:102E80008EEA896E12EB0E024FEAD94E8EEA483E68
:102E90008EEAC90E8EEA587E8EEA991E43EB0E0327
:102EA000DCE91401DCE90489361847EB01074FEA35
:102EB000580E8EEAC97E8EEA182E8EEA096E8EEAC8
:102EC000D81E8EEA496E16EB0E064FEA590E8EEAB0
:102ED000C87E8EEA192E8EEA086E8EEAD91E47EB5E
:102EE0000E074FEADA4E8EEA4B3E8EEACA0E8EEAA3
:102EF0005B7E8EEA9A1E8EEA8B6E16EB0E064FEA0A
:102F0000DB4E8EEA4A3E8EEACB0E8EEA5A7E8EEA7F
:102F10009B1E47EB0E07DCE91601DCE906AB18EB5C
:102F2000000849EB01094FEA5A0E8EEACB7E8EEA81
:102F30001A2E8EEA0B6E8EEADA1E8EEA4B6E18EBB4
:102F40000E084FEA5B0E8EEACA7E8EEA1B2E8EEAD0
:102F50000A6E8EEADB1E49EB0E094FEAD24E8EEA6C
:102F6000433E8EEAC20E8EEA537E8EEA921E8EEAAF
:102F7000836E18EB0E084FEAD34E8EEA423E8EEA7D
:102F8000C30E8EEA527E8EEA931E49EB0E09DCE9EF
:102F900008011AEB040A4BEB050B4FEA500E8EEAC0
:102FA000C17E8EEA102E8EEA016E8EEAD01E8EEA67
:102FB000416E1AEB0E0A4FEA510E8EEAC07E8EEA7F
:102FC000112E8EEA006E8EEAD11E4BEB0E0B4FEAED
:102FD000D64E8EEA473E8EEAC60E8EEA577E8EEABF
:102FE000961E8EEA876E1AEB0E0A4FEAD74E8EEACD
:102FF000463E8EEAC70E8EEA567E8EEA971E4BEB51
:103000000E0BACE8CC0F5CE90E45DCE90267001959
:1030100041EB05014FEA560E8EEAC77E8EEA162E68
:103020008EEA076E8EEAD61E8EEA476E10EB0E0011
:103030004FEA570E8EEAC67E8EEA172E8EEA066E8D
:103040008EEAD71E41EB0E014FEAD84E8EEA493E7A
:103050008EEAC80E8EEA597E8EEA981E8EEA896E36
:1030600010EB0E004FEAD94E8EEA483E8EEAC90EAA
:103070008EEA587E8EEA991E41EB0E015CE90C4502
:10308000DCE90489361947EB05074FEA580E8EEA4A
:10309000C97E8EEA182E8EEA096E8EEAD81E8EEA56
:1030A000496E16EB0E064FEA590E8EEAC87E8EEA7E
:1030B000192E8EEA086E8EEAD91E47EB0E074FEAEC
:1030C000DA4E8EEA4B3E8EEACA0E8EEA5B7E8EEABE
:1030D0009A1E8EEA8B6E16EB0E064FEADB4E8EEAD8
:1030E0004A3E8EEACB0E8EEA5A7E8EEA9B1E47EB54
:1030F0000E075CE90A45DCE906AB18EB040849EB6E
:1031000005094FEA5A0E8EEACB7E8EEA1A2E8EEA17
:103110000B6E8EEADA1E8EEA4B6E18EB0E084FEA43
:103120005B0E8EEACA7E8EEA1B2E8EEA0A6E8EEA4D
:10313000DB1E49EB0E094FEAD04E8EEA413E8EEA85
:10314000C00E8EEA517E8EEA901E8EEA816E18EBDA
:103150000E084FEAD14E8EEA403E8EEAC10E8EEA4C
:10316000507E8EEA911E49EB0E09DCE908451AEB08
:10317000020A4BEB030B4FEA540E8EEAC57E8EEA31
:10318000142E8EEA056E8EEAD41E8EEA456E1AEB78
:103190000E0A4FEA550E8EEAC47E8EEA152E8EEA8E
:1031A000046E8EEAD51E4BEB0E0B4FEAD64E8EEA1E
:1031B000473E8EEAC60E8EEA577E8EEA961E8EEA4D
:1031C000876E1AEB0E0A4FEAD74E8EEA463E8EEA1B
:1031D000C70E8EEA567E8EEA971E4BEB0E0BACE8BE
:1031E000C30F5CE90E23DCE90267A41845EB030575
:1031F0004FEA560E8EEAC77E8EEA162E8EEA076ECC
:103200008EEAD61E8EEA476E14EB0E044FEA570E76
:103210008EEAC67E8EEA172E8EEA066E8EEAD71EDC
:1032200045EB0E054FEAD84E8EEA493E8EEAC80EAF
:103230008EEA597E8EEA981E8EEA896E14EB0E0491
:103240004FEAD94E8EEA483E8EEAC90E8EEA587E83
:103250008EEA991E45EB0E055CE90C23DCE9048936
:10326000B61847EB03074FEA580E8EEAC97E8EEA7E
:10327000182E8EEA096E8EEAD81E8EEA496E16EB7B
:103280000E064FEA590E8EEAC87E8EEA192E8EEA95
:10329000086E8EEAD91E47EB0E074FEADA4E8EEA29
:1032A0004B3E8EEACA0E8EEA5B7E8EEA9A1E8EEA4C
:1032B0008B6E16EB0E064FEADB4E8EEA4A3E8EEA26
:1032C000CB0E8EEA5A7E8EEA9B1E47EB0E075CE918
:1032D0000A23DCE906AB18EB020849EB03094FEAC5
:1032E0005A0E8EEACB7E8EEA1A2E8EEA0B6E8EEA8C
:1032F000DA1E8EEA4B6E18EB0E084FEA5B0E8EEA72
:10330000CA7E8EEA1B2E8EEA0A6E8EEADB1E49EB1F
:103310000E094FEAD44E8EEA453E8EEAC40E8EEA7E
:10332000557E8EEA941E8EEA856E18EB0E084FEAE3
:10333000D54E8EEA443E8EEAC50E8EEA547E8EEA63
:10334000951E49EB0E095CE918231AEB000A4BEBBA
:10335000010B4FEA520E8EEAC37E8EEA122E8EEADF
:10336000036E8EEAD21E8EEA436E1AEB0E0A4FEA05
:10337000530E8EEAC27E8EEA132E8EEA026E8EEA1B
:10338000D31E4BEB0E0B4FEAD64E8EEA473E8EEA2B
:10339000C60E8EEA577E8EEA961E8EEA876E1AEB6E
:1033A0000E0A4FEAD74E8EEA463E8EEAC70E8EEAE6
:1033B000567E8EEA971E4BEB0E0B8CE8F00FACF1AD
:1033C000600C00BD2DE9F04F04EE101A00F1400C26
:1033D000B0E8F807ACE8F807B0E8F807ACE8F80799
:1033E000FEF71EFEFFF730FCFEF71AFEFFF72CFC7F
:1033F000FEF716FEFFF728FCFEF712FEFFF724FC8F
:10340000FEF70EFEACF1800808F1400998E80F0CB9
:10341000B9E8F0500019694192197B411AEB0C0A86
:103420004BEB0E0BA8E80F0C98E80F0CB9E8F05026
:103430000019694192197B411AEB0C0A4BEB0E0BF8
:10344000A8E80F0C98E80F0099E8F000001969410E
:1034500092197B4188E80F00BDE8F08F1FB5144C2E
:10346000207A8DF80100E0798DF80000A079ADF8A0
:1034700004006079ADF80200684606F02BF908B147
:10348000A72110E0E068029002A806F039F908B11F
:10349000AB2108E007480068039003A80FF0F1FA99
:1034A000002803D0AF21032000F0DCF81FBD00008E
:1034B000202400206C37000010B528B114220449E4
:1034C00010F059FA002010BD6FF0150010BD00007B
:1034D0009037000070B56FF02C03B8BB1E4C6078BD
:1034E00008B1981170BD01B36FF01505AAB11B4862
:1034F000891E06292BD2DFE801F0030616192A1CC3
:103500001178417017E0917839B1D17829B11178EB
:103510001B2902D351781B2901D2284670BD11689E
:10352000C0F8051007E01168C16004E011788170EF
:1035300001E0118841820122084900200BF0D4FEED
:10354000B0F5803F05DB6FF00B0070BDFFE718465C
:10355000FBE70121A170F8E72800002020240020CB
:1035600010B5074C607820B106F0A8FB20780BF06E
:1035700079FC00F087FD00F05FFE0020607010BD58
:103580002800002070B50C46050002D00CB1600781
:1035900002D06FF0150070BD00F020F9A8B12846E8
:1035A0000BF026FC0A4D00220A49287020460BF039
:1035B0009BFE0FF087FE0021287806F069FBFFF7DD
:1035C0004DFF01206870002070BD4FF0FF3070BDCE
:1035D000280000202024002030B589B004000CD041
:1035E0000BF0ACFB4FF0FF3520B10BF03FFAB0F51C
:1035F000FA7F05D9284609B030BD6FF01500FAE70B
:10360000134D14486C6000F00BFA00206870A8702D
:1036100001462022684610F028FA20220E4968460A
:1036200010F0A9F9202269460C4810F0A4F9EFF334
:10363000108472B600F034FD094800F009FE18B19C
:10364000C521032000F00EF804B962B60020D2E7CD
:10365000280000205D340000703700002024002086
:10366000093800000EB572B6154A5568DDB1002262
:1036700003466E460A2403E0B0FBF4F0521CD2B2BB
:103680000028F9D1B0540AE0D8B2B0FBF4F7B3FB8C
:10369000F4F304FB1700521ED2B23030B054002AAB
:1036A000F2D13046A847BFF34F8F06480168064A5B
:1036B00001F4E06111430160BFF34F8F00BFFDE7EC
:1036C000280000200CED00E00400FA05064810B5C3
:1036D00081784078014302D04FF0FF3010BD06F0F2
:1036E000FDFA002010BD000028000020064810B59B
:1036F00081784078014302D04FF0FF3010BD06F0D2
:103700004BF8002010BD000028000020064810B52E
:1037100081784078014302D04FF0FF3010BD0FF0A8
:103720004FFB002010BD000028000020064810B507
:1037300081784078014302D04FF0FF3010BD06F091
:10374000DFFA002010BD000028000020064810B558
:1037500081784078014302D04FF0FF3010BD0FF068
:103760003FFB002010BD00002800002001000000E9
:1037700000010100001B1B03020000004C1D0000A3
:1037800000001F000000000000000000000000001A
:10379000D80C2D2F36AEE25C8026804C3F4D165360
:1037A0005096C773054A10B5526812B1BDE8104073
:1037B000104792210420FFF755FF0000402400200D
:1037C000054A10B5926812B1BDE810401047982123
:1037D0000420FFF747FF000040240020054801684F
:1037E00029B1416819B1806808B1012070470020F3
:1037F000704700004024002002490DC881E80D00F8
:103800000020704740240020F8B5124C002625689F
:1038100011E00098022802D003280CD106E02068AD
:1038200010B10020266005E028210CE0206868B176
:1038300001202660A847684600F0D0FC0028E8D0A8
:10384000052805D035210420FFF70CFF2D21FAE7CC
:10385000F8BD0000300000202DE9FC41254E054652
:10386000001D06F144073060387858B1BA783C46FC
:10387000791C2846921C10F07EF80020207004204D
:10388000BDE8FC811B4801F05DFF0446022804D01E
:10389000042C07D0082C27D02AE0164928460BF024
:1038A000C3FD25E03078082804D105213E200BF027
:1038B0008DFD60B10F4928460BF01BFE0028D3D0C8
:1038C000A97828780BF082FD0028CDD010E0B088D0
:1038D000ADF8000001A968460CF0FAF80028C3D042
:1038E000A7210820FFF7BEFE024928460BF0CAFDBB
:1038F0002046C5E74C24002070B50A7882703AB3A0
:10390000012A25D81323037000230AE001EB4304A6
:1039100000EB4305A678EE706488240A5B1C2C71CA
:10392000DBB29342F2D300230BE000BF01EB43056F
:1039300000EB43042E796671AD882D0A5B1CA571DE
:10394000DBB29342F2D3012101EB8200C0B270BD21
:10395000002070BD402803D2401EC1B2054805E0DA
:10396000FF2805D04038C1B2024808300BF0A3BF91
:10397000012070473C000020401EC1B201480BF0FE
:103980009ABF00004C00002010B5074A0168064BA2
:1039900091614068D0611C681832A1431160596878
:1039A0008843506010BD000034000020064A0168C2
:1039B00091604068D060083241F48C211160034965
:1039C000084350607047000034000020F8074002B0
:1039D000024902680A61406848617047340000206B
:1039E00007484FF0FF3100220160C90C416000F12F
:1039F00008011F200A604A600831C1E900027047CF
:103A00003C00002010B5FFF7EBFF0FF052F9044621
:103A10000248006800B18047204610BD54000020D5
:103A20000149086070470000540000200221018015
:103A3000418000210171D821417142F60C51C180B1
:103A400001498160002070472F36AEE210B5022890
:103A500004D340F203211720FFF704FE0149085C5C
:103A600010BD000094250020F8B5050000950DD08C
:103A70000026087849780446A14200D90C46AA07D6
:103A800006D04FF4E5711720FFF7ECFD0126F0E7B3
:103A9000124F387079703146684600F0D3F8002133
:103AA0000B460098C01C20F00300009066B907EB9D
:103AB0008102D060002005E0D2F80CC04CF8203024
:103AC000401CC0B2A042F7D30098491C00EB840010
:103AD000C9B200900229E4D3401BF8BD9425002010
:103AE00070B50446857900F0E9F80C4AE17902EBFB
:103AF00085020EE0D36853F8213043B1481CE071D1
:103B0000A180D06850F821002060002070BD491CC1
:103B1000C9B28142EED3E171052070BD9425002029
:103B2000F0B421B1012902D0F0BC002070470F4A47
:103B300000252B464FF6FF7402EB8106575C0AE026
:103B40005A19D6F80CC092B25CF822C0BCF1000F32
:103B500004D05B1C9BB29F42F2D8224602801046E2
:103B6000A242E1D0F0BC00F035B80000942500205E
:103B70002DE9F0410646A0F57F400C4643F20207CE
:103B8000FF3820D0022C02D30720BDE8F081304658
:103B900000F048F8050016D00C48294650F82420BB
:103BA000304690470A48002100EB8407F86840F847
:103BB0002610204600F078F80246294678680CF076
:103BC0001FFA0020E1E73846DFE70000D43C0000A0
:103BD0009425002070B50E4605460CF04BFA58B1FE
:103BE0000F4800EB8604E06850F8250038B14FF428
:103BF000C5711720FFF736FD40F28911F9E76068BB
:103C000000280BD0304600F04FF8014660680CF0F9
:103C10009FF9002802D0E16841F8250070BD00003E
:103C20009425002070B50C4605460CF023FA0028B8
:103C300005D0034800EB8400C06850F8250070BD33
:103C4000942500202DE9F843164E884605460024A9
:103C50002868C01C20F003002860204600F024F8EB
:103C6000315D4843B8F1000F01D0002200E02A681E
:103C70000146009232B100274FEA0D000CF099F98D
:103C80001FB106E001270020F8E706EB8401009A47
:103C90004A602968641C0844E4B22860022CD7D327
:103CA000BDE8F88394250020034931F810004FF651
:103CB000FC71C01C08407047D03C000003490878E4
:103CC0004978884200D208467047000094250020B9
:103CD000F8021801711D01001B1301002DE9FF4FAF
:103CE000244C064681B020689A46934658B1017A22
:103CF000B14203D9406850F8260040B143F20200B7
:103D000005B0BDE8F08FA5211820FFF7ABFC1946E0
:103D100002980CF0D2F9804658460E990CF0C3F97F
:103D2000054608EB0500001D87B22068A14639460C
:103D300000680CF00DF904001AD067802580294630
:103D4000201D0E9D07465A46092300950CF07AF86F
:103D50002088414638440A23029ACDF800A00CF08E
:103D600071F8D9F80000406840F826400020C7E705
:103D70000420C5E75800002070B5144C23688BB1AF
:103D8000197A814212D95A6852F8201071B100256F
:103D900042F820504A8818680CF032F92168002057
:103DA0000A7A0CE0C6211820FFF75CFC43F20200FF
:103DB00070BD4B6853F8203033B9401CC0B282420A
:103DC000F7D808680CF011F9002070BD58000020E9
:103DD0002DE9F0410D46040090464FF0000606D054
:103DE0000027A00705D086211820FFF73BFC0127FC
:103DF000F7E7CDB1114600200CF0DBF80C3000EBFA
:103E000085068FB90A4F04F10C00AA003C602572A8
:103E1000606000EB85002060002160680FF025FEE7
:103E2000414638680CF0C5F83046BDE8F081000026
:103E30005800002070B5084D286800280AD00024DA
:103E400004E02046FFF798FF641CE4B22868007A7B
:103E5000A042F6D870BD000058000020094910B5F6
:103E600002460968002049B10B7A934205D9496896
:103E700051F82210002900D0081D10BDEC21182097
:103E8000FFF7F0FB580000200A4910B50246096808
:103E9000002059B10B7A934207D9496851F8221092
:103EA000002902D031F8040B084410BDFA21182073
:103EB000FFF7D8FB5800002070B51E4B456804463C
:103EC0000022A1B101206070588881085FF00000D5
:103ED00004EB400304EB80061A83198400FB0153B2
:103EE00073602318401C1A750428F1D370BD6270EA
:103EF0005FF0000004EB40010A830A8404EB8001B8
:103F00004A602118401C0A750428F3D35888B0F57C
:103F1000FF7F01D2460800E0FF260CF042F9656001
:103F200020842918A1606684E560A0842161E6846C
:103F300070BD00005C0000202DE9F04158B1002563
:103F40001144244ECCB200273470810705D04E2195
:103F50000920FFF787FB0125F2E71F2B04D84FF656
:103F6000FF7101EA830109E05900FF2B0CD903F12D
:103F7000FF02B2EB430F00D2114689B24FF6FC723A
:103F8000C91C114035B107E07C22B2EB430FF4D3DA
:103F90007C21F2E77060718004EB840207EBC203BE
:103FA000002276684FF0010C0DE04DB902EB82075C
:103FB00000EB030E06F837C006EBC707C7F804E0AE
:103FC000521C0B44D2B2A242EFD3DB1D23F00700F8
:103FD000BDE8F0815C00002070B5104A00205168F7
:103FE000127814E000EB800311F833306BB100EB72
:103FF000800011EBC0040CD00025A57001212046E3
:10400000FFF75AFF2570204670BD401CC0B2904299
:10401000E8D3A9210920FFF725FB00005C00002060
:10402000044810B5408884080CF0BBF8844200D3E3
:10403000204610BD5C00002030B50D4901204860CD
:10404000821EC1F808230B4988600023C1F80032A2
:10405000C1F80823084C2360251D28608860C1F83A
:1040600008232360286006490448086030BD00002A
:1040700000E0004000F0004000F500400000F63F86
:1040800008F5014010B5FFF7D7FF0CF061F90349BF
:104090000148086010BD00000000F63F08F501402F
:1040A00010B5FFF7C9FF0CF053F900F087F8054988
:1040B0000348086000F0B8F8BDE8104000F0DCB834
:1040C0000000F63F08F501402DE9F84F82463848D8
:1040D0000FF06FFBDFF8D8B028B101260BF101001B
:1040E000FF21017000E000264FF48075314C4FF045
:1040F00000082F1D01216160C4F80081C4F804810B
:10410000C4F804A52160DFF8B0901CE0D9F80000E5
:10411000C00618D50E200CF02AF9EFF3108000909D
:1041200072B603212046C4F8041329460CF02CF97A
:1041300030B9394620460CF027F908B90FF0D0FB0A
:10414000009800B962B6294620460CF01DF928B93E
:10415000394620460CF018F90028D7D039462046B9
:104160000CF012F90028C5D106BB9BF801108DF8A0
:104170000010009900919DF8001009B1012500E0A0
:1041800000250BF1010080F800800320C4F808032B
:10419000C4F80481C4F800810E200CF0E8F804484B
:1041A0000FF01EFB15B11120BDE8F88F0020FBE7D2
:1041B0006003002000E0004010ED00E010B506486C
:1041C0000FF00AFB18B127211D20FFF74BFA024818
:1041D0000021417010BD00006003002070B511493E
:1041E0000A68EAB100231D4601244A68521C4A604D
:1041F000092A00D34D600E7904FA06F20E681642C1
:104200000BD0EFF3108372B60C6894430C6003B9C3
:1042100062B649680160002070BD5B1C092BE4D3C5
:10422000052070BD6400002002480021016041604B
:10423000704700006400002010B5044C2078FF286F
:1042400003D00AF00FFEFF20207010BD00000020F8
:1042500010B5084C617809B10F2010BD0AF0C8FDF7
:104260002070FF2801D0002010BD73211F20FFF710
:10427000F9F9000000000020014900204870704753
:10428000000000200648074A818C5288914204D1E0
:1042900090F8220008B1002070470120704700000C
:1042A000B82A00204C0300200149488070470000D4
:1042B0004C0300200848094A818C5288914209D158
:1042C0004FF6FF71818410F8221F19B1002101708F
:1042D0000120704700207047B82A00204C030020BE
:1042E000074810F8221F012907D001210170054855
:1042F000034900888884012070470020704700002F
:10430000B82A00204C0300200649074B8A8C5B88A2
:104310009A4205D191F8222012B101600120704724
:1043200000207047B82A00204C03002009498A8CDD
:10433000A2F57F43FF3B02D00021016007E091F826
:1043400022200449012A02D0016001207047002088
:1043500070470000B82A002001490880704700001B
:104360004C0300200549002081F822004FF6FF7021
:10437000888403490880488070470000B82A0020DC
:104380004C03002005498A8C824205D1002081F827
:1043900022004FF6FF70888470470000B82A002082
:1043A0000A4A10B1012807D00EE0507860B1D2F867
:1043B00002000860D08804E0107828B19068086096
:1043C0009089888001207047002070476203002098
:1043D000084A012338B1012804D11370086890609D
:1043E00088889081704753700868C2F802008888F6
:1043F000D080704762030020064910B1012802D026
:1044000005E0487800E0087808B1012070470020F6
:1044100070470000620300200149087770470000E0
:10442000FA23002001488078704700006C000020CB
:104430000148C078704700006C00002070B50C4641
:10444000054600F01FF918B1D0212720FFF70AF91F
:10445000034801210CF0D1FB0248C0E90B5470BDA8
:10446000D82300206C0000200149012048717047CA
:104470006C0000202DE9F84F5B4D0A9C2E78002E31
:104480006BD1002A69D0002B67D0002C65D005F1D4
:104490001406C5E90F0186E81C0000276F712F7113
:1044A000AF706F70EF70AF81EF8100F03DF906469D
:1044B00000F034F9044606F085F805F0DDFD94F9C6
:1044C0006E0006F003F9E06906F0E6F9606906F0AF
:1044D000D9F996F8330006F00FFA05F13C00406870
:1044E00090F81A0208B105F0EDFF94F86B10012066
:1044F00005F02CFF002870D03C4805F093FF208881
:10450000FFF7C2FC68632088FFF7A8FC06F1880269
:10451000A86392E80C11DFF8D89089E80C11D6F85E
:104520009820C9F81920D6F89C10C9F81D1000F081
:1045300033F90146208FBA460CF0BCF8A18E8142B7
:1045400000D20846A871A84694F86B10E08F96F840
:104550002370A58F082904D102E040F2451140E004
:1045600004210CF0A7F80FB9001D80B2854200D2DB
:104570002846C5B288F8075088F8085096F82300F6
:10458000D04690B1012789F81870D6E92012C9E900
:10459000041294F86B000BF083FF03462A4614497B
:1045A0003846CDF8008005F0D3FC012000F054FB24
:1045B00010480068032812D00B2810D00C480E2297
:1045C00000214A300FF051FA0948B18A4A3041803F
:1045D0002188018096F833100171BDE8F88F40F210
:1045E00002212720FFF73EF86C0000205C4E0000FF
:1045F000B0230020501500402DE9FC4188460746B5
:1046000000F092F81A4C0546B807616A4E7816D544
:10461000A06A30B36289D21C0FF0ADF9A06A606263
:10462000694601AAA06B0BF08AFB00980BF03DFBDA
:10463000C8F8000031460122A06B0BF0EDFAF80734
:104640000DD0D5E920011835401C41F10001C5E924
:104650001A0115F81809012808D001202876BDE8AC
:10466000FC8140F266412720FEF7FCFF0020F5E7C1
:104670006C0000200248C089C0F380207047000011
:104680006C0000200448007808B10C2070470349F2
:1046900000200877704700006C000020FA230020FB
:1046A0000C4810B5017849B100F13C0100780228AE
:1046B00008D040F21E212720FEF7D4FFBDE81040AD
:1046C00000F0D8B94868D0F83002BDE8104005F0D5
:1046D000B1BE00006C000020F8B5002605464E7003
:1046E0001D20094F0C4608702E720E223946201DDF
:1046F0000FF041F9287A8DF80000009800909DF89D
:1047000000000028F0D1F8BD08240020024A938957
:1047100003439381526910476C00002001484068B0
:1047200070470000A80000200148406880307047B2
:10473000A8000020014A0021526910476C000020A7
:1047400070B50546012918D8124CA1698847A0B157
:10475000207990B9E5B904F110000178C80605D4B4
:10476000E06A0078C00601D4012000E00020A26ABF
:104770002AB962891AB1C90601D4012070BDA18984
:104780008A0703D5226AD278022A01D00843F4D1DD
:10479000002070BD6C00002010B5FFF7BFFF04467D
:1047A000FFF7C2FF0246417F1648252910D026296F
:1047B0000ED0927F252A0BD020290DD021290BD095
:1047C000232A0FD094F86A00042800D1082010BDD5
:1047D000406890F8CE120EE0232A03D0406890F88B
:1047E0003E0105E0416891F83E0191F863100840F0
:1047F0000BF04CFE014694F86A00BDE810400BF047
:104800005DBE0000A80000202DE9FF5F8B468146B9
:10481000FFF78AFF0026664C07468DF8086003966E
:10482000019620783546022804D040F2EA4127203C
:10483000FEF718FFA07B400606D44020FFF77AFF62
:10484000E08940F04000E08197F82300B9F1000FC3
:104850003AD080B105F04AFC05F024FC58B9606AF2
:10486000417841B10078397EC0F3C000884202D15E
:104870000120607097E0606A4178618121B1A06B8E
:104880000BF033FBA06200E0A562E08940F4807089
:10489000E081606AF97D0078C0F38000884207D02B
:1048A00003A800F08BF9E08940F48060E08100E02B
:1048B0000126606A397E0078C0F3C00088420DD1BD
:1048C00002A800F031F909E008B105F009FCA07870
:1048D000401CA070E08940F40070E081DFF8D0A0B7
:1048E00097F822000AF13C0A90B1FFF717FF31490F
:1048F0000D76D7E91E23C1E9042390F86A000BF076
:10490000CFFD0346FB222B492846009505F020FBEE
:104910004FF00008BBF1000F04D1A1780120FFF790
:104920000FFF20B105F09AFF4FF0010802E00020D0
:1049300000F0D0F99DF8080018B101A90220FFF796
:104940005BFE1C48BA8A4A303EB11AB9C2880AB91D
:10495000028912B14289521C4281B9F1000F08D07C
:10496000C188491CC1801248A5703C3001F03EFA54
:1049700002E00189491C0181039840B10BF095F9CF
:10498000DAF80410401C05720E220CF0B4F90198FC
:1049900030B1DAF8041005722A2201980CF0ABF954
:1049A000B8F1000F01D000F065F8BDE8FF9F0000EE
:1049B0006C000020B02300202DE9F8438846814692
:1049C000FFF7B2FE294D04462878012804D040F2B2
:1049D00075412720FEF746FE207C0027012628B1DE
:1049E000277400210420FFF791FEA674296A087835
:1049F000C043800709D1A07D88BB0220FFF786FE57
:104A0000286A0078C043800729D0286A407810B10E
:104A10000220A07500E0A67594F8230098B1FFF776
:104A20007DFE13492D7A0E76D4E92023C1E90423B3
:104A300090F86B000BF034FD03462A460C493046D3
:104A4000009705F085FA38EA090004D000210846ED
:104A5000FFF776FE28B1BDE8F84300F00BB803205D
:104A6000D7E7BDE8F843002000F0F6B86C0000205E
:104A7000B023002010B505F0DFFB05F0FDFA0D4C6A
:104A8000E089FFF757FE0C48007F58B10A490E2213
:104A900001F10E000EF06FFF0748242207491D3078
:104AA0000CF03DF9E2692179607890470020207090
:104AB00010BD00006C000020FA230020D946000041
:104AC000084810B50078022804D040F24D21272074
:104AD000FEF7C8FD044901200873BDE81040FFF748
:104AE000C9BF00006C000020FA23002030B4044647
:104AF0000C48007A0BB1001DC0B23AB9FF2805D1AD
:104B000094F86B2094F86A309A4209D021B194F855
:104B10006B1030BC05F0C6BEFF2094F86A10F8E7B1
:104B200030BC70476C0000202DE9F0410746FFF7CC
:104B3000FBFD214C05460126616A087800F0030060
:104B400001280CD002280AD003281BD12E74E0893A
:104B500040F40060E0810120FFF7D8FD12E04878C2
:104B600080B1E18941F40061E181A16A002918D096
:104B7000FB2818D8607920B1BDE8F0412020FFF76C
:104B8000D9BD3E70287E012812D02E76606A40780A
:104B9000002806D0F5E92001401C41F10001C5E9DB
:104BA0000001BDE8F081207940F010002071F8E7A5
:104BB00000202876EAE700006C00002070B505466A
:104BC000FFF7B2FD0446807D00282DD002280CD1CD
:104BD0001B482946406B0AF0F7FF30B3D4E91E01A9
:104BE000401C41F10001C4E91E010025A575A07C0F
:104BF00020B1A57400211020FFF788FD607C70B102
:104C00006574FFF757FB98B100210820FFF77EFD80
:104C1000D4E91E01401C41F10001C4E91E01E07D00
:104C200001280AD00120E07570BD40F2E33101E0B7
:104C300040F2FA312720FEF715FDE57570BD000042
:104C40006C00002003480078002801D0FFF712BF55
:104C5000704700006C0000202DE9F0410646FFF788
:104C60005DFD8046FFF760FD184C05463246E06A60
:104C7000606295F8233001214046FFF737FF95F831
:104C80002300002770B1206B05F042FD1048012180
:104C90000176D5E92012C0E90412216B606A05F0A3
:104CA000A9F904E0606A05F033FD05F0E5F916B9ED
:104CB000384605F0E3FB002198F86A20084605F025
:104CC000AFFD02202070BDE8F08100006C000020E4
:104CD000B02300202DE9FC470446FFF725FD0546DB
:104CE000FFF71CFD00278DF800700646DFF8649181
:104CF00095F8233022463946FFF7F8FEA87D4FF09D
:104D00000108A9F1200440B1012820D002282FD0A9
:104D100003283BD040F2FF2157E0A0795021ADF8A5
:104D2000040088534846FFF7EFFA30B18020216A2B
:104D3000FFF7ECFC85F811802CE06A4601A9606B56
:104D40000BF0C6FB206210B195F85B1011B1424820
:104D500020621FE09DF8001021B9078087700121B3
:104D60000BF04BFFBDF80410206A0BF0CEFE11E0F3
:104D7000B6F85000ADF804006A4601A9606B0BF06C
:104D8000A7FB206230B940F2E9211EE04846FFF758
:104D9000BBFAC0B1206A0823017801F0F701017065
:104DA000EA7D03EAC202114301F0FB0101702A7E91
:104DB000042303EA8202114301F0EF010170C943A9
:104DC000890705D007E040F2F2212720FEF74AFCD0
:104DD000C07802280FD0606B0AF0F4FF08B10121FF
:104DE0000AE0206A0078C043800704D0FFF74AFA3F
:104DF00080F0010100E00021206A027842EA0111FE
:104E0000017095F8221081B1417871B1206B05F0E5
:104E10007FFC114828380776D5E91E12C0E9041234
:104E2000216A206B05F0E6F803E005F071FC05F05F
:104E300023F996F86B200121002005F0F1FC84F89D
:104E40000380216A0A8822828978A17484F800800C
:104E5000BDE8FC878C000020D8230020C14A000058
:104E600009480000B9490000454C0000004870475F
:104E7000B12C002004498A78824203D9084490F872
:104E80004301704700207047DE2A002004498A78D9
:104E9000824203D901EB0010833070470020704735
:104EA000DE2A0020054A01EB410102EB41010268C4
:104EB000C1F80B218088A1F80F017047DE2A00207D
:104EC0002DE9F0410E4607461546062130460BF007
:104ED000E3FC0D4C60B1002004E02118401C81F877
:104EE0003B51C0B2A1788142F7D80120BDE8F081E2
:104EF000314638460BF0FBFA082803D0204480F8EE
:104F00003B51F2E70020F1E7DE2A002004498A78CD
:104F1000824203D901EB0010C01C7047002070478B
:104F2000DE2A002010B540F2D312002108480EF00E
:104F30009CFD0822FF2107480EF097FD054800213F
:104F4000001F017041704FF46171418010BD00007D
:104F5000DE2A002054030020014908707047000039
:104F600050030020014800787047000050030020E3
:104F70000B4B10B59C7884420FD9184490F803016C
:104F800003EBC00090F853310B70D0F8541111604E
:104F9000B0F858019080012010BD002010BD000025
:104FA000DE2A002007498A78824209D9084490F80D
:104FB000030101EBC00090F85A0100F001007047B6
:104FC00000207047DE2A00202DE9F04798469146E0
:104FD0000C46054600F036F90646102806D000F0CB
:104FE00001F9102802D01220BDE8F087184FB878D8
:104FF00008282AD2102E05D100222146284600F08A
:1050000005F90646BC781022601CB87007EB041541
:10501000E81C49460BF0D2FB05F183001022414603
:105020000BF0CCFB102140460BF036FC3C44102129
:1050300084F84301484604F596740BF02DFCE077A4
:1050400004F8296C0020E073CEE70720CCE70000CD
:10505000DE2A0020064810B58078401E44B204E0E5
:10506000E0B200F04DF9641E64B2002CF8DA10BD15
:10507000DE2A0020014840887047000050030020CD
:1050800038B14AF2B811884203D803494880012058
:1050900070470020704700005003002005498A78BF
:1050A000824203D9084490F83B0108B100207047C0
:1050B00001207047DE2A002070B50D46064600F03C
:1050C000C1F8104C102807D004EBC00191F85A1118
:1050D000C90701D0012070BD6178082910D21028BD
:1050E00008D004EBC000012180F85A116078401C00
:1050F0006070EFE701222946304600F087F8F5E7B7
:10510000002070BDDE2A002070B50B4D2878401EAF
:1051100044B20AE005EBC40090F85A01C00702D07F
:10512000E0B200F035F9641E64B2002CF2DA0349F3
:105130000020487070BD0000DE2A002050030020CF
:105140002DE9F04100242546184E29E006EBC5075D
:1051500097F85A01C00721D0284600F043F80346CB
:10516000FFF7D4FE01460020102B09D0F21892F868
:105170003BC1BCF1010F02D092F84B2102B10120DA
:10518000401E01420AD10A4807F5AA71035520467C
:10519000641C97F85321E4B205F068FC6D1CEDB275
:1051A0003078A842D2D8BDE8F0810000DE2A002085
:1051B000540300200246094810B500780B4658B148
:1051C0000748817841B10BB1C01C01E0044883302D
:1051D00004F018FE012010BD002010BD5003002077
:1051E000DE2A0020084910B5034600208A7806E030
:1051F0000C1894F803419C4204D0401CC0B2824277
:10520000F6D8102010BD0000DE2A002070B50C4B2F
:1052100004461878451C1D70102803D34621282009
:10522000FEF720FA03EBC0030D68C3F854518988D8
:10523000A3F8581183F8534183F85A2170BD000038
:10524000DE2A0020F0B51A4C0346002025782AE01B
:1052500004EBC0020F7892F854C192F8536187EAC8
:105260000C075E403E444F7892F855C187EA0C0720
:105270003E448F7892F856C187EA0C073E44CF78B7
:1052800092F857C187EA0C073E440F7992F858C14B
:1052900092F8592187EA0C073E444F795740F7426C
:1052A00004D0401CC0B28542D2D81020F0BD00000E
:1052B000DE2A002070B50546FFF794FF10281CD1A8
:1052C0000E4C2078401EC0B22070A84215D004EBCE
:1052D000C00204EBC50102F58070D2F85321C1F879
:1052E0005321D0F85700C1F857012078FFF77AFF13
:1052F000102802D0204480F8035170BDDE2A00201F
:105300002DE9F047214C0646A719A078401EC5B2EA
:10531000A57097F80381AE422AD004EB051A04EB7E
:1053200006190AF1030109F1030010220EF023FB14
:105330000AF1830109F1830010220EF01CFB6019B1
:1053400005EB450290F8031187F8031106EB4601BF
:1053500004EB420204EB4101D2F80B31C1F80B31EE
:10536000B2F80F21A1F80F2190F83B0187F83B011B
:1053700004EBC80090F85A01C00704D14046BDE8CC
:10538000F047FFF797BFBDE8F0870000DE2A002056
:1053900005494A78521E4A7001EBC001002281F88B
:1053A0005A21FFF787BF0000DE2A00202DE9F047D1
:1053B000044600F180054FF0010971B104F1A60720
:1053C0007E1E012925D002294AD003291FD1394642
:1053D0003046BDE8F0470BF0BDBA4FF43E720021F5
:1053E0000EF043FB85F825902248E86607202867E1
:1053F00014F8EC0F20F004002070FE2085F8A600C1
:105400007F2068761C48A8600020C5E90000BDE840
:10541000F0874FF00008A4F8368284F82B822169C7
:1054200016480A460844B0FBF1F0C4F8C40040F640
:10543000B830A4F8C800638B284600F021F839463C
:1054400030460BF087FA0EF027FA18B1606900F0C9
:1054500053FB10B184F81A82D9E784F81A92D6E780
:105460000169B4F8DA32D4F8D4222846BDE8F0470E
:1054700000F006B82F49043400E0FCFF7FC3C901E7
:1054800010B50024A0F84C4030F8504F4C43B4FB0A
:10549000F2F420F8104940F27124634302EB031345
:1054A0005B1EB3FBF2F3C381094BB3FBF2F35B1C4E
:1054B00083820389634302EB03135B1EB3FBF2F3A6
:1054C000436003684B43B3FBF2F1016010BD000081
:1054D000005A6202024991F900100BF0ECB9000089
:1054E0007003002008B57F208DF80000684605F0A5
:1054F000BDF940B105484078404241B29DF90000F5
:105500000BF0D9F908BD9DF9000008BD700300201B
:1055100070B590F8322090F83130012403FB01215E
:105520002522B1FBF2F302FB131100EBD10280F84C
:10553000321001F0070392F8262004FA03F31A420E
:1055400004D000BF80F83310002070BD90F83020E8
:10555000B1FBF2F302FB1311491CC9B20023C518B9
:1055600095F82B208A4212D395F82650002200BFCE
:1055700004FA02F6354201D0491EC9B221B1521CCB
:10558000D2B2082AF4D304E002EBC301DAE7891AA5
:10559000C9B25B1CDBB2052BE1D31F2070BD00003C
:1055A00070B5491C0023C9B20124C518AA798A42E2
:1055B00012D395F80150002204FA02F6354201D0C8
:1055C000491EC9B221B1521CD2B2082AF4D305E057
:1055D00002EBC300C0B270BD891AC9B25B1CDBB25A
:1055E000052BE2D39D214620FEF73CF8417841B1DE
:1055F000C0782B2803D2044A105C884201D10120D4
:105600007047002070470000B43B010010B5012234
:10561000C1702B2902D2064A525C06E0FF2904D051
:1056200040F275412A20FEF71DF8427010BD0000BF
:10563000B43B01000449897C490700D408B100202B
:105640007047012070470000A82500200348807C97
:10565000800701D40120704700207047A825002052
:105660000348807CC00701D00020704701207047AC
:10567000A82500202DE9FE43884699461546044694
:1056800069460AF077FFE0BB019E002780367DB1B6
:105690002046FEF7F9FB04000ED029460AF064FB11
:1056A00018B11B494988A94208D20020BDE8FE83F1
:1056B000012086F8240024E0672125E0014602AAA3
:1056C00020460AF04AFB02980780877096F824105B
:1056D00009B14FF0020841460BF08FFA02982A46B2
:1056E0004946C01C0EF047F9204629460AF0F3FA55
:1056F00048B168460BF0DCFA0198A0F8227286F8EF
:1057000024700120D2E77C212B20FDF7ABFF0000A5
:10571000A8250020094882B0007A8DF80000009882
:1057200000909DF80000002805D10222044903489A
:1057300002B00BF0E0BA02B070470000C0250020B4
:105740003D0D01002DE9F84FDFF89881DFF898A1B1
:1057500083464FF001090026D8F80400007A8DF83E
:105760000000009800909DF800102A2906D19AF8B0
:10577000131019B1BAF8140000287DD000278DF855
:105780000060684600F012F99DF800100029F8D179
:10579000002871D00446007A8DF80000009800902F
:1057A0009DF80050A81E302867D2DFE800F01827C7
:1057B00085218585276F696F6F6F2D6F85218585A1
:1057C0006F6F21858585856F4585856F216F6F8515
:1057D0006F2185854F55758585858585854F6268DF
:1057E00012B94FF4D27164E05946204690473CE02C
:1057F0006268002AF8D140F2BB115AE06268002AC0
:10580000F2D140F24B2154E060685D4680B10488DB
:105810002046FEF739FB68B16E700D222A70EC80CD
:10582000A5F80890314685F804900AF034FB57E05B
:10583000CE213EE0AE213CE0626822B159462046CE
:105840009047012711E040F2632132E06268002AAC
:10585000CAD140F26F212CE08BF8016016218BF841
:105860000010D4F80910CBF804102672212D26D090
:10587000142D27D0222D01E017E01DE029D02DE0C6
:105880006268002AB0D140F2812112E06268002AE9
:10589000AAD140F296210CE01448026822B1606857
:1058A00028B10088594690470220BDE8F88F40F2A1
:1058B0009F211020FDF7D6FE40F2BD21F9E7FFF74A
:1058C000C5FE08E09BF80E0000F00100FFF7B2FEF5
:1058D00001E0FFF7C5FE00287FF43EAF002FFBD1AB
:1058E0000420E2E7D4250020A8250020B0000020F5
:1058F0000149087000F0B0B8720300200249014865
:10590000086070470D590000B000002038B50D0048
:1059100014D0A88000216972FEF7A0FA04460AF0AC
:10592000FEF968B101466A4620460AF016FAE88098
:1059300048B1FB280AD94FF4867132E0FC2130E0EF
:1059400040F205112DE04FF485712AE000980BF02C
:1059500000F9012804D0022802D04FF48E7120E013
:1059600028722868A8B10099EA88C91C0EF003F8CB
:1059700020460AF09CF978B1204600210AF08BFA03
:1059800068B10948C17C002902D0818A491E818200
:1059900038BD40F2231104E04FF4947101E040F26D
:1059A0002D111020FDF75EFEA825002038B5024617
:1059B000114B002010705868017A8DF80010009982
:1059C00000919DF800500124012D06D0EFF31081C5
:1059D00072B605685D6011B102E0002038BD62B6A4
:1059E000017A8DF80010009900919DF80030002B8D
:1059F000F4D1147038BD0000D425002038B5D0B1E2
:105A0000416000F108010A70EFF3108372B6104C88
:105A10000460211F4A684AB1127A8DF80020009A6A
:105A200000929DF80050012D00D10C600A681060B2
:105A300008602BB105E040F2E2211020FDF712FED4
:105A400062B604480078BDE8384009F0EFB90000BC
:105A5000D825002072030020084810B500214161BC
:105A60008161C161016212220DF0FFFF0348143011
:105A700001210173011D4160016010BDC02500209E
:105A8000F0B450810C89134694818A89DA8148895F
:105A90001882CD895D82CE8DAE4208D14D8D854272
:105AA00005D10D8E954202D18A8DA24201D00122EC
:105AB00000E000221A754885588AC885988988852B
:105AC000D8890886F0BC1422014918460BF027B982
:105AD000FB0E01005081888A9081C88AD081088B92
:105AE0001082488B134650822122024918460BF03F
:105AF00002B90000310F0100F0B56FF01F02010C78
:105B000002EA90261F25A1F5AA4054380DD0A1F530
:105B1000AA40553809D0A1F52850AA3805D0A1F5DA
:105B20002A40AA3801D0012000E0002000221346BC
:105B30004FEA020482EA0107FF431F437F1C0FD094
:105B400006F00107520842EAC73205F001075B0878
:105B500076086D08641C43EAC733162CEAD3F0BDFF
:105B60000020F0BD10B504480BF046FA0248BDE82D
:105B7000104008300BF040BAB4000020014800F09B
:105B800009B80000B4000020014800F003B800008C
:105B9000BC00002010B5D0E90021094B094C53434B
:105BA0005443514081EAB21282EA41224FEAF14164
:105BB000C0E9002143EAD46303EB8303184610BD18
:105BC0006037EFC6BB79379E10B54068002290F869
:105BD0008C308030091DDB0701D0012010BD0C790D
:105BE0000B6809490B4004F00701C3660167A0F880
:105BF000582090F85A10491C80F85A10C16841F09A
:105C00000101C160002010BD2F49043710B5041DEB
:105C100004F0C8F8034A01F00701104020606160F9
:105C200010BD00002F4904372DE9F8430378406880
:105C30000F1D00F1800500F5A57406464FF0000821
:105C40006A7F072128460AF0BFFCB0B13868154AC0
:105C50003979104001F00701E866296785F8568018
:105C600085F81D8094F8681040468DF80010009962
:105C700000919DF8001091B902E00120BDE8F88381
:105C80003188A4F86A1084F869003968E166796897
:105C900021670822044904F160000BF02CF8002071
:105CA000ECE700002F4904376511010070B50D1DA8
:105CB000446804F077F8064A104001F0070294F8AF
:105CC000EC10014061F3070028606A6070BD0000BD
:105CD0002F490437416882B001F5A57091F8B221CF
:105CE0008DF80020009A00929DF80020002A0BD128
:105CF0000988A0F86A101A2180F86910082203495F
:105D0000603002B00AF0F7BF02B0704765110100C1
:105D100070B544680D46037894F89D2080340026C1
:105D2000082120460AF050FC20B9207B800701D5CD
:105D3000012070BD94F85D00800719D428460AF050
:105D400076FF84F8670035F8050FA4F868006888C6
:105D5000A4F86A0094F85D0040F0020084F85D0049
:105D6000C00709D00322114904F15E000AF0D7FFF1
:105D700094F85D00C00710D1E068810703D54F217A
:105D80004020FDF76FFC40F00200E06094F85A00FC
:105D9000401C84F85A00A4F85860607F012802D1A2
:105DA000667784F85660002070BD000093110100F2
:105DB000074900F500600013097840B2494249B232
:105DC000084400F30700002800DC0020C0B2704740
:105DD000C4000020044A9268C2F580534B434243FA
:105DE00003EB223070470000C4000020F8B544687F
:105DF000064604F1800500F07FF894F82810012988
:105E00001AD1002818D0706890F852118DF800103F
:105E1000009900919DF8001000F5A57000290BD1A4
:105E200021884181697E0173A97E4173BDE8F840F4
:105E30001F2202490AF05FBFF8BD000035120100C1
:105E400000F500610D4A10B500F50060091300135C
:105E50004BB292F900404042002140B2A34202DA24
:105E600092F9021005E092F90140A34204DD92F993
:105E70000310084400F30701084610BDC4000020C9
:105E80002DE9FC4100224A70A0F5FA750A70A0F5D0
:105E9000BA7495F86B000CF0E8F90646A068FFF7B5
:105EA000CFFF070021D020460BF0CCF900281CD0F2
:105EB000288869460AF05EFB18B189217A20FDF72F
:105EC000D1FB761CF1B202233A4668460CF0ECF99D
:105ED00000280AD1064807490079A0FB016507F0B0
:105EE00097FD80196941C4E90001BDE8FC8100000B
:105EF000C400002040420F002DE9F0410746FFF7A3
:105F0000F1FA7C68054684F8990080347F283CD0FB
:105F100094F833007E68A0762946A068FFF75AFF00
:105F2000A0601B48407990B1786800F18008D0F8F3
:105F30008800FFF785FF50B140460BF083F930B180
:105F400078683122134900F5FA700AF0E8FE94F9F6
:105F50001B000021281A00D5404296F829208242D1
:105F600010DCFF2A0ED0207F401CC0B2207796F8AC
:105F70002A20904202D8E07E7F2803D10020E576D7
:105F8000207701210846BDE8F0810020FBE70000F2
:105F9000C4000020815E000070B50446007C00B3A0
:105FA00002281ED05FF0010004F1510184F8500076
:105FB0000D46C0B1E07DF0B1D4F81100C4F8510035
:105FC000B4F81500A4F85500207C0BF064F9207695
:105FD0000820607694F8500029460BF048F9A8B9DB
:105FE0000EE00020E0E70020FEF7DAF90028EBD110
:105FF00040F2B94101E040F2BD412D20FDF732FBF6
:1060000094F8500029460BF03BF900B10120A0762E
:10601000207E30B194F8570004F158010AF067FA75
:106020006076FFF727F80C49A0FB012304F1480034
:106030000BF0B6FA002120460BF06BFA002084F832
:106040005E00A078400705D52046BDE870400021DD
:1060500000F0D0BD70BD000040420F0030B50C46CE
:106060008DB005460146242202A80DF084FC0BA841
:106070000BF0F3FAA07A8DF8180020788DF808005C
:10608000B4F80100ADF800009DF8000000F0010137
:10609000C0F3400241EA4201C0F3800241EA8201BA
:1060A000C0F3C00241EAC201C0F3001241EA02118A
:1060B000C0F3401241EA4211C0F3801041EA80105F
:1060C000ADF80A00207D012806D0022804D040F255
:1060D000EA210620FDF7C6FA8DF80C00617A0BA8BC
:1060E0000BF0A2FA207D0121022802D1607D401C24
:1060F000C1B2A07E401CC2B20BA80BF05CFABDF886
:106100000A00000701D5002020E00BA80BF065FA7B
:10611000BDF80A10282200F011FE40F2712100F2B1
:10612000D920B0FBF1F04843D4F8021040F27123BB
:106130000A0A40F271214A43D4F80510090A59436A
:10614000904201D8049204E0884201D8049000E013
:106150000491A07C8DF81700207E012800D000203B
:106160008DF81400686B0AF02AF8686B0AF0CFF813
:10617000242202A928460DF0FEFB0B98A862BDF868
:106180003000A885E07A68B102280BD05FF00100EA
:1061900085F85700E068A865208AA5F85C000DB076
:1061A000002030BD0020F3E70A4A10B5002111702D
:1061B000094C606000F022F810B140F22D3104E08B
:1061C000A068002804D14FF44C712D20FDF74AFA45
:1061D00010BD0000E4250020D00000200249014845
:1061E00088607047246D0000D000002002490860DC
:1061F0008968096808470000D0000020084810B5E9
:10620000007810B10C24204610BD0024182221462D
:1062100003480DF02AFC03F0E7FF03F00BFEF2E762
:10622000E4250020044910B50978012901D100F0C6
:10623000B5FB002010BD0000E42500200249014804
:1062400008607047C96A0000DC00002010B50446F1
:106250008078C0F3C00058B13C23FF222046E1699A
:1062600000F0C2FB1122044904F16C000AF043FD66
:10627000012084F8690010BDAB1401002DE9F04144
:106280000F00044623D004F1280005460BF0CEF998
:10629000B0B9A078C0F3C00050B328460BF09DF908
:1062A000064628460BF0C2F9301AC0B20BF013FABA
:1062B0000146354842681144416028460BF0D4F944
:1062C00028460BF096F9014620460BF05EF92F4D5B
:1062D00094F85E600021686801800BF0BCF860886B
:1062E000132813D009DC102836D0122809D131E048
:1062F0002046BDE8F04100F051BB15280FD01D2805
:106300000DD040F272612D20FDF7ACF900216868D4
:106310000AF078FB012168680BF09DF820E001216C
:1063200068680AF06FFB012168680BF094F836B1D9
:1063300004F15F0168680AF080FB012106E004F1C6
:10634000580168680AF079FB94F8571068680AF0F9
:106350007AFB05E0062100E0022168680AF052FBA2
:10636000204600F0BDFC60881D2807D0152805D008
:1063700094F83C20A16B68680AF034FB394620464B
:10638000BDE8F04100F0F6B9E4250020D00000207F
:106390002DE9F0412F4D80462878022805D0287835
:1063A000032802D040F62D512BE02B4C2668307B81
:1063B00018B1FFF797F886F82E00D4F804C000272C
:1063C000B8F1000F9CF8000000F00F0627D02168FC
:1063D000C00901F1510391F850200CF1090109F0B5
:1063E000EEFFE0B1394660680AF0ECFAB8B12A78FD
:1063F00020683146022A07D02A78032A04D040F6C2
:1064000006512D20FDF72EF9A2682B7852696FF006
:10641000070606EB8303D2589047064600E00126A4
:10642000A87B18B103F0E0FE03F004FD002E0FD0AE
:1064300020680BF066F930B103F0FEFEA0688068BA
:10644000BDE8F04100472068BDE8F04100F0A6BA81
:10645000BDE8F081E4250020D000002010B503291C
:1064600002D005290AD102E000F092FB03E00449C2
:10647000096809B1884708B1002010BD012010BD8E
:10648000DC000020094A0300106801D000F086BA41
:10649000002909D09168064A096912786FF00F0344
:1064A00003EB82028958084770470000D0000020A3
:1064B000E425002070B504464088102819D0104DFE
:1064C000A87B20B103F0D6FC402003F09BFE0D48D2
:1064D000406804F01DF9A078400704D40021227917
:1064E000084604F09DF9002003F0C8FF0220287040
:1064F00070BD2046BDE870400121FFF7BFBE00001F
:10650000E4250020D000002010B5124C206800F0D7
:1065100025F820680BF0F5F8002820680BD00E490C
:106520000A78022A0BD00A78032A08D040F63741AD
:106530002D20FDF797F8BDE8104000F02FBAA268B3
:106540000978D2686FF0070303EB81015158BDE869
:1065500010400847D0000020E425002010B5017B42
:1065600021B10446FEF7BEFF84F82E000548807B6B
:10657000002805D003F038FEBDE8104003F05ABCF7
:1065800010BD0000E42500202DE9F0415D4D0446DA
:1065900086B0287800284ED12078FF284BD04FF0C5
:1065A0000008A5F80C80C5F8048085F8018085F8FE
:1065B000028084F86980544B544E0FCB8DE80F0055
:1065C000B06840680390684603F02CFF03F0FAFFC0
:1065D00004F07CFA03F008FE03F02CFC4C4804F0B5
:1065E00051F94C4804F058F904F1280007460BF023
:1065F0003BF838460AF0FDFF014620460AF0C5FF89
:1066000094F90E0004F062F82179002003F09EFE58
:106610000121A86098B104F13801606B09F03EFED9
:10662000074604F14001606B09F03BFE4FB194F85E
:10663000201051B905E00C2006B0BDE8F0812970AA
:106640005EE020B194F8210008B1012700E00027A6
:10665000A07E20B9207E10B9A078400723D5D4E9C8
:1066600012106FF00042504070EA010106D007F0AE
:10667000CFF9D4E91223801A994100D29FB1FEF7D5
:10668000F9FC2549A0FB012304F148000AF088FF2A
:10669000012120460AF03DFFA078400703D50121E3
:1066A000204600F0A7FAFEF74BFD7068C01C09F009
:1066B00011FFA873A078C00722D0CDF81080FF206A
:1066C000CDF81480E873E66906F10A0713E0049C2C
:1066D000B44210D0727A607A3B4604F10A0109F0A4
:1066E0006EFE40B1A078E873D4F803002861B4F8D6
:1066F0000700A88204E004A8FDF7F2F90028E6D01C
:10670000002099E7E4250020046D0000D00000205F
:10671000D6BE898E5555550040420F0010B504462F
:10672000FFF732FF002808D104480078012803D081
:1067300000212046FFF7A2FD002010BDE425002027
:106740000A4810B50A490468087800280DD008786E
:10675000022802D00878032802D12046FFF7FEFE67
:106760002046BDE8104000F019B910BDD00000204F
:10677000E42500202DE9F041044629480D464068F3
:1067800003F0C6FF274E0420307055B360881028F0
:1067900023D004F128008046B5680AF01EFF0746A2
:1067A00040460AF043FF381A401EC0B261882822D2
:1067B00000F0E4FA0544A078C0F3C00030B170687E
:1067C00005440AF08CFF2844C4F8D80022792946F1
:1067D000002003F0B3FF20B90CE02179002003F082
:1067E0007BFD6088132811D007DC102815D01228F3
:1067F00007D10BE040F6A85105E0152806D01D286A
:1068000004D040F6BC512D20FCF72CFF2279BDE8C6
:10681000F0410121002004F003B8BDE8F081000040
:10682000D0000020E425002038B5044690F8BC00D4
:106830000B468DF80000009800909DF8000000289D
:106840003AD1207884F8BD00FF2B10D004F1BF02AC
:10685000511E1846FEF78CFB30B194F8BE0040F094
:10686000020084F8BE0011E041F2080121E0134863
:1068700040680178C1F3801184F8BE10D0F803108D
:10688000C4F8BF10B0F80700A4F8C30094F92E00B4
:106890007F280CD084F8C5007F2084F82E0004F1F6
:1068A000B400BDE83840202205490AF024BA40F679
:1068B0006C612D20FCF7D6FE38BD0000D000002012
:1068C000FB1401002DE9F04790460E4604460329CB
:1068D00004D094F8680008B1012000E0002081464F
:1068E00003F09CFC0546032E03D00127052E05D09E
:1068F00008E0A0780227C0F3400001E0A078C007BC
:10690000002842D0B9F1000F3ED12248807B40B12F
:1069100009F0E3FD88F80000FF2802D0FEF742FBF3
:1069200005431D4E94F8572004F15803716811F87F
:10693000030BC0F3801009F042FD98F80010FF2906
:1069400004D090B9607E88420FD008E038B17168F9
:1069500011F8030BC0F380100AF086FD28B1002067
:10696000A178490703D590B90EE00120F8E775B981
:10697000E07B08B1B84207D1716811F8030BC0F38E
:1069800080100AF071FD10B10020BDE8F0870120F1
:10699000FBE70000E4250020D000002070B504468D
:1069A000008E104D401C2086A87B002620B103F0ED
:1069B0001BFC03F03FFAAE732E7094F8690008B127
:1069C00001210AE0607B38B1218E884204D8012180
:1069D00020460AF0A8FE70BD00212046BDE87040A8
:1069E0000AF0A1BEE42500202DE9F041044680F81C
:1069F00075300888A4F87600FF2084F893004FF6DD
:106A0000FF7016460D46A4F89400002B4BD1286960
:106A100009F0C1FDA4F88C00288BA4F88E00688BC7
:106A2000A4F8900095F81B0284F89200207E04F1EF
:106A300051010F46002520B194F850000AF020FCC7
:106A400040B994F86A0070B194F8500039460AF0E1
:106A50000EFC40B1D4F85100C4F88000B4F85500E1
:106A6000A4F8840003E0C4F88050A4F884501548CA
:106A7000FF2E40680178C1F3801184F8791050F836
:106A8000031F17D0C4F886108088A4F88A0004F188
:106A90007A02511E3046FEF76BFA30B114F8790FC6
:106AA00040F002002070BDE8F08140F68B412D20BF
:106AB000FCF7D8FD44F87A1F8088A080E560258225
:106AC000F1E70000D0000020F8B50446FF208DF863
:106AD000000001266A4605212046FFF7F3FE60B15B
:106AE000284D274F6968FA7B07F1100311F8030B53
:106AF000C0F3801009F063FC10B100263046F8BDE9
:106B00006A68E069127810F8A51FC2F340121140BC
:106B1000017001222046E16900F09AF800239DF8F7
:106B200000202046E169FFF75FFF1122164904F1BA
:106B30006C000AF0E0F8E06905220188A4F8B010C2
:106B400090F8A50084F8B200104904F1A6000AF0FC
:106B5000D2F80021E06939700A46214600F086FA31
:106B60006868E169D0F8032041F8032FB0F80720E6
:106B70008A800078E169C0F380108870BEE7000069
:106B8000E4250020D0000020AB1401009B1401007C
:106B9000F8B50446FF208DF8000001256A46032160
:106BA0002046FFF78FFEE8B1207B20B19DF8001052
:106BB0002046FFF739FE0D4E002170680180042148
:106BC00009F020FF204600F08BF894F84420216C57
:106BD000706809F04EFF064905200870706803F0E0
:106BE00097FD00E000252846F8BD0000D0000020F9
:106BF000E425002070B504460E46407EFEF786F977
:106C0000050019D0102109F047FE002814D10120F9
:106C100084F85E0004F15F0132460C46284609F014
:106C2000FEFB2146054C606809F007FF6068BDE87F
:106C30007040012109F007BF70BD0000D0000020A6
:106C4000024801210068FFF719BB0000D0000020B6
:106C50002DE9F041214E80460C467068154650F8EB
:106C60000F1F6161416821F07F41E161408909F0B6
:106C70008EFC0746206170683946807D09F003FE6E
:106C8000A08470683946B0F8170009F0F8FD20625A
:106C9000706830F81B1F2183418861834168C4F804
:106CA000A610017A84F8AA10417A01F01F0184F835
:106CB000B110407A400984F81B0204F162000572A9
:106CC0004572FF218172002136380AF0C3F898F826
:106CD0000E0084F86E00BDE8F0810000D0000020B6
:106CE00070B5074D044600F15101686809F0B2FE25
:106CF00094F850106868BDE8704009F0B1BE00001B
:106D0000D000002009650000916300008564000048
:106D1000000000005D640000B56400008F140100F5
:106D2000951401001D67000041670000416C0000E0
:106D3000206D0000186D0000146D000010B5421E9B
:106D4000022A01D9CA2109E0401E102909D01229BE
:106D50000CD013290AD0152905D0D8212F20FCF7F3
:106D600081FC054904E00449891D01E00249891FAD
:106D700031F8100010BD0000F6160100421E10B5DB
:106D8000D2B2012A03D91D2901D0EE210DE0132929
:106D900013D004DC10290BD0122904D10DE01529E1
:106DA00008D01D290ED04FF481712F20FCF75AFC1A
:106DB000074804E00648083001E00548001D30F8A7
:106DC000120010BD40F25A3110FB01F010BD00005E
:106DD000E41601002DE9F041044690F8E000164663
:106DE0000F4600285ED121464D4806F001FC0546BD
:106DF000202857D05022002104F1C8000CF035FEA5
:106E000084F8C8500125C4F8CC7084F8E05037B13C
:106E1000FEF7BAFE00F00700401C87F84C0220463F
:106E20000AF01EFEA4F8F000022084F8F200A84642
:106E300084F8F350002504F8E85F07F065FD074685
:106E40000CF00FFC2189E83C884200D80846384401
:106E5000CC3087B220460AF0C6FA30B30CF0D5F930
:106E600000F5CD6081B2304607F06EFE3044C4F8C4
:106E7000EC00903406F0CCFDC0196941C4E91A0158
:106E800084F8408024F86E5C01200AF024FC00F5B0
:106E90008870301A60644FF0FF304108C4E91E0169
:106EA000903C25E00C20BDE8F081002120460AF04E
:106EB00029FDDFF87080C4F8EC000020B8F8041059
:106EC00049B1618C39B1FEF75FFEB8F80410B0FB30
:106ED000F1F201FB1200074406F09AFDC019694166
:106EE000C4E93E019EB1801951EB0501C4E942019C
:106EF00094F8C80004F1E8010AF0B0FD58B1A4F814
:106F00000051002120460AF09EFA0020CBE74FF006
:106F1000FF304108EAE74FF4F4713020FCF7A2FBA0
:106F2000D91B0100E0000020014988807047000063
:106F3000E0000020054800210170012282704170AC
:106F400042F21071818000F003B80000E0000020E0
:106F50001CB50949D1E90001CDE9000102E0009822
:106F60000AF0F5FB6846FCF7BBFD0028F7D000F0FF
:106F7000A9F800201CBD0000247800000149087019
:106F800070470000E000002008494FF47A72B1FB1E
:106F9000F2F110B501F5257109F075FF40F64801D1
:106FA000884200D3084680B210BD00007D52010027
:106FB0002DE9F0410F4CD4E9026703F0C3FA05460E
:106FC00002463946304609F0ECFA0646A068864289
:106FD00005D02169301A0844206106F04BFCA660F8
:106FE000B54201D8607810B10020BDE8F0810120E1
:106FF000FBE70000E000002010B5044606292ED271
:10700000DFE801F0051103141528002106E0D4F88B
:10701000AC0210B120460AF0B4FC01212046BDE8C4
:10702000104000F0F7B8032084F85C0210BD03F0B4
:107030008FFAC4F8AC0294F86B0003F04DFBD4F85F
:10704000AC12091A084882680A448260C268114476
:10705000C16010BD2046BDE810400AF07DBC4FF471
:10706000E8613020FCF7FEFAE000002070B50C4625
:10707000054612B140F26A7110E003F063FA01466E
:10708000002220460AF05CFD94F8C8002A46054913
:1070900006F064F9002804D140F253713020FCF767
:1070A000E1FA70BD7B1C010010B50C2804D340F23E
:1070B0008B310620FCF7D6FA014931F8100010BDDB
:1070C000407800002DE9FC41154D01206870002436
:1070D0004FF6FF760BE0002108F0C2FF070009D051
:1070E00097F8A40206F06CF938460AF01CFD0094EB
:1070F00001940DE04FF490713020FCF7B3FA009842
:1071000030B190F85C1219B10088B042E3D104E0CC
:107110006846FCF7E5FC0028F1D06C70BDE8FC8106
:10712000E00000202DE9F047044639481E4690460D
:10713000807889460025002863D007F0BBFCE0B3C7
:10714000B4F8480202285CD394F85C02022858D0B4
:1071500094F8720288BB94F81B02FFF7A5FF00F5B4
:10716000C86081B2318094F85C02002701280DD0FC
:10717000206907F0E9FCB4F836224244A2EB090189
:10718000D4F86422821A01FB027535E094F8A1005C
:10719000032839D00121002009F0CEFA216A4718CE
:1071A0003188D4F8540207F0CFFCD4F85022D4F838
:1071B0005812821A01FB025500E022E0C4F8500286
:1071C0003188384607F0C0FCD4F86012C4F8600279
:1071D000411A0D443188206907F0B6FCB4F8362214
:1071E0004244A2EB0901D4F85822891AD4F8642247
:1071F000821A491E01FB0255C4F86402012084F87A
:1072000072022846BDE8F087D4F85402C6E70000B1
:10721000E000002038B500250446012902D11048BD
:10722000407870B1042084F85C0200BF0AF0A2FB31
:10723000A4F8A252B4F89400A4F86E0284F8715233
:1072400038BD0095B4F8241201230022204600F036
:1072500009F80028EAD040F2B5613020FCF702FAC4
:10726000E00000202DE9FF4F8BB0044690F86B0042
:1072700099460F46079305900BF0C7FF054694F813
:107280001B02FFF711FF2844ADF8040094F89E009C
:107290000D2804D0002008900D9810B12EE0012098
:1072A000F9E794F85C02032828D1089830B3B4F8C1
:1072B000CC02B84222D1D4F86402C4F8500220694A
:1072C000C4F85402B4F8A202B4F836120844C4F860
:1072D0005802204600F0C0FAD4F8D0022062B4F878
:1072E000CE02A084D4F8D4022061B4F8D80220835E
:1072F000B4F8DA026083022084F85C02B4F89400E7
:1073000004F51E75381A0FFA80FAB4F8A002381A7C
:107310000FFA80F8B8F1000F08DAD4F89002D4F828
:107320009412D046C4E9A6010120079001AB524651
:1073300041462046FFF7F6FE049094F85C02DFF821
:1073400034B340B101287DD0022851D003287AD02F
:1073500040F243518AE10121002009F0EDF906468F
:10736000206ABDF80410304407F0EEFBC4F8600258
:10737000BDF80410206907F0E7FBC4F8640207A910
:1073800006A803F047F8D4E9A601DDE9062306F0D4
:1073900051FB824620460AF0DFFA94F86B00D4F8DD
:1073A000A88203F0C5F94AF2A13101444FF47A7082
:1073B000B1FBF0F0216AD4F860223144081A811A36
:1073C00041442039A1EB0A065000A18C60300144F1
:1073D00094F86B000AF030FB2230CBF81400D4F89C
:1073E000A802301AB0F5DE7F58D240F2DC413DE110
:1073F000216AD4F854020844BDF8041007F0A4FB35
:10740000C4F86002BDF80410206907F09DFBC4F8C1
:10741000640220460AF0A0FAB4F8360210BBB9F1B3
:10742000000F1FD094F86B80404603F081F94AF2B8
:10743000A13101444FF47A70B1FBF0F0D4F860123E
:10744000084401E02BE047E0226AD4F854121144CA
:107450000E1A404603F040F9D4F8AC12081A06445C
:10746000203E06E0216AD4F854020844D4F86012A1
:10747000461AD4F85822D4F85012D4F8600201FB0E
:1074800002004000A18C6030014494F86B000AF0C7
:10749000D3FACBF81400012084F85C0261E0D4F840
:1074A00064222069B4F83612861A01EB0A00D4F877
:1074B0005812D4F850C2401AD4F86032401E0CFB67
:1074C000013100FB02104000A18C6030014406FB3A
:1074D00008F694F86B0040E02069D4F8641200FBD1
:1074E00008F008FB110694F89D00252803D094F8B5
:1074F0009E00252809D1B4F8CC02381A00B2002821
:1075000003DB94F8CF0200B105900798D8B1B4F826
:107510003602C0B9D4F8AC0200287DD094F86B00D4
:1075200003F006F94AF2A13101444FF47A70B1FB3D
:10753000F0F0361A94F86B0003F0CEF8D4F8AC12E1
:10754000081A0644203EB4F8361201EB0A00D4F8BB
:10755000641248434100603105980AF06DFACBF897
:1075600014000498DBF81420311AD4F864622069FE
:10757000801BA0F24620CBF81800824200D81046AB
:10758000C4F8300200262E7064202881D4E9A62099
:1075900051187041C5E9041004F12C0009F044FCB5
:1075A000D4F8301208446860D5E90401C4E9A601A2
:1075B000A4F8A072AE72B4F82002C01B00B200287A
:1075C00001DD0220A872089838B3B9F1000F1CD071
:1075D000B4F84812F1B3B4F84A0200BFA4F84A0262
:1075E00094F84C22401C42438A420ED2A87A60B1E1
:1075F000AE72B4F84A02401CA4F84A02FEF7BEFA82
:1076000000F00700401C84F84C0294F8A4022946BC
:107610000AF024FA40B301E009E00BE00D9880F095
:10762000010084F8700200200FB0BDE8F08F40F236
:107630002E511BE0B9F1000FCAD194F85C0200286A
:10764000E3D0D4F864122069411A284609F086F87C
:10765000000400E006E0000CD7D0189901B10880C2
:107660000120E1E70020B9E740F28C513020FBF720
:10767000F9FF0000E000002070B504460BF0F1FFB8
:10768000642801D9054600E0642594F86B002821A0
:107690000AF0F0F82844D4F8641200F510700E18BF
:1076A00094F86B0028210AF0E5F800F529722046CD
:1076B000E16A09F058FB054632462046216909F087
:1076C00052FB09498542C86000D2284688600A7882
:1076D00002B9C860D4F87C02A0F269100861BDE864
:1076E000704006F0C7B80000E00000207CB50446FA
:1076F00006F08EF9D4F89032D4F89422C01A61EBD7
:10770000020100221346121A8B4102DB40F209618A
:107710004DE0421C71F1000102DB40F20A6146E0DB
:10772000226900210AB1B0FBF2F194F89E000D2805
:10773000B4F86E021BD0B4F894205318C31A1BB2CD
:10774000002B01DB401C01E0491C5018A4F86E021C
:1077500094F871028DF80000009800909DF80000E8
:1077600040B9B4F86E02B4F82412884202D1401C29
:10777000A4F86E02B4F8A202401CA4F8A202B4F865
:10778000CE00B4F8CC10401AB4F89410401E08444F
:1077900085B226E001A8002300901A462046FFF794
:1077A00061FD00283AD0012804D040F24961302020
:1077B000FBF758FFB4F86E02B4F82012421A12B266
:1077C000002A09DABDF804200244AA1A12B2002ADB
:1077D00002DAA4F86E1204E0BDF804100844A4F81C
:1077E0006E02B4F86E12681A00B20028D2DA94F869
:1077F000A10088B15FF0080084F8BD000B220849A1
:1078000004F1B40009F077FA20460AF0B7FA2046EE
:10781000BDE87C400AF087B93E20EDE77CBD000062
:107820003510010000000000000001000000000011
:107830000000010000000000141E000030110000D4
:10784000F401FA00960064004B0032001E001400A0
:107850000A0005000200010010B50446D0F8D40269
:107860002169884209D1B4F8D812228B914204D1FF
:10787000B4F8DA12628B914214D02188A4F8CA11AC
:1078800008F089FEA4F8CC01B4F8D802A4F8CE011F
:10789000B4F8DA02A4F8D0010922074904F5DF7030
:1078A00009F03DFA02212046FDF780FD002004F892
:1078B0009E0F0320E07010BD7910010006480549B5
:1078C0000165064941650748054901650649416565
:1078D000704700003D8C000014010020218D000045
:1078E0009D1F0100C0010020C71F01001E481D4947
:1078F00081601E4941601E4901601E4981621E4926
:10790000C1621E49C1601E4981611E4901631E4951
:1079100001621E49C1641E4981641E4941641E49B9
:1079200041631E49C1611E4941621F481D49816072
:107930001E49C1611E4941621E49C1621E49016161
:107940001E4941611E4941641E4941631E498161CE
:107950001E4901631E4981641E49C1641E49816339
:107960007047000061900000140100202D8A000083
:10797000998A00005F1E0100A91E0100598B0000BA
:10798000C11E010025910000F58B0000311E010091
:107990000B1E0100D98F00000D900000999000008F
:1079A000018C000011210100C001002001920000A3
:1079B000991F010031200100731F0100F320010015
:1079C000A1200100D12001008D9100003321010090
:1079D000F71F010021200100EF20010006480549A2
:1079E0008165064901660748054981650649C16503
:1079F00070470000A18D000014010020858E00005A
:107A000057200100C001002081200100F8B57C4C06
:107A10000121A4F110062170002560607580757049
:107A2000357080F82B120088FCF72EFA80B1606860
:107A30000088FCF791FC60680088FCF735FC606802
:107A4000B0F82212C9B180300AF0A7F918B114E0D9
:107A500040F659516CE0606890F830118DF80010D4
:107A6000009900919DF8001039B190F89F200123F2
:107A70001946803008F0A8FD80B1606880300AF0B7
:107A80008CF928B1606890F8260100BF00F0B4FBC3
:107A9000606890F82D1289B1B5801EE06068A0F88A
:107AA000D05090F8311180F828110021022000F008
:107AB00063FE606880F82A520220E7E790F8C6115A
:107AC0008DF80010009900919DF8001019B9C18C33
:107AD000028B914200D8018BB180B0F82612491E6A
:107AE0008FB2B0F828123944A0F8281230F8CC1F11
:107AF0003944018001F0B2FB20B1606850F8C01F2A
:107B0000394401606168B1F82202012802D8401CA2
:107B1000A1F822020FB181F8345281F82A52B1F84B
:107B2000262201F1800008F0F3FE20B14FF45A61E3
:107B30003120FBF797FD606890F89E100A2901D06C
:107B40000B2919D1B0F89420B0F8CC32D21A12B265
:107B5000002A11DBD0F8CE12C0F8A61090F8D2128D
:107B600080F8AA100321FDF721FC606880F89E5080
:107B7000FF2180F8F41026E0252911D1B0F89410E7
:107B8000B0F8CC22891A09B2002909DB80F89E508E
:107B900000F0ACFE0028606880F83C5129D012E06B
:107BA00090F89D10252901D027290CD1B0F8941008
:107BB000B0F8CC22891A09B2002904DB80F89D5064
:107BC00000F094FEA8B10F480090D6E904010E4BD6
:107BD0000E4AFCF74FFC60680123052190F89E20B7
:107BE000803008F0F1FC002809D0BDE8F840FCF72F
:107BF0003BBCBDE8F8400021084600F0C9BBF8BD19
:107C00000C01002091830000CD7E00003988000027
:107C100004480021406820F8D81F8178491C8170F1
:107C2000704700000C010020074810B5416811F8AA
:107C3000DA0F401E40B20870002804DA40F2012139
:107C40003120FBF70FFD10BD0C0100201D4908B5C8
:107C5000496891F89E20C0B1112A06D0152A07D094
:107C6000162A09D01C2A28D109E001210B2008E09E
:107C700014480AF036F906E000F09CFD03E001210B
:107C8000062000F079FD012008BD222A04D02F2A09
:107C900013D101211120F4E791F83C0102280ED004
:107CA00091F83C01012808D191F83D018DF80000C0
:107CB000009800909DF8000008B1002008BD012147
:107CC0001720DEE70C01002038B5002876D13C4CA7
:107CD0006068D0F88C10CA0702D00121092069E041
:107CE0008A070AD501210C2000F046FD606810F8D3
:107CF000DD1F41F0010101705EE04A0702D501215C
:107D0000132057E00A0706D590F8201180F82811B3
:107D1000012107204EE011F0300F47D090F83311C9
:107D20008DF80010009900919DF80010D9BB90F8D3
:107D3000321100258DF80010009900919DF8001077
:107D4000C1B190F89E1025292ED090F89D102529BC
:107D50002AD0002300F2CE2200F5997108F0F5FF39
:107D6000606850F88C1F21F0200141F01001016083
:107D700080F8A650606890F88C10C9061ED508F0EF
:107D8000FFFF05216068FFF737F900F025F961680A
:107D900001F12C00C28BA1F82821408CA1F82A0106
:107DA0000121152006E009E00123D3E7480605D5A7
:107DB0000121242000F0E0FC012038BD002038BD66
:107DC0000C01002070B50D46064608F0FCFE044686
:107DD000304608F0FAFE294600F01EF8B8B12046F9
:107DE00008F09CFC01000DD00A48406890F86B2018
:107DF0008A4207D090F83C11012905D090F867001D
:107E0000204204D0012070BD90F83F01F8E7002027
:107E100070BD00000C01002070B50D46044608F04E
:107E20007DFC50B31649496891F86A20824224D0FB
:107E300091F83C31012B05D091F86630234213D0E4
:107E40001DB11AE091F83E31F8E791F86310214234
:107E500013D15AB1042A0ED004280CD0082A0AD013
:107E6000082808D0824208D9002070BD40F2A31132
:107E70000620FBF7F7FB8242F6D3012070BD00001D
:107E80000C01002010B5104C01230021606890F80F
:107E90009D20803008F098FB40B1606801230421E8
:107EA00090F89E20803008F08FFB08B1002010BDB4
:107EB000606890F8CA000028F9D00021122000F074
:107EC0005BFC012010BD00000C0100200D490246A2
:107ED0004878A0B901F11000406842B189780907DB
:107EE00003D590F89F00072809D00120704700F1C2
:107EF0002C018A8C818E8A4201D8FFF759B8002064
:107F000070470000FC00002038B5324C0546606820
:107F1000803009F042FF00285BD1002D59D1606804
:107F20000123194690F89F20803008F04DFB00286F
:107F30004FD1606890F830118DF8001000990091D1
:107F40009DF80020002142B1A0F8D01090F8311126
:107F500080F828110021022030E090F89E200123B3
:107F60000421803008F030FB0546FFF7ADFE002805
:107F70002FD12846FFF76AFE00282AD1FFF782FF9B
:107F8000002826D1606890F89D1009291AD0002D8C
:107F90001FD100F01DFB00281BD1606801230021C8
:107FA00090F89D20803008F00FFB002811D0606809
:107FB00090F8C40200280CD00021FF20BDE8384012
:107FC00000F0DABB90F8211180F828110021072079
:107FD000F4E738BD0C0100200848436893F86000BE
:107FE000012806D003F5B17203F12C011888FDF7C2
:107FF00047BD022083F86000704700000C0100209C
:10800000F8B52B4D060005F1100433D100F0AAF8A5
:1080100000F052F806002DD16988480706D560683F
:1080200090F89F00062801D101202870880716D5F6
:10803000A868C0782B2807D21E4951F8201019B122
:108040001B48103088470AE0FF2804D040F6021190
:108050003120FBF707FB1648103009F081FFA878A4
:10806000C00607D5606890F89E100A2902D10B213E
:1080700080F89E106878000718D5606801230521F4
:1080800090F89E20803008F09FFA08B108260DE095
:108090000025694603200095FCF7AEFA009828B148
:1080A00005722A226168009808F025FE3046F8BD66
:1080B000FC000020C001002070B5284D0020A978E8
:1080C000C90717D0E86805F110040123C678606875
:1080D000052190F89E20803008F076FA58B1B61E3F
:1080E0000A2E06D2DFE806F0070705050707050593
:1080F0000707082070BDE868FDF778FA38B3E8682C
:10810000C5781DB1012D01D0162D13D1606890F8EE
:108110009D0008F0B1FA68B1616891F89D002028CF
:1081200008D0212803D0162D0FD0022070BD2E209C
:1081300081F89D002B2D0AD2094850F8251031B145
:10814000BDE87040054810300847202070BDBDE8EC
:1081500070400248103000F059BD0000FC000020C3
:108160001401002070B5234EB078000740D506F109
:1081700010046068803009F010FE48B16068FE218C
:10818000002580F8261190F89E101A290CD104E0E1
:1081900040F60E113120FBF765FA80F8DB50FFF74F
:1081A00043FD606880F89E50606890F89D1020291B
:1081B00002D0312913D10BE090F89E0008F05CFA50
:1081C00008B12E2000E02120616881F89D0006E0C2
:1081D000012180F8C51280F89D5080F8D650606863
:1081E00090F89F10072903D10221317080F82611E1
:1081F00070BD0000FC00002038B505466846FCF75D
:1082000095F808B32222002100980BF02EFC0321E0
:10821000009808F0F2FC0098017801F0EF0101707D
:108220002946FDF7F3F9594C112D2DD00FDCA5F19E
:1082300002050D2D1FD2DFE805F0211E519E9E2163
:108240001E5E1E9E3A348C0040F6B53199E0172D23
:1082500070D008DCA5F11205052D0CD2DFE805F081
:108260008B8B50503300232D77D0242D75D0252DA6
:1082700073D0FF2D77D040F6614182E060680099AD
:1082800090F82801087176E0606890F82311009852
:1082900008F09FFC606890F82211009808F09DFC9F
:1082A00069E06168009891F82211017163E000981B
:1082B0000C21017159214171002181714B21C17142
:1082C0001221017257E00098D4F8041091F83E1181
:1082D0000171616891F83F1141714CE0616800984B
:1082E00001F5107108F030FC6168009801F58E719D
:1082F00008F027FC3FE025480099FDF7D7FC3AE05D
:108300006068B0F84C10009808F07FFC6068B0F826
:108310002A11009808F07DFC6068B0F848100098B9
:1083200008F07BFC6068B0F82811009808F079FC30
:1083300021E0FFE7616891F83C0101280098C5D071
:1083400091F866100171616891F86710C4E704E064
:1083500009E00098FDF75AFC0DE00C4A2846009908
:1083600009F03BFF07E0606890F8C722D0F8C81218
:10837000009808F034FCFBF7B3FF002804D140F666
:1083800065413120FBF76EF938BD00000C0100207B
:108390002DE9F35F8C4E8A4670680088FBF774FD08
:1083A00007000CD0A6F110054FF000046888C00546
:1083B0000AD57068A0F8CC4080F8344209E040F655
:1083C00045713120FBF74EF9716831F8CC0F401C34
:1083D000088000F043FF4FF0010940B368880005B2
:1083E00006D5706890F8A31011B1C0F8C0401EE027
:1083F0007068D0F8C010491CC0F8C010D0F8C42074
:108400008A4201D3531A00E00023B5F804C00CF1EE
:10841000050C634501D880F8CA90914207D3C0F893
:10842000C0400F22694900F5AC7008F078FC6888FC
:108430004FF0020B10F4407F0ED0706890F8A1103E
:1084400011B1032908D102E080F8A19001E080F881
:10845000A1B00121FEF7D0FD7068B04690F8A110E0
:10846000012904D16988490501D580F8A1B0009996
:10847000002979D1A978490602D5A0F8484204E03C
:10848000B0F84812491CA0F848125046FFF7B8FD52
:1084900040EA0A008246FFF737FDD8F80460B6F8D4
:1084A0002802401CA6F8280296F82C0228B1FCF7F6
:1084B000E1F8B0B1A6F8284213E0FBF7B9FF08B124
:1084C000A6F82842FBF7AEFF58B196F83402401CDC
:1084D000C0B286F83402022803D9A6F8284286F8EA
:1084E0003442D8F804004646012390F89E2000212B
:1084F000803008F069F820B9706890F89E000B2869
:108500005FD170680123002190F89D20803008F031
:108510005BF850B370680123002190F89F208030F1
:1085200008F052F808B3706890F8A110022948D1F9
:1085300090F83402C8B9384607F03EFBA8B170681D
:10854000803009F02AFC80B97168B1F82202012854
:1085500037D981F82A92B1F8CE20B1F8CC00931E19
:10856000984203DB012004E01CE02AE0101A401EC0
:1085700080B2B1F82832AA88934201D3012202E0E6
:10858000D21A521C92B2904200D91046012801D151
:1085900081F82A427168B1F894201044A1F82402AD
:1085A00000F028FFA8785246C0F38011009800F030
:1085B00069FED8F8040080F82B42BDE8FC5FFBF7A9
:1085C00079BE01207168E3E70C01002081110100F0
:1085D0007CB5684C01230021606890F89D208030B4
:1085E00007F0F2FF00287AD0606890F84311002568
:1085F00039B100210E2000F0BFF8606880F84351C7
:10860000B5E090F8421119B190F8DD10890716D045
:1086100090F832118DF80410019901919DF8041021
:1086200041B190F833118DF80010009900919DF838
:10863000001089B190F83C11012930D040E00021B0
:108640000C2000F099F8606810F8DD1F41F001017E
:10865000017080F865508AE090F89E1025291CD0A2
:1086600090F89D10252918D05FF0000300F2CE226B
:1086700000F5997108F069FB606880F832510021BB
:10868000142000F079F8616801F12C00C28BA1F888
:108690002821408CA1F82A0169E00123E6E790F83F
:1086A0003D118DF80010009900919DF8001039B926
:1086B00090F89E2001230B21803007F085FF78B1D0
:1086C000606890F849118DF80010009900919DF8AC
:1086D0000010B9B30021232000F04EF847E030E04D
:1086E000606890F86A0009F060FB0546606890F8E1
:1086F0006B0009F05AFB0646606890F83E11284668
:1087000009F05EFB50B1606890F83F11304609F007
:1087100057FB18B1002000F041F911E06068012317
:10872000032190F89E20803007F04EFF40B960682A
:108730000123022190F89E20803007F045FF10B100
:1087400000207CBD02E000211620C5E790F846011C
:108750008DF80000009800909DF800000028F0D0EF
:108760000021252000F008F8606880F846510120BB
:10877000E7E700000C01002070B50D4C06460D46E1
:108780006068803009F009FB20B140F66A41312071
:10879000FAF768FF62680020012D82F8266104D094
:1087A00022F8D20F0120107170BDA2F8D80070BD60
:1087B0000C01002038B51F4C0025606890F8B012FD
:1087C00001290CD0022933D190F8DC1000294FF098
:1087D00006011AD080F828110121022023E090F828
:1087E00012128DF80010009900919DF800100029D8
:1087F0001ED100F5847300F50E71002200F2B12045
:1088000007F09AFE012105200DE0032000F0B4FCE2
:10881000606890F8EC00800810F0010F01D0112082
:1088200000E00D200121FFF7A7FF606880F8B0523B
:1088300038BD00000C01002070B52B4B0246588853
:108840001043588003F11000402A40680DD096076D
:108850004FF000054FF001044FEAC2760CD54EB13F
:1088600040F6B2613120FAF7FDFEBDE87040042108
:10887000FEF7C2BB99601CE0C6B1D960C978062971
:1088800002D00B2912D109E090F89E1018290DD1C1
:108890000021C0E93E1180F8A24007E090F89E1048
:1088A000122903D180F8A25080F8DC40910716D538
:1088B0009968C978052902D00B2910D109E090F8F0
:1088C0009E1016290BD10021C0E9401180F8A34069
:1088D00005E090F89E10112901D180F8A350900670
:1088E00001D50820587070BDFC0000202DE9F04132
:1088F000294C0125636893F8CE1209B1012700E0E5
:10890000002793F8CF0208B1012600E000260FB936
:1089100093F86A100EB993F86B0083F86A1083F825
:108920006B0003F16202FF209072184609F017FDF8
:10893000606890F83C01012801D007B916B1002009
:1089400000F02CF860682C3008F06EFA064660687B
:1089500008F016FA30B1616801F5B17231F82C0BEC
:10896000FDF78EF805216068FEF746FB60682C3045
:1089700008F05AFA0446A6420AD203F08FFF0146D5
:10898000A01B652800D2652003F0AAFE00B10025D7
:108990002846BDE8F08100000C01002010B5104C05
:1089A00061680A88A1F8A62181F8A40191F86A00FB
:1089B00009F0FBF9616881F8A80191F86B0009F0F2
:1089C000F4F963681522074983F8A90103F5CD700E
:1089D00008F0A5F96168002081F83C0110BD000095
:1089E0000C0100203F32010070B50F4D6C6894F807
:1089F0009D10212902D02E2903D011E0FFF7CEFFD0
:108A000008E094F89E2004F1800001230B2107F078
:108A1000DBFD38B16968002081F89D0081F8D6003F
:108A2000002070BD2A20E9E70C01002070B5044643
:108A300040680123002190F89E20803007F0C4FD9B
:108A4000B8B1134DE86808F02AF86168A1F8CC02C3
:108A50006168B1F8941009F0C1F960B1616828202B
:108A60000B2281F8BD0060680A49B43008F043F970
:108A70000BE0012070BD6168E86801F2CE2108F0CA
:108A800009F861680A2081F89E00002070BD00008E
:108A9000FC0000203510010070B504464068012339
:108AA000002190F89E20803007F08EFDE0B1284D27
:108AB0000021E86807F0F6FFC0B1E8686168B0F827
:108AC0000D00A1F8CC026168B1F8941009F086F9A4
:108AD00088B1616828200B2281F8BD0060681D49BB
:108AE000B43008F008F930E0012070BD2046BDE840
:108AF000704000F08BB8E86807F0FEFF07F047FD14
:108B0000064660683146C0F8D462E868007907F02C
:108B1000BAFE6168A1F8CE02E8683146B0F80500F7
:108B200007F0ADFE6168C1F8D002E86807F0E7FF22
:108B30006168A1F8D802E86807F0E4FF6168A1F86D
:108B4000DA0261680D2081F89E00002070BD0000EF
:108B5000FC0000203510010070B504464068012378
:108B6000002190F89E20803007F02EFD70B96068DB
:108B700090F89E20132A09D001230521803007F0A8
:108B800023FD08B1082070BD012070BD606890F819
:108B9000DC0008B9FFF73CF8144D616801F50E716F
:108BA000E86807F0C8FF6168E86801F58C7107F0B4
:108BB000B9FF60680188A0F8E6126168E86801F50D
:108BC0003A7107F0B3FF6168E86801F53C7107F09E
:108BD000A6FF60680A22064900F5377008F08BF896
:108BE0006168152081F89E00002070BDFC00002007
:108BF000EB1001000149C968FCF7E6BFFC0000204A
:108C00000149C968FDF710B8FC00002010B54268A2
:108C1000D2F88C100B0701D5012010BD41F00801DE
:108C2000C2F88C1004494068C968C97880F82011DE
:108C3000FEF7EEFF002010BDFC0000202DE9FC41F6
:108C40000546406890F88C0010F0300F02D00120EB
:108C5000BDE8FC81314CE06807F087FF30B3E06885
:108C600007F07DFF8046E06807F07DFF0746E0687B
:108C700007F073FF0646E06807F073FF0146CDF882
:108C8000008068683B4632462C3008F007F9A0782F
:108C900081074FF0010003D5A168C97814290AD0D3
:108CA000696891F89D101D2905D007E02846BDE8A8
:108CB000FC41FFF7ABBF696881F86000686890F815
:108CC0006010012911D090F833118DF8041001992A
:108CD00001919DF8041041B990F832118DF80010FF
:108CE000009900919DF8001041B150F88C1F41F09F
:108CF00010010160FEF78CFF0020A9E750F88C1FDF
:108D000041F02001016005481030436803F12C0157
:108D1000188803F5BC72FCF7DDFEEBE7FC000020D1
:108D20002DE9F8430446406801230A2190F89D206C
:108D3000803007F049FC70B3184DE86807F015FF64
:108D4000E8B1E86807F00BFF0746E86807F00BFF9B
:108D50008046E86807F001FF0646E86807F001FF73
:108D6000014600976068434632462C3008F096F87A
:108D7000606808F005F805216068FEF73DF9616854
:108D8000002081F8D600616881F89D00FFF724F982
:108D90000020BDE8F883FFE70120FAE7FC0000208F
:108DA00038B50446406801230B2190F89E2080309E
:108DB00007F00AFC60BB60680123002190F89E2048
:108DC000803007F001FC08B3606890F89D0025280A
:108DD0001ED02A4DE86807F0DAFED8B1E86862686C
:108DE000417901F0070182F86310007900F0070172
:108DF000606880F86210606890F83D218DF800206E
:108E0000009A00929DF800207ABB08E0012038BD4E
:108E1000202038BD2046BDE83840FFF7F7BE90F867
:108E20003C21012A21D000F16A0290F86330557884
:108E30008D4206D11178994203D1022180F83C116C
:108E400013E00E481030416801F5CB700A8820F815
:108E5000022B91F8622000F8012B91F8631000F8C2
:108E60000D192222064907F046FF6168222081F889
:108E70009E00FEF7CDFE002038BD0000FC00002063
:108E8000693201002DE9F8434568044695F89D00D4
:108E9000212808D05FF0000695F89E00232804D012
:108EA0008EB39D3502E00126F6E79E35DFF820817E
:108EB000D8F80C0007F077FE002740B33146D8F809
:108EC0000C00FEF77FFF10B36A4646466068D8F88C
:108ED0000C1007F08EFCC0B3F06807F062FE61680A
:108EE000A1F8CC026168B1F8941008F077FF68B37C
:108EF000616828200B2281F8BD0060683549B430D4
:108F000007F0F9FE58E0FFE70220BDE8F88360684B
:108F10004FF0000990F83C11012918D080F83C71FD
:108F20000EB3D8F80C0061680122C07881F82101E5
:108F300082406168C2F3006068B1092081F89D0039
:108F4000606890F8D600A8B908E015E028E01E2077
:108F5000FFF724FDE4E740F2834101E040F28B415A
:108F60003120FAF77FFB2F70FEF75EFE2046FFF7F9
:108F70004DFE81464846C8E7606890F83C110129DB
:108F800009D080F83C71606800F19E01A94213D1BC
:108F900080F89E7010E00020FFF700FD2F70F2E7D0
:108FA00061689DF8000081F8CE0261689DF80100BB
:108FB00081F8CF0225202870606800F19E01A94247
:108FC00002D1FEF731FE01E080F8D67000209CE768
:108FD000FC0000203510010070B5044640680A4DC1
:108FE00010F8EC1F41F004010170E86807F0EFFD94
:108FF0000646E86807F0EFFD014622463046BDE828
:10900000704000F095B80000FC00002002461348B4
:10901000C068017911481030436893F89D002128F9
:1090200010D02E280ED028280ED004280ED00F28BD
:109030000ED01D280ED093F89E0023280CD0FE20C1
:1090400000F076B81620FBE72320F9E70E20F7E7BB
:109050001220F5E71420F3E71720F1E7FC000020C9
:1090600010B5044640680123194690F89F208030CF
:1090700007F0AAFA08B1002010BD0648C06807F042
:10908000D4FD616881F8A0006168062081F89F0026
:10909000F1E70000FC00002070B504461F480025E1
:1090A000C06803796068162B90F89D0013D006DC29
:1090B0000E2B09D0122B07D0142B2CD104E0172B28
:1090C00002D0232B27D11FE022460121184609F0A8
:1090D00032F805461FE0212801D02E281BD120465A
:1090E00008F088FE606890F89E10222913D00821AD
:1090F000EC3008F033FE60680B21EC3008F02EFEF7
:109100001A20FFF74BFC06E0282804D10448016828
:1091100009B120468847284670BD0000FC000020A9
:10912000700200200149C968FCF7F2BDFC00002074
:1091300003460020172B17D00ADC0E2B14D0122B5D
:1091400012D0142B10D0162B12D10846FFF74CBCAE
:10915000232B03D0242B01D0252B09D1054A1268DB
:10916000002A05D0184610470021184608F0E3BF32
:10917000704700006C020020034A526882F8230105
:1091800082F82211704700000C01002070B50446DF
:10919000406890F89E101C2904D040F64E01312002
:1091A000FAF760FA002580F8DB50606890F8DC1070
:1091B00061B180F8DC5060680D220188A0F81612B9
:1091C00060680D4980F8145260680CE00188A0F8CE
:1091D0001612606880F81452616801200C2281F830
:1091E00018020649606800F20A2007F084FD6068F2
:1091F00080F89E5070BD0000D5100100B71001002E
:10920000154910B589680A79416891F89D30092B94
:109210000AD191F82131934206D1002281F89D2094
:10922000406880F8D62010BDD1F88C301C0707D5D7
:1092300023F00800C1F88C00BDE81040FEF7F4BC34
:10924000FF2A04D040F2EA713120FAF70BFABDE8A8
:10925000104008F085BE0000FC000020084810B552
:10926000406890F8A31041B990F89E200123062190
:10927000803007F0A9F9002800D0012010BD0000BF
:109280000C010020F8B5594C0646154660680022CE
:1092900011B1A0F8362206E0B0F83612B0F8262256
:1092A0001144A0F8361290F830118DF80010009992
:1092B00000919DF8001039B990F89F2001231946BC
:1092C000803007F081F930B1606830F8D01FB0F815
:1092D000562111440180606890F8D62032B1B0F870
:1092E000D210B0F826321944A0F8D21090F9DA3032
:1092F000002B06DDB0F8D810B0F826723944A0F87B
:10930000D81090F8BD1009BBBEB93849103909789A
:10931000022906D001290AD0F5B1E9060BD51E2194
:1093200042E090F8281106293ED016213CE090F842
:10933000A01059B954E0290701D53D2134E0A90610
:1093400001D5232130E0A90701D02A212CE040F6E5
:109350005E613120FAF786F92AB1B0F8D210B0F880
:10936000D420914216D2002B05DDB0F8D810B0F809
:10937000D42091420ED2B0F8D020B0F8CE108A425C
:109380000AD390F830218DF80020009A00929DF8C1
:1093900000200AB1222107E090F8A12072B1B0F8B4
:1093A000CC208A421CD3082190F8BC208DF80020E4
:1093B000009A00929DF800206AB905E0B0F8CC1040
:1093C00006290DD33E21EFE780F8BD100B22084996
:1093D000B43007F090FC6068BDE8F84008F0CEBCFF
:1093E000BDE8F8400021FDF707BE00000C01002099
:1093F0003510010070B52E4D686890F8A11051B17C
:10940000012908D0022909D0032907D040F6D74105
:109410003120FAF727F9B0F8241237E090F89F10BE
:10942000072936D0B0F8CC20B0F8CE100024931C19
:10943000994206D3891A891E0C04240C01D0641E9B
:10944000A4B290F8CA1039B190F89D2001230921E7
:10945000803007F0B9F840B3FFF700FF78B16A68D1
:109460000020D2F8C410D2F8C020931C994203D334
:10947000881A801E00D0401EA04200D284B20CB1D7
:10948000641EA4B26868B0F824122144A0F8201227
:1094900070BDB0F8CC100329BDD330F8941F428FB3
:1094A0001144491CA0F88C1170BD0024EAE70000AB
:1094B0000C01002070B544680D2204F59875002158
:1094C00004F16F000AF0D1FA4FF4A3700021A4F860
:1094D00044110155A5F81710697608465FF07F0121
:1094E00004EB4002401CC0B282F874100228F7D38B
:1094F00094F96E10204608F00CFF0020FF2122187E
:10950000401CC0B282F877100228F8D370BD00006A
:1095100003494A8802800978817000207047000062
:10952000A82500203EB50C4605460088694607F090
:1095300021F8002228B1C4F80220A2712280022062
:109540003EBD019911F1800181F87420D1F8260007
:10955000C4F8020091F82A00A0712888208091F8B0
:1095600074008DF80800029802909DF80800002809
:10957000EAD13EBDFEB50D4606460088694606F0B6
:10958000F9FF00281AD1DDF80440002784F86C7038
:1095900014F86A0F09F03BFCA870607809F037FCFA
:1095A000E870A0788DF80800029802909DF80800F5
:1095B0006A3C0028EAD1308828800020FEBD0000E7
:1095C00003498A880280C9884180002070470000D2
:1095D0007C0200203EB5002402A98DF804408DF8DD
:1095E0000840009182784178007801AB09F08AFD4B
:1095F000002812D19DF8040009F0BDFC70B19DF85F
:10960000080009F0B8FC48B105489DF804108173C2
:109610009DF80810C173048200203EBD11203EBD9C
:10962000A82500202DE9FC410F460546067809F0E3
:1096300055FC00280AD1284609F02AFC002805D14B
:109640000120FAF703FA864202D30720BDE8FC8125
:109650000121304606F004FD040004D008F0A0F813
:1096600068B10C20F2E70121304606F0EFFC04005F
:1096700013D0174890F90010204607F053FE2046FB
:1096800007F0BBFE3870E87429462046FCF7E6FC7C
:109690000646687ED0B12EB118E041F2E83139209B
:1096A000F9F7E0FF00226846616B06F08BFD0022AF
:1096B0000121606B06F000FE04226846616B06F033
:1096C00081FD00221146606B06F0F6FD3046BDE7D5
:1096D00074020020017871B1417861B141881B2981
:1096E00009D381881B2906D3044902680A6080884F
:1096F000888000207047122070470000A8250020B5
:10970000006840F2E241884203D3034988600020A8
:109710007047122070470000A8250020034AD2E9B4
:10972000041201604260002070470000689C000045
:109730000EB50088694606F01DFF60B9019809F072
:1097400096FC40B10198014690F84221803001F525
:10975000A17162B901E002200EBD90F866208DF87B
:109760000820029A02929DF8083001220BB13A209B
:109770000EBD90F85D309B0706D0032205495E3090
:1097800007F0CDFA00200EBD0A70684607F090FA87
:10979000F8E700009311010010B5052000F0F6FA7B
:1097A000FEF78CF802490148486010BDE1970000BF
:1097B000740200201CB50949D1E90001CDE900017E
:1097C00005E0009807F0ECFF08B101201CBD6846D9
:1097D000FAF786F90028F4D000201CBD689C000030
:1097E0002DE9FE431346334A0F46B0F8541014884F
:1097F000B0F852608C4200D2214688469188B1422E
:1098000000D20E46518840F64804A14200D32146BA
:10981000D588A54200D32546A14200D20C464FF47C
:10982000A4721B2E01D0954204D1B8F11B0F3ED07B
:1098300094423CD06A46194609F0C0FBBDF80600C8
:109840004146404500D90846F880BDF80810A142BD
:1098500000D80C463C81BDF80210B14200D80E463B
:109860007E80BDF80410A94200D80D46BD80FF21BE
:1098700039701B38E02802D940F66E5114E01B3EC7
:10988000E02E02D94FF457610EE04FF4E060A4F5EA
:10989000A474844202D940F6725105E0A5F5A4757E
:1098A000854204D940F674513920F9F7DBFEBDE852
:1098B000FE8300007C02002010B50D4800210D4BF6
:1098C000C17481821B221A804FF4A4745C809A8038
:1098D000DC808173C17303230370022343704280D1
:1098E000828040F6A66282608174017310BD000020
:1098F000A82500207C02002010B50121002006F0E0
:10990000AFFB04000AD1012106F0A0FB040007D040
:10991000064890F90010204607F004FD204610BDCF
:109920004FF42C713920F9F79DFE000074020020DD
:109930002DE9F04387B00C468046054607F060FDF0
:1099400098B1284607F04FFD30B1B4F8011012204D
:1099500000290BD0802909D8284607F035FD40B1F1
:10996000404607F0A0FC30B109E0422007B0BDE856
:10997000F0830C20FAE7404607F02FFDC8B34046BD
:1099800007F00EFF0028F4D1404607F0A7FC00289E
:10999000EFD14046FCF700FBB4F8010042F2107131
:1099A00000FB01F9E178404607F005FD404607F06D
:1099B00016FD08B3002101A8FAF7B2F804007BD025
:1099C0000021FBF7F3FCBDF804002080214640464F
:1099D00007F02DFD00F0E6F9400940EAC160C0073C
:1099E000414D04F12C0011D06988AA88C1840285F8
:1099F0000FE0FFE71220B9E74A4600214046FDF795
:109A0000E9F90028B2D041F222615FE01B22C28452
:109A1000028500F0C7F988074FF0010605D58DF8DB
:109A2000086002A80394FFF745FDA868E06241F6CC
:109A30004C57404607F0DBFC10B9404607F0F5FCF8
:109A400027612188ADF80810A97B8DF80A10E97B01
:109A50008DF80B10298AADF80C1005A9009130463D
:109A600004AB02AA214609F0DFFA40B10021BDF89B
:109A70000400FAF77DF8F0B141F27C6126E09DF830
:109A800010008DF818009DF814008DF81900BDF82D
:109A90000C00ADF81A0006A9204606F03BFE6878D7
:109AA00000902B78AA8869882088FAF717F928B1DE
:109AB00041F287610AE0FFE7092057E74A4621465D
:109AC0004046FDF787F920B141F289613920F9F765
:109AD000C9FD0648436823B1002204F59971204668
:109AE0009847002042E70000A825002074020020CB
:109AF0002DE9F04188B00446008806A906F03AFD39
:109B0000002847D1079890F880118DF80810029925
:109B100002919DF80810803001B101218DF80C10E0
:109B2000017B4FF00008890602D59DF80C1049B161
:109B30005FF000018DF8041005216C3008F059FC2D
:109B400010B104E00121F5E79DF8040008B3218974
:109B5000E08809F025FA00281CD1A188608809F066
:109B60001FFA002816D12189E08809F00FFA002891
:109B700010D1A188608809F009FA06000AD1079877
:109B800000F59975FF276F709DF80C1029B13A26E2
:109B90002EE01A2008B0BDE8F081414603AA09F082
:109BA0000DFA6188BDF81200814200D20846E880B3
:109BB000A188BDF81400814200D208462881E288BD
:109BC000BDF80E108A4200D2114669802289BDF884
:109BD00010108A4200D2114640F64802A9809142F4
:109BE00000D31146A980904200D202462A812F70EC
:109BF00085F801803046CDE71CB50C49D1E902015A
:109C0000CDE900010AE0009C204607F0C9FD28B11B
:109C1000204607F01BFC08B101201CBD6846F9F77F
:109C20005FFF0028EFD000201CBD0000689C0000F2
:109C300010B50446C188808809F0B2F900280FD118
:109C40006188208809F0ACF9002809D10548A1886D
:109C5000818021880180E188C18061884180002065
:109C600010BD00007C020020000000000000010088
:109C700000000000000001000C4B120C59004B12B8
:109C800000000000000001000000000000000100D2
:109C900010B5FBF72DFE054C606809F08FFA09F04E
:109CA0002DF8FBF75FFF0120207010BD840200201B
:109CB00001480078704700008402002010B5064C6F
:109CC000A06809F07BFAE06809F078FA09F07BF8FF
:109CD0000020207010BD00008402002010B505494E
:109CE000054809F05EFA0448BDE810400349001D2C
:109CF00009F057BA94020020880200209C0200203C
:109D000010B50849084809F04CFA07480749001DF2
:109D100009F047FA0448BDE810400549083009F049
:109D200040BA0000AC02002088020020B4020020EB
:109D3000A4020020014840787047000084020020FF
:109D400010B5FCF74BFAFDF7F5F8BDE810400148F7
:109D5000FCF72ABAC12C00200A4910B5012048702E
:109D6000FCF76CFAFDF7C2FD06F027FB0649A1F5EA
:109D70008170FAF763FB002006F04FF9BDE8104050
:109D8000FBF7BCBD84020020C32D0020044AC1089B
:109D900000F0070301209840535C0343535470477D
:109DA000200000200149D1E9000170472000002077
:109DB000064801880079020642EA112000F00100FD
:109DC0000018C0B240F001007047000020000020E1
:109DD00010B504F04BFE0022084B114633F8214029
:109DE000844203D303EB8100827803E0491CC9B2AB
:109DF0000C29F3D30248027010BD00000E3201009E
:109E00007303002070B5054616460C46022000F08C
:109E1000B7F906490120F61E087005480660044897
:109E200008380560001F046070BD00007403002046
:109E300010F5004010B50C4C207880B10B494FF460
:109E40000000086000F06AF8002120B10120607075
:109E50000748006801E061701020A0702170BDE823
:109E60001040002000F08CB97403002008F5014078
:109E700000F4004010B5022000F082F904490120EE
:109E8000087000F059F803494FF40000086010BD55
:109E90007403002004F50140034800210170417063
:109EA000102181707047000074030020074810B52E
:109EB000017841B100F032F818B105480068C0B22D
:109EC00010BD102010BD807810BD0000740300206C
:109ED00000F40040084810B5017859B10748D0F89F
:109EE000000128B100F00CF8002800D0012010BDBE
:109EF000022010BD407810BD7403002000F0004027
:109F00000548D0F8041111B1D0F8080108B10020BB
:109F1000704701207047000000F00040054810B570
:109F2000D0F8000120B1FFF7EBFF08B1012010BD10
:109F3000002010BD00F0004004480021C0F80011CE
:109F4000C0F80411C0F808117047000000F000408C
:109F50002DE9F04104461E4690460F46012000F0D0
:109F60000FF91E4D1E4804F003012E7100683204E3
:109F700061F3070066F30F20000C1A4E42EA0060FE
:109F80000843C6F804051848076009F069FC38B9A9
:109F900015481030016821F0FF0141EA0801016015
:109FA00000F0E4F80CB1042C07D111480D490F4A18
:109FB000091DC0F81025C0F8141501206870EC7058
:109FC0001CB1012C01D0022C06D128700021C6F84A
:109FD0000011C6F800123060BDE8F0817703002060
:109FE0007CA1000000F0004008F5004000F10040B6
:109FF00088F0014070B51C4A5378A3B11B4B19601F
:10A00000191D0860012595701046D678184B007808
:10A01000184C002156B1042E1BD008B3C4F804110B
:10A020006806186070BD40F2BD111AE078B1204694
:10A03000C4F804114FF400361E60711209F05FF984
:10A040000028EFD065600A48001D066070BDB3218E
:10A0500007E01570C4F80411C4F80052256070BD03
:10A06000C6213C20F9F7FEFA770300200CF50040EA
:10A0700004F5014000F0004070B5054D002428783B
:10A0800010B100F073F82C706C70AC7070BD0000F3
:10A0900077030020024800210170417081707047F1
:10A0A000770300200B4810B5007858B14FF4827147
:10A0B000094809F024F940B108480068002800D098
:10A0C000012010BD40F2232101E04FF409713C2032
:10A0D000F9F7C8FA7703002000F0004000F40040D0
:10A0E000014801218160704700F000402DE9F047F0
:10A0F0001B480078D8B1DFF86C804FF48276314687
:10A10000404609F0FCF8002828D10220C8F80403D2
:10A11000154C2068C04340F30015206840F0100043
:10A1200020604FF400474FF0E0296D1C08E040F23A
:10A130002F213C20F9F796FAC9F8807209F0D0FB7C
:10A140003146404609F0DBF80028F5D01DB92068FB
:10A1500020F0100020600220C8F80803BDE8F08756
:10A160007703002000F0004010ED00E002490148B4
:10A17000086070470000020208F50140000001007D
:10A1800010B5044600F020F8002C0ED00B4A0B4806
:10A190000B491432012C05D0022C07D082213D201E
:10A1A000F9F760FA02230360116010BD0323036016
:10A1B000116004494FF40000086010BD00F5004034
:10A1C000C52E002004F50140054810B500210160AE
:10A1D0000160FFF751FF03494FF40000086010BD14
:10A1E00000F5004008F501400548D0F8001221F0C4
:10A1F0004001C0F800120021C0F86015704700004F
:10A20000001000400449C1F86005D1F8000240F098
:10A210004000C1F80002704700100040014890F86B
:10A22000220070470C2600200249085C00F51660E9
:10A23000704700007EAF0000F8B5244CD4F804034A
:10A2400010F0100F01D0012700E000271020C4F803
:10A2500008030220C4F800021D4800251D4980F8AB
:10A260002C504FF460200860D4F850054FF48876E5
:10A2700010F0FF0F19D0FF208DF80000C4F8105126
:10A280000120206105E000BF9DF80000401E8DF810
:10A2900000009DF8000028B13146204609F05EF824
:10A2A0000028F1D09DF8000058B100F057FCC4F828
:10A2B000105100F0E5FD002F02D01020C4F8040377
:10A2C000F8BD40F6AA013E20F9F7CCF90010004095
:10A2D0000C26002008F501402DE9F041184D0746F5
:10A2E00095F82C00C2070FD0164CD4F8002242F08B
:10A2F0000102C4F8002240F0020085F82C0001267B
:10A300003FB1012F0BD010E040F285713E20F9F7EC
:10A31000A9F9084600F00EFE6E72266005E00846B8
:10A3200000F0EEFD0220687266600748C6640648C9
:10A330000C30D0F840153846BDE8F04100F072BD51
:10A340000C26002000100040008000402DE9F0475E
:10A350002C4C06002C4D94F82C00DFF8B08040F017
:10A360000200894684F82C004FF0000702D0012E2D
:10A3700020D036E0084600F0DDFD01206072E07973
:10A38000012805D1D5F8000240F00800C5F8000208
:10A39000A06A40F48010A0624FF48010C8F800005A
:10A3A0001B4931F819004FF47A7100F5FA70B0FBCF
:10A3B000F1F716E0084600F0A3FD02206072E07994
:10A3C000012805D1D5F8000240F00400C5F80002CC
:10A3D000A06A40F40010A0624FF40010C8F800001A
:10A3E000292700F027FC09F033F920B1FFF724FFFB
:10A3F0000020BDE8F0870021304600F013FD38460C
:10A40000F7E700000C2600200010004004F5014092
:10A4100078AF0000024A136B0360506B086070470E
:10A420000C26002010B51DC8014981E81D0010BD93
:10A43000FC2500200F4910B5CA69824202D340F6BC
:10A440003A110BE001220A7308610B494A640A1DA4
:10A45000D2F84035834204D340F643113E20F9F749
:10A4600001F90023C1F84431C2F84005BDE81040AD
:10A4700000F0ACBC0C2600200080004070B50F4CF2
:10A4800003460220207394F82150962094F820105F
:10A49000227D012D0ED000F0ABFD20610848002187
:10A4A000C0F844112169E06908440549091DC1F853
:10A4B000400570BD00F0BAFDEFE700000C2600205B
:10A4C0000080004010B509F0E7F9002806D00448E4
:10A4D000016821F0010141F08071016010BD0000B0
:10A4E000741700402DE9F04138220021134809F08B
:10A4F000BCFA00F0C5FC09F088F9114D104E00249B
:10A500000F4F0835103628B909F096F910B909F03F
:10A510009DF908B1242206E009F0D8F910B909F034
:10A52000CBF940B14022FF21384609F09EFA2C6059
:10A530003460BDE8F0813822F5E700000C260020E9
:10A54000000E00400148C069704700000C26002042
:10A5500001488069704700000C26002010B500F00B
:10A5600043FCFFF769FE04F01DFD30B1401C04D030
:10A5700040F26D513E20F9F775F80F480F4A816A95
:10A5800041F044611160002484620473C4618461F9
:10A5900000F02AFC0A48C0F84841C0F84441C0F81D
:10A5A0004041C0F84C41012008F0C7FEBDE8104012
:10A5B000012008F0B5BE00000C26002008F501407F
:10A5C0000080004070B5012008F0B7FE374C002035
:10A5D000C4F8FC0F0120C4F8FC0F09F04DF9344D0C
:10A5E00018B1286840F48060286009F039F928B172
:10A5F0002868304920F069000843286009F04CF9C8
:10A6000038B12B48001D016821F47F4141F4B0515D
:10A610000160274928483C31086004F0FDFC40B146
:10A620004FF08050D0F83003411C02D02049103147
:10A6300008604FF01020006E411C04D01F490A68CA
:10A6400060F317420A6040F2031140F25B60C4F805
:10A650003415C4F838050120C4F8300500F042F87C
:10A6600040F20120C4F850060220C4F80002144948
:10A670004FF04060086013490020134D08861031E8
:10A68000C86181F82C002870012008F049FE1020D4
:10A69000C4F804034FF0E0210220C1F8000168680B
:10A6A000002802D0BDE87040004770BD0010004097
:10A6B0003C170040960000802C0000898C1500405B
:10A6C00004F50140FC250020BC020020014948752A
:10A6D000704700000C260020014951F82000704707
:10A6E000CCAF0000084910B508750849012806D00C
:10A6F000022806D040F686513E20F8F7B3FF03202B
:10A7000000E00420086010BD0C2600201015004059
:10A710000549C1F80405054810F82C1F41F0010156
:10A72000017000F04DBA0000001000400C2600201F
:10A73000014951F820007047D8AF00002DE9F047DB
:10A74000304E314C8846070015464FF0010906D0BF
:10A75000012F12D040F62D013E20F8F783FF10465E
:10A7600000F0E8FB294884F8099030F815104046BD
:10A7700000F08EFB054630460CE0104600F0C0FBB2
:10A780000220607249F6BA71404600F081FB05462E
:10A790001C48001D00F03AFBDFF87480C8F84055F3
:10A7A000DFF874A01B48CAF810051020C6F804038F
:10A7B000A06A4FF4002640F40020A062174806600B
:10A7C00000F038FA4146C8F84C9011480C30D0F8E7
:10A7D0004005A84210D30020C1F84005CAF814056E
:10A7E000A06A20F40020A0620C48001D0660FFF75C
:10A7F00023FD0020BDE8F0872946384600F012FB13
:10A800000120F7E7001000400C26002078AF000080
:10A81000008000404081004098F0014004F5014074
:10A820000D4B10B5D8719A7251B1022018720128DF
:10A8300008D002280FD040F663213E20F8F712FF1F
:10A840000120F3E7587A022805D100F07DF9BDE830
:10A85000104000F0B1BA10BD0C26002002490020C3
:10A86000C1F8400570470000008000400449D1F85D
:10A87000481501F07F014942017001207047000036
:10A88000001000400349020EC1F824250002C1F85F
:10A890001C057047001000400149C1F83C05704795
:10A8A0000010004010B50022012906D0022902D074
:10A8B00040F2D92114E04FF080720B490A430B4952
:10A8C0000A600B4908430949091D08600948D0F886
:10A8D0005005C0B2032801D00B2804D140F2F12169
:10A8E0003E20F8F7BFFE10BD08011000141500400F
:10A8F0000000030200100040014988757047000005
:10A900000C2600202DE9F04753484FF0010AC0F80B
:10A910004CA051480C30D0F8407508F097FE4F4CD1
:10A92000C4E90C0700F01AF94D49A06A0860DFF885
:10A9300034810020A062D8F8002240F21D139A430F
:10A94000C8F8002284F82C0000F088F90546424837
:10A950000830D0F84005404EE061361DD6F840057D
:10A96000A06194F82100217D84F82010617A84F898
:10A970002110A14600243946284600F0E3F910B919
:10A98000C8F810A00124354FE807A7F1100702D03E
:10A990003868804734E0A80729D5680721D408F033
:10A9A0007BFFF0B908F068FFD8B92F480068C0F302
:10A9B0004252C0F3006100F00F0CC0F30313C0F368
:10A9C000032871B1BCF1000F03D013B1B8F1000F2F
:10A9D00007D1C0F30440012803D1032A01D245F076
:10A9E000040545F380002146401C7A6807E015F015
:10A9F000280F05D045F34011BA682046491C9047FE
:10AA0000E80601D5F868804799F8091048460229F8
:10AA100020D1017B00291DD0022904D0012909D0B1
:10AA200040F666410DE0C169D9F810000844C6F847
:10AA300040050BE00169D9F81C00814204D840F6BA
:10AA400067413E20F8F70EFEC6F84015BDE8F04716
:10AA500000F0BCB9BDE8F087008000400C26002063
:10AA600008F50140001000405014004070B5164B2E
:10AA70008C8803EB8005C5F820460C78D1F80110CE
:10AA800044EA0121C5F80016D3F840160124844099
:10AA9000C9B2E5B2294332B1012A0AD040F2D451F9
:10AAA0003E20F8F7DFFDD3F84006C0F30720A043AF
:10AAB00004E0D3F84006C0F30720284341EA002011
:10AAC000C3F8400670BD000000100040014901209D
:10AAD00008707047BC0200200B48817D0B48405C29
:10AAE00000F51660B0F5166F04D2A0F6381040F4E9
:10AAF000807001E0A0F51660054AC2F8080501F073
:10AB00007F00C2F8540570470C2600207EAF00007D
:10AB10000010004008B50B496B4691F91520897D5E
:10AB200000F0D0FA9DF9000000F0A0FA0DF101004C
:10AB300004F05CFA002804D040F215613E20F8F7DA
:10AB400091FD08BD0C2600200348017A012902D19D
:10AB5000807AFFF7DFBF70470C2600200D4810B544
:10AB6000407A01280CD0022813D104F021FA0028E1
:10AB70000FD0401C0DD040F6C1013E20F8F772FD09
:10AB800004F028FA002804D0401C02D040F6BB0193
:10AB9000F3E710BD0C26002008480021C0F8001182
:10ABA000C0F80C11C0F81011C0F80411C0F814114D
:10ABB000C0F81811C0F808117047000000100040DC
:10ABC000184810B590F82C00C10729D0810714D57A
:10ABD0001548D0F8001241F00101C0F80012D0F879
:10ABE0005005C0B20B2805D00A2803D0032801D095
:10ABF000022815D140F23E610FE0400710D50A4807
:10AC00000A490830C1F814054FF4A071084808F04B
:10AC1000AAFB002804D040F246613E20F8F722FD4E
:10AC200010BD00000C2600200010004098F00140EC
:10AC30000080004008480146C27991F82C1012B1FA
:10AC4000012A03D006E041F0020101E041F00401D5
:10AC500080F82C10FFF7B4BF0C2600202DE9F0413E
:10AC6000344D0024287B38B14FF4A271324808F0EB
:10AC70007AFB08B1012600E00026687A2F4F4FF4D6
:10AC80008671012802D0022806D016E0384608F066
:10AC900065FB90B1082410E0384608F05FFB00B176
:10ACA0000224D7F80004C04340F30000401C01D147
:10ACB00044F004040EB144F0010414F00B0F07D16A
:10ACC0004FF48871384608F049FB08B144F010048D
:10ACD0001B480078F8B1D7F8400610F0FF0607D0FF
:10ACE0004FF48A71384608F039FB08B1012000E0C2
:10ACF000002085F822003EB14FF48C71384608F0F0
:10AD00002DFB08B1012000E0002085F82300D7F8D2
:10AD1000100485F82400FFF73FFFE00606D5200762
:10AD200004D4687A012801D144F020042046BDE80B
:10AD3000F08100000C260020008000400010004040
:10AD4000BC0200202DE9F0411A4C0D46217A29B1B0
:10AD500010F0110F07D0FFF76FFA24E000F090F821
:10AD6000002020731FE0012901D0012600E0002609
:10AD7000E07901280ED0002700F082F896213046B5
:10AD800000F094F801464FB13B358D4204D90020C4
:10AD9000BDE8F0810127EFE70120E071A27A30469B
:10ADA000FFF7CCFC08B10120F2E740F6C4213E20B9
:10ADB000F8F758FC0C2600200348D0F8001241F4A4
:10ADC0008871C0F800127047001000400448816A82
:10ADD00041F48001816203494FF4800008607047AC
:10ADE0000C26002004F50140074A002008320649DD
:10ADF000C2F840050A1DC2F84005C1F840050249E5
:10AE00000C31C1F840057047008000400349C97902
:10AE1000002902D10249C1F8140570470C26002010
:10AE200098F0014010B5144A20B1012811D040F229
:10AE300069711CE001F12800C2E902100F490E48B7
:10AE400004F0CEF8002815D0401C13D04FF4EB616D
:10AE50000DE001F12900C2E902100849064804F09A
:10AE6000ADF8002806D0401C04D040F265713E20A9
:10AE7000F8F7F8FB10BD0000C4020020A8AF0000E6
:10AE800002480021C1710172417270470C260020F6
:10AE9000054AD279012A06D04FF47A7201F5FA7187
:10AEA000B1FBF2F1401A70470C26002070B5134C2C
:10AEB00003460D4694F8212000205AB1214691F80E
:10AEC000201063B1012B11D1012A284612D008F0BD
:10AED0004FFA09E040F66E013E20F8F7C3FB012A65
:10AEE000284604D008F052FAE169084470BD00F029
:10AEF000D1F8F9E700F0C0F8F6E700000C260020D2
:10AF000010B5FFF7EFFBFFF7E7FDFFF71DFEFFF7BB
:10AF100053FF08F0C1FC002808D108F0ADFC002860
:10AF200004D10348016841F4C021016010BD000054
:10AF30006815004010B50446FFF7D4FBFFF7CCFDC1
:10AF40002046FFF7E7FD08F0A7FC00280DD0094ACE
:10AF500011685006022CD0F8200307D0C0F3062059
:10AF600021F4FE4141EA0020106010BDC0F30660EC
:10AF7000F6E700008815004000002CA6E0A10406BA
:10AF8000080A0C0E10121416181C1E202224262843
:10AF90002A2C2E30323436383A3C3E404244464821
:10AFA0004A4C4E021A5000000100000010110040EF
:10AFB0000000000000000000000000000000000091
:10AFC00000000000141E000030110000000000000E
:10AFD000280000001800000000000000141E0000FF
:10AFE000301100000000000070170000A00F0000EA
:10AFF00070B5054614460846FFF79AFB05EB450178
:10B00000C1EBC511C0EBC101074850F8240008444A
:10B010004FF47A7100F6B730B0FBF1F52046FFF738
:10B020005BFB2844401D70BDB8B0000070B50E4DEC
:10B030001C46083D0C4B35F8111000EB400553F849
:10B040002230C5EBC01001EBC00003F6B733184443
:10B050004FF47A71B0FBF1F51046FFF73DFB284441
:10B060002044401D70BD0000B8B000000149C0B2CE
:10B07000086070470C150040054A32F811104FF473
:10B080007A7201F2E731B1FBF2F10844801E704799
:10B09000B0B00000054A32F811104FF47A7201F591
:10B0A0007A71B1FBF2F1084470470000B0B00000C3
:10B0B0000000DC05E803000000000000141E000092
:10B0C000301100002DE9F8431E4617460C46054690
:10B0D00000F056F8DFF8A490804699F80000A842E6
:10B0E00010D199F801104846A1420BD190F90210F5
:10B0F000B94207D1C278424504D181883180807934
:10B10000B07037E03A462146012D09D0022D09D012
:10B11000042D09D0082D09D040F2624106200CE030
:10B12000002004E0012002E0032000E002206B4642
:10B1300000F09EF818B13D217520F8F793FA2046EB
:10B14000FFF772F80246002331469DF9000003F034
:10B1500059FF014689F807103188A9F80410B17821
:10B1600089F8061089F8005089F8014089F80270C2
:10B1700089F8038099F90700BDE8F8837C03002073
:10B180000148007870470000DC02002070B5174CC1
:10B190006078002823D10120607008F057FB6FF021
:10B1A000270528B908F088FB10B908F08FFB20B1FB
:10B1B0000F486060A570082010E008F01CFB40B943
:10B1C00008F023FB28B908F037FB10B908F048FB5A
:10B1D00030B1074831306060A5700420E07070BD68
:10B1E00040F23F11742003F04DFD0000DC0200200E
:10B1F000ED3B0100064A00B592F90320904201DBC5
:10B20000104600BD00F008F80249085600BD0000D5
:10B21000DC020020DF3B01000246134810B590F924
:10B2200003309A4201DB0D2010BD90F902309A42A2
:10B2300001DC002010BD01B10121D41A4368185D62
:10B240000A4C24569442F5D0084C08443F34C0B20E
:10B25000D2B2A342EED10029ECD0012A01D0022AB9
:10B26000E8D1401CC0B210BDDC020020DF3B010071
:10B270002DE9F0411C4690460D4606466FF0150735
:10B28000042804D81CB108F08CF8A84202D838462B
:10B29000BDE8F0810548424650F8260018B14057F5
:10B2A000824200DD024622700020F1E744260020A1
:10B2B00070B50D4604000CD094F8286000210220DF
:10B2C000092D6ED2DFE805F008113636667189A6C1
:10B2D00094004FF4CB71F7E094F8260004287BD05B
:10B2E0000328FCD040F2A111EEE094F826000428D7
:10B2F00004D0032802D040F2A511E5E0052084F82F
:10B30000260084F8291094F82400B8BB00212046B8
:10B3100008F0A8F82078012807D0D4E9040100BF7C
:10B32000C4E906010021226A48E094F8270001F0F0
:10B33000C5FAF5E794F82610042904D0032902D0B1
:10B3400040F2C311C0E094F8242022B121463046D7
:10B3500008F0C8F8B0E0042900D0012084F82600E5
:10B36000226A022D0BD006213046904700286DD06E
:10B37000007800286AD040F2DD11A5E034E0052114
:10B3800030469047002870D0007800286DD04FF4E8
:10B39000EC7199E094F82600052803D04FF4F2717F
:10B3A00092E080E00221226A08E094F82600052855
:10B3B00002D04FF4F57187E0226A012130469047B0
:10B3C0000146204607F0F9FF022875D0E8B30128AE
:10B3D0006CD040F22A2177E070E094F8260005282E
:10B3E00002D04FF4F8716FE0BDE8704000F09EB8F5
:10B3F00094F82600052802D040F2F51164E0226A94
:10B400000A21304690470146204607F0D6FF4FF408
:10B41000FC7159E094F82620052A07D094F82530CD
:10B420000BB1032A02D04FF4FE714DE094F82420B2
:10B430002AB121463046BDE8704008F053B894F870
:10B4400029209AB184F8291001E032E034E084F830
:10B450002600226A082130469047002837D000781D
:10B46000002834D04FF402712EE030E094F825200B
:10B470005AB184F8251094F82700214607F0F0FF10
:10B48000002824D140F20D211EE084F82600226A13
:10B49000072130469047002819D00078002816D0A0
:10B4A0004FF4057110E040F219210DE00421226AE9
:10B4B00084E70321226A81E7002D08D108F0C8F84B
:10B4C000002804D040F233216A2003F0DBFB70BD7A
:10B4D000002819D003781349134A13B1012B0ED059
:10B4E00011E00379012B00D06BB943790BB1012B2B
:10B4F00009D18368643B8B4205D2C0680EE00379B2
:10B50000012B02D00BB10020704743790BB1012B06
:10B51000F9D1C368643B8B42F5D280689042F2D87F
:10B52000012070473D860100FF3F420F10B5054CDA
:10B53000206810B1804700202060BDE8104002F074
:10B540007FB80000E40200202DE9F0410E4605001E
:10B5500004D000F047F8074600240BE06FF0150018
:10B56000BDE8F081204600F043F890F8260030B1A5
:10B57000641CE4B2BC42F5D36FF00B00F0E7274641
:10B58000FF2CF9D0204600F033F8044607F0C5FF41
:10B5900084F828702146084802F02AF884F8270029
:10B5A000202806D00120256284F82600377000206C
:10B5B000D6E76FF02200D3E7B1B2000010B58207E2
:10B5C00002D06FF00D0010BD054A1170506028B117
:10B5D00001EB41010A01002108F047FA002010BDEB
:10B5E000E80200200148007870470000E8020020CF
:10B5F00005490A78904201D300207047496800EB62
:10B60000400001EB00107047E80200200E4910B521
:10B6100091F83200202812D091F83200A1F5806212
:10B62000C0EBC00002EB800091F832104068C1EB23
:10B63000C10152F82120BDE810400421104740F616
:10B64000BC01702003F01EFB582A002070B505468F
:10B65000202A28D019481A4C00EB831C03EB430323
:10B660000CEB42002344202922D00CEB410140780E
:10B670004C784870204601460CEB41009142057021
:10B680004078F8D193F82220202A1ABF0CEB42020E
:10B69000547083F8214020220CEB410C8CF80120DF
:10B6A00083F8221070BD4FF42671702003F0EAFA7F
:10B6B00093F82040407883F82000DBE7D829002069
:10B6C000582A00202DE9FF4F8DB015460C4602F098
:10B6D00003FA284420F07F4008902168081A0002ED
:10B6E000C11700EB11600012002800F3F080DDF8B4
:10B6F0004080CD4808EB48010844099090F820505C
:10B700002020CA4E0DF1180A0DF11C098DF8180001
:10B71000202D1CBFC64800EB881B38D0C5EBC500E8
:10B7200006EB800000F10801C0682768381A0002A3
:10B73000C21700EB1260001229D4E08900B3C88957
:10B74000F0B90868039003F0DFF8B0F5C67F08BFD2
:10B750000D200BD0A0F54070563808BF1C2005D036
:10B76000A0F500709F3814BF00203220411C0398C0
:10B77000381A0002C21700EB12600012884206DB82
:10B780000BEB45008AF800504578202DC6D19AF879
:10B79000000089F80000202D1CBFA54800EB881B85
:10B7A00000F03E81C5EBC50006EB80076168D7F865
:10B7B000088007F10800A8EB01010902CA1701EB94
:10B7C0001261091227D4C089002800F02981E0897C
:10B7D000002840F02581D4F800A003F095F8B0F5DA
:10B7E000C67F08BF0D200BD0A0F54070563808BFAB
:10B7F0001C2005D0A0F500709F3814BF0020322017
:10B80000411CA8EB0A000002C21700EB12600012F4
:10B81000884280F2058189F80050387E217C884278
:10B8200006D90BEB45004578202DBBD100F0F8B8C8
:10B830009DF81C00C0EBC00006EB8000C18AC56803
:10B84000E1BBE189D1B3876803F05EF8B0F5C67F4C
:10B8500008BF0D200BD0A0F54070563808BF1C2043
:10B8600005D0A0F500709F3814BF00203220411C85
:10B87000E81B0002C21700EB1260001288421DDABA
:10B8800003F042F8B0F5C67F08BF0D200BD0A0F53D
:10B890004070563808BF1C2005D0A0F500709F38B6
:10B8A00014BF002032209DF81C10401CC1EBC101C8
:10B8B00006EB81018968084420F07F450898281A22
:10B8C0000002C11700EB11600012002803DD11B067
:10B8D0000020BDE8F08F2068A84202D9A168491C69
:10B8E000A16061680DF1180A081A284425F07F410B
:10B8F00020F07F40C4E9001010980B9009980DF1DA
:10B900001C0890F8205020208DF81800202D3CD0E5
:10B9100047490B9801EB801BC5EBC50006EB800087
:10B9200000F10801C0682768381A0002C21700EB4E
:10B930001260001229D4E08900B3C889F0B9D1F8A7
:10B94000009002F0E1FFB0F5C67F08BF0D200BD0DC
:10B95000A0F54070563808BF1C2005D0A0F5007037
:10B960009F3814BF00203220411CA7EB09000002C1
:10B97000C21700EB12600012884206DB0BEB450099
:10B980008AF800504578202DC6D19AF8000088F832
:10B9900000000B98202D1CBF254901EB801B3FD0D8
:10B9A000C5EBC50006EB80076068D7F8089007F183
:10B9B0000801A9EB00000002C21700EB12600012A0
:10B9C00022D4C88960B3E08950BBD4F800A002F04B
:10B9D0009BFFB0F5C67F08BF0D200BD0A0F54070CF
:10B9E000563808BF1C2005D0A0F500709F3814BF42
:10B9F00000203220411CA9EB0A000002C21700EB14
:10BA00001260001288420BDA88F80050387E217CE0
:10BA100088427FF60DAF0BEB45004578202DBFD156
:10BA200011B00120BDE8F08F582A002058260020D0
:10BA3000D82900202DE9F84F0F46064601EB4700B4
:10BA40004B4999460844924690F8204020201070B7
:10BA5000A1F58068202C1CBF464800EB871B38D01E
:10BA6000C4EBC40008EB800000F10801C068356831
:10BA7000281A0002C21700EB1260001229D4F089C4
:10BA800000B3C889F0B90868009002F03DFFB0F536
:10BA9000C67F08BF0D200BD0A0F54070563808BFF8
:10BAA0001C2005D0A0F500709F3814BF0020322064
:10BAB000411C0098281A0002C21700EB1260001205
:10BAC000884206DB0BEB44008AF800404478202CC7
:10BAD000C6D19AF8000089F80000202C1CBF254828
:10BAE00000EB871A40D000BFC4EBC40008EB80070E
:10BAF0007068BD6807F10801281A0002C21700EB40
:10BB00001260001222D4C88970B3F08960BBD6F8E5
:10BB100000B002F0F9FEB0F5C67F08BF0D200BD0D3
:10BB2000A0F54070563808BF1C2005D0A0F5007065
:10BB30009F3814BF00203220411CA5EB0B000002EF
:10BB4000C21700EB1260001288420DDA89F800403B
:10BB5000387E317C884202D80020BDE8F88F0AEB9D
:10BB600044004478202CBFD10120BDE8F88F0000AC
:10BB7000582A0020D82900202DE9F74F98B0154603
:10BB800002F06CFA044602F0E7FC06461998012818
:10BB900018BF022805D040F692114FF0700003F054
:10BBA00071F8F94901200860F849896808600020A7
:10BBB0008DF846000A90401E0B90F549C5EBC50074
:10BBC00001EB800101F10800896990E80D100CAFCC
:10BBD000109187E80D1007F04DFDBDF83E809DF8EF
:10BBE0003C1002464144491CEA4B08449A4254D84E
:10BBF000E94DA94258DC6A4291425DDB591C814201
:10BC0000DCBF00F5F700A0F1F85005DD0028BCBF4F
:10BC1000A0F5F70000F1F8501490E048B8F1000FDB
:10BC2000808BADF8440014BF4FF0010A4FF0000ABA
:10BC300002F0B0FF1690BAF1000F08D0D748C06AE2
:10BC4000B0F1FF3F02BF16980028012701D04FF046
:10BC5000000702F059FEB0F5C67F08BF0D200BD0DB
:10BC6000A0F54070563808BF1C2005D0A0F5007024
:10BC70009F3814BF002032204FF00009CB461390AC
:10BC8000464536D9149BDFF80C936FEA060C6946DB
:10BC900017AA03EB0C004B4504D940F29E517020CB
:10BCA00002F0F0FFAC4504DD40F29F51702002F03D
:10BCB000E9FFBB4B9C4504DA4FF4B461702002F0FD
:10BCC000E1FFB84B8342DCBF00F5F700A0F1F8506C
:10BCD00005DD0028BCBFA0F5F70000F1F85001F029
:10BCE00017FF00980C9920F07F400090081A20F070
:10BCF0007F49002F18BFDDF84CB005D19DF84400F6
:10BD0000002818BF4FF0020BB4F1807F08D00C98C8
:10BD1000001B0002C11700EB11600012012802DABB
:10BD20000320189D0DE057B19C4890F8300030B1C9
:10BD30009DF8440010F1000B18BF4FF0020B254690
:10BD4000002083440C98A0EB090020F07F41481E9E
:10BD500020F07F40421B1202D31702EB1362121233
:10BD60005A4504DBB9F1000F18BF0C912DE0B9F171
:10BD7000000F05D09DF8450020B902F0E3FB08B1A3
:10BD8000AFB90CE02FB99DF84400002818BFABF103
:10BD9000020B4FF000098DF844904E4607E09DF8E5
:10BDA000440020B100208DF84400ABF1020B0C9848
:10BDB000A0EB0901481E20F07F40421B1202D3175E
:10BDC00002EB136212125A457EDB744AD26A891A58
:10BDD0000902CB1701EB1361169B09123BB9B2F1B3
:10BDE000FF3F1CBF139A9142B8BF002100DB012125
:10BDF0003AEA010168D1199905464FF00009059109
:10BE000001F0F0FF281A0002C11700EB11604FEAA1
:10BE1000202B02F079FDB0F5C67F08BF0D200BD0B6
:10BE2000A0F54070563808BF1C2005D0A0F5007062
:10BE30009F3814BF002032200B3058451FDD059875
:10BE4000012801D047B112E0B4F1807F1CD140F647
:10BE50001311702002F016FFB4F1807F07D0601B31
:10BE60000002C11700EB11600012042804DD2C460B
:10BE7000204601F0DDFF07E0002862DC04E02C46EC
:10BE8000204601F0D5FFD146B4F1807F54D00C9804
:10BE90000D9A001B121B20F07F4022F07F420128E8
:10BEA0004FD3B0F5000F98BFB2F5000F49D8204628
:10BEB00007F0E0FB1499384A0D1A4FF0000BAA1A4C
:10BEC0007BF1000218D300E03BE0334B421AD31A57
:10BED0007BF1000310D32F4BAB423EBFC0F5902047
:10BEE00000F1F450451807D393422ED2C1F59021AA
:10BEF00001F1F45108444542284FB87F50B31998D6
:10BF0000012805D0022002F0E3F9012002F0E0F957
:10BF1000B0452BD2A5EB06014FF0020002F022F94A
:10BF200088B3B8F1000F1CBFA5EB0801012043D076
:10BF300002F018F938B33FE040F63121702002F0EA
:10BF4000A1FE1BB00020BDE8F08F40F60531702047
:10BF500002F098FEB04534BF304640461E30A8423D
:10BF6000CDDB40F64521702002F08CFE1CD9A5EBFC
:10BF70000801012002F0F6F828B1002E1CBFA91B11
:10BF8000022019D0D4E742E008050040F00200206A
:10BF900058260020FF7F841E0040420F582A0020B0
:10BFA00000C0BDF00080841E56EA080004D040F6B0
:10BFB0007611702002F066FE2946002002F0D2F8C9
:10BFC00028B30126BAF1000F04BF97F8300000280B
:10BFD00002D0B9F1000F24D0F86AB0F1FF3F04D0CD
:10BFE00002F098FC4FF0FF30F862B9F1000F1CD05E
:10BFF0001398201A20F07F41052002F0B3F860B3B7
:10C0000097F83000002808BF87F8306015E002205C
:10C0100002F05EF9012002F05BF91BB00020BDE8E0
:10C02000F08FF86AB0F1FF3F12D097F8300020B1DE
:10C03000052002F04DF987F830B0A5EB0800A0F11B
:10C04000190100290EDC40F66E21702002F01AFE64
:10C0500002F07CFC01F0C6FEC6E74FF43E71702092
:10C0600002F010FE032002F07DF8B8B10E4880689F
:10C07000C0F800B00D48C0F800B00DF1280898E8ED
:10C080007F1038607960BA60FB603C617D61BE61A1
:10C09000C7F81CC01BB00120BDE8F08F40F6762128
:10C0A000702002F0EFFD0000F002002008050040C3
:10C0B0002DE9FF4F0D46144606464FF0000A2A8927
:10C0C0004168504662F31F40AA7AD14662F30709DD
:10C0D000EA7A83B062F30F292A78C4F800A062F3E9
:10C0E0001749C4F804A0C4F81090C4E902109D4F89
:10C0F0007068A0FB0789306807F0BCFA10EB0801F4
:10C100004AEB090228784FEA6709C9F1000B70B1C0
:10C11000E08994F81180C043D5F804A004F10C0222
:10C1200048457CDD40F29F51702002F0ABFDDFF806
:10C1300038C2D5E9040311EB0C0A42F1000CB0EB54
:10C140000A0A73EB0C0C72D2411A73EB02016ED324
:10C15000B0EB0806B7422BD8E089A6F1F458A8F551
:10C160009028C143814A08EB010042452BD3494541
:10C17000D8DC594566DB8742DCBF00F5F700A0F14B
:10C18000F85005DD0028BCBFA0F5F70000F1F8501D
:10C190006A4601A901F0BCFCE0899DF80010301A44
:10C1A000401A401EB84202D3A068401CA060464618
:10C1B000E0896E4BC1436D6894F81180701804F1EA
:10C1C0000C029E4204D940F29E51702002F05AFDAA
:10C1D0004945A7DC594535DB8742DCBF00F5F70050
:10C1E000A0F1F85005DD0028BCBFA0F5F70000F174
:10C1F000F850214601F08CFC206820F07F41701936
:10C20000401C2160B8F1000F08BF7A3004D0B8F1AB
:10C21000010F08BF48303AD101F05EFC01E00EE0AA
:10C2200005E020F07F40606007B0BDE8F08F306827
:10C23000401E20F07F40206000F57A70F3E7014651
:10C24000584504DA4FF4B461702002F01BFD8742B8
:10C25000DCBFA1F1F450A0F5902005DD0028BCBFA3
:10C2600001F1F45000F59020214601F051FC2068C6
:10C27000B8F1000F20F07F410AF10100216008BFF2
:10C280007A3009D0B8F1010F08BF483004D040F22D
:10C290003961702002F0F6FC01F01EFC20F07F41B5
:10C2A0006160B4F80E9001AA69464846376801F00B
:10C2B0002FFC02F051F901F00FFC80462C4890F859
:10C2C000321020292AD0C068401D20F07F4000BFD6
:10C2D000D4E90021891A014421F07F41C4E9000119
:10C2E0003168814202D9A068401CA0603268286988
:10C2F0002146069BFFF7E6F900281CBF07B0BDE802
:10C30000F08FD4E90010401A316821603168084488
:10C3100020F07F40606007B0BDE8F08F0937B9F1C9
:10C32000000F16D002F036FC98B902F0EDFAB0F525
:10C33000C67F08BF0D200BD0A0F54070563808BF4F
:10C340001C2005D0A0F500709F3814BF00203220BB
:10C3500007440098804584BFA8EB0000074427F0FD
:10C360007F40B5E70080841E0040420FFF7F841E9F
:10C37000582A002070B51E4D95F83200202818BFAD
:10C3800070BD95F8312002EB4200284490F820401F
:10C39000202C27D0174B03EB821101EB4401497885
:10C3A00080F82010FF2085F8290085F832402146CA
:10C3B000022000F091F8002085F82800A8770E49A7
:10C3C000C4EBC40001EB8000007E002808BF02F02F
:10C3D000C3FD002009494968002908BF70BDBDE8B8
:10C3E0007040084740F23231702002F04BFC0000F0
:10C3F000582A0020D829002058260020F0020020CA
:10C400002DE9F05FDFF8C08098F8315005EB45006A
:10C41000404490F82140202C08BFBDE8F09FDFF891
:10C42000ACB0DFF8ACA0AAF560790AEB8517072657
:10C4300017F8140001280ED0042808BF02260AD0DD
:10C4400005280CBF0326062805D040F6DD014FF075
:10C45000700002F017FCBBF1000F18BFAFF30080B3
:10C46000EFF3108072B607EB44014A7805EB450103
:10C47000414481F8212091F82220A24204BF2022C9
:10C4800081F82220C0B12A462146012000F024F87C
:10C49000C4EBC40109EB810059F821204068314602
:10C4A000904798F8315005EB4500404490F8214002
:10C4B000202CBAD1BDE8F09F0648002818BFAFF382
:10C4C000008062B6DFE70000582A0020000000006C
:10C4D000D829002000000000DFF858C010B5002364
:10C4E0000CEB821C07281FD2DFE800F005050505CC
:10C4F0000404040001230CF81100002B08BF10BD38
:10C5000002EB42020C48024492F8220020280EBF9F
:10C5100082F821100CEB4000417020200CEB41030D
:10C52000587082F8221010BD40F26E21702002F087
:10C53000A9FB0000D8290020582A00202DE9F05F2F
:10C540000F468046DFF860A101EB47005044B8F188
:10C55000010F90F82040254618BFB8F1020F05D012
:10C5600040F6AC214FF0700002F08CFB4FF0000B56
:10C57000202D42D09AF81E000026002808BF02266F
:10C5800001F030FCDFF824C1C4EBC4010CEB8101E5
:10C590008A68C968121A091A22F07F4221F07F4185
:10C5A000964299BFB2F5000FB1F5000F404A02EB79
:10C5B000871920D9224609EB42014C78202C12D051
:10C5C000C4EBC4010CEB81018B68C9681B1A091A02
:10C5D00023F07F4321F07F419E429CBFB3F5000FC3
:10C5E000B1F5000FE6D8202A05D03B4620210420D3
:10C5F000FFF72CF80446AC4216D12E48002818BF8D
:10C60000AFF3008001F0EEFB03469AF833002028D8
:10C610000DD0DAF80800991C081A0002C11700EBC7
:10C6200011600012002802DD0020BDE8F09F202DDF
:10C6300014D02A4641461846FFF79EFA00281EBF2E
:10C640008AF833500220BDE8F09F3B462A4620215D
:10C650000420FEF7FBFF0020BDE8F09FDAF82C0075
:10C66000B0F1FF3F05D002F055F94FF0FF30CAF8A6
:10C670002C009AF8300020B1052001F029FE8AF83C
:10C6800030B0042001F024FE01F092FE20208AF850
:10C69000330009488068C0F800B00848C0F800B00E
:10C6A0000120BDE8F09F0000582A002058260020F5
:10C6B000D829002000000000F002002008050040FA
:10C6C000064910B591F83220202A1CBF887710BD8A
:10C6D00040F29A31702002F0D5FA0000582A00206A
:10C6E0002DE9F04F694E07468DB096F83200884626
:10C6F000202855D096F8320006F10804C0EBC0009F
:10C70000A6F5806909EB800A20208DF8200096F8B4
:10C7100031000AAA00EB4000304409A990F82050EB
:10C72000F06802903068384401F0F2F9DAF80C0051
:10C730000999652F084438D3554A0021D21B71EB63
:10C74000010232D32268821A22F07F42B2F5000F32
:10C750002BD820F07F406060304684F8108090F83D
:10C7600031000DF1200A202D1CBF4A4901EB801B2E
:10C7700050D000BFC5EBC50009EB80086168D8F850
:10C78000086008F10800711A0902CA1701EB12616A
:10C7900009122DD4C08900283CD0E08948B139E085
:10C7A00040F67331702002F06DFA0DB00120BDE843
:10C7B000F08F20680C9002F0A7F8B0F5C67F08BF94
:10C7C0000D200BD0A0F54070563808BF1C2005D0B6
:10C7D000A0F500709F3814BF00203220411C0C9837
:10C7E000301A0002C21700EB12600012884211DA00
:10C7F0008AF8005098F81810207C814205D80298D9
:10C8000060600DB00220BDE8F08F0BEB450045786D
:10C81000202DAFD1052001F05BFD1C4C4FF0FF3007
:10C82000606094F831309DF820202021202A03D028
:10C830000520FEF70BFF04E003EB4300204490F8D3
:10C84000200094F83120134901EB821194F8322032
:10C8500001EB42014870206838442060FF2084F8D2
:10C860002900607E012805D1E068401E20F07F404D
:10C8700001F092FB9DF82000202803D00648407864
:10C8800002F0D4FA0DB00020BDE8F08F582A002045
:10C890000040420FD8290020F0020020064810B5C1
:10C8A00090F8321020291CBF007E10BD40F66D317B
:10C8B000702002F0E7F90000582A002070B5C0EBA4
:10C8C000C001094800EB810408492069A0FB01561A
:10C8D000A06806F0CFFEE18A227D401C1144084486
:10C8E000401946F1000170BD582600200080841ECA
:10C8F000F8B56F4D012605F580646E4AE16A082897
:10C9000072D2DFE800F004779FB1CF44B6BBB1F13B
:10C91000FF3F04D102F01AF801F064FAE062E08A05
:10C9200010B102F037F980B1FFF724FDFF2084F841
:10C9300027006168B1F1FF3F03D0052001F012FC30
:10C9400040B1607E012810D109E040F669017020F5
:10C9500002F098F940F66E01702002F093F9E06859
:10C96000401E20F07F4001F017FB94F8320094F84D
:10C970003210C0EBC00005EB80004068C1EBC10184
:10C9800055F8212001B00121BDE8F040104794F88E
:10C99000300058B1B1F1FF3F04D101F0D7FF01F0F1
:10C9A00021FAE062002084F83000F8BDFFF7E2FCD5
:10C9B0004FF0FF30606094F827008DF800009DF87C
:10C9C000000090B194F8320094F83210C0EBC0002F
:10C9D00005EB80004068C1EBC10155F8212001B092
:10C9E0000621BDE8F04010475CE040F6850170206C
:10C9F00002F048F9FFF7BEFC84F8266002F0CAF89E
:10CA000020B1E06AB0F1FF3F05D009E040F69301A4
:10CA1000702002F037F901F099FF01F0E3F9E062CC
:10CA200094F8320094F83210C0EBC00005EB80009F
:10CA30004068C1EBC10155F8212001B00021BDE8DB
:10CA4000F040104701F06AFDE08A10B102F0A2F850
:10CA500028B101F077FD002818BF6677F8BD40F6D1
:10CA60009D01702002F00EF9134806609068066080
:10CA7000F8BD1078BDE8F84002F0D8B9FFF77AFCAD
:10CA800094F8320094F83210C0EBC00005EB80003F
:10CA90004068C1EBC10155F8212001B00521BDE876
:10CAA000F04010474FF40B61702002F0EBF80000EB
:10CAB00058260020F0020020080500402DE9F34F21
:10CAC0008246ED488DB00068EC4DC005C00D0ED01B
:10CAD000103840B20028B8BF00F00F0000F1E0208D
:10CAE000ACBF90F8000490F8140D40090DD00E98DA
:10CAF0004FF0000B0078002818BF012818D040F232
:10CB00003B714FF0700002F0BDF895F832004FF025
:10CB1000010B202807D00E98007848B140F23771F9
:10CB2000702002F0AFF840F23471702002F0AAF8E1
:10CB3000D34C24B1002140F23E70AFF300800020BE
:10CB4000CDE90A00CF49CAEBCA0001EB80004FF0E3
:10CB50000109009024B1002140F24970AFF3008038
:10CB6000B9F1000F0AD000BF95F831604FF000080E
:10CB700085F82980BBF1000F07D038E0C2480028B3
:10CB800018BFAFF3008062B6EEE73746012020EA17
:10CB90000706BE48402200EB871100EB861006F026
:10CBA000EAFE24B1002140F25E50AFF3008007EBB3
:10CBB000470106EB4600294428440A8C028491F878
:10CBC000221080F8221024B1002140F26250AFF30D
:10CBD000008024B1002140F25370AFF3008095F83B
:10CBE00029008DF818009DF818000028B2D124B152
:10CBF000002140F25D70AFF3008006A801F0F8F864
:10CC0000DDE90601CDE90801334601AA08A80E991D
:10CC1000FFF74EFA24B1002140F26470AFF30080B8
:10CC20009A4A089902EB861701A817F81A20012AD8
:10CC300018BF022A38D1CDF82C80019A029BA2EBB2
:10CC4000010222F07F42A3EB010121F07F41022A81
:10CC500060D3B2F5000F98BFB1F5000F5AD84FF06E
:10CC6000010807AB06AA3146FEF7E4FE002859D0BA
:10CC70009DF818109DF81C2033468A4256D0052096
:10CC8000FEF7E4FC07EB4A0148709DF818002028E5
:10CC90001CBF07EB400080F801A053D0324651463C
:10CCA0005FF00300FFF718FC24B1002140F2697027
:10CCB000AFF300807648002818BFAFF30080EFF391
:10CCC000108972B624B1002140F26F70AFF300807A
:10CCD00095F829008DF818009DF8180000287FF4B9
:10CCE00039AF24B1002140F27770AFF300809DE8A6
:10CCF0008F1000F10800B8F1000F80E88E1051D0BD
:10CD000024B1002140F28470AFF30080BBF1000F2A
:10CD100039D11FE0324651460420FFF7DDFB4FF0CA
:10CD20000108C1E7324651460420BBE7202919BF5C
:10CD300007EB4100407806EB4600284408BF90F816
:10CD400020009FE706EB4601294481F820A0CDF89A
:10CD50002C80A3E70B9810F0FF0F14D095F8320049
:10CD6000202810D124B1002140F28970AFF3008057
:10CD700031460220FFF7E2FB0A9020B90E980078B6
:10CD8000E8B101282AD024B1002140F2A670AFF307
:10CD90000080FF20BBF1000F18BF85F8290026D0C6
:10CDA0004FF0010824B1002140F2B770AFF30080CA
:10CDB0000A98384E022823D0012829D02DE024B12A
:10CDC000002140F29170AFF3008095F83120514678
:10CDD0000420FFF781FB4FF00108E3E7002C3FF44C
:10CDE000B9AE002140F29C70AFF30080B2E695F836
:10CDF00031200121914385F8311085F82900CFE7D2
:10CE0000A8680899401A06F035FC716821B904E059
:10CE100071684FF0FF3001B18847B9F1000F24D09D
:10CE200024B1002140F2C770AFF30080B8F1000FC9
:10CE300011D095F8310000EB4000284490F8210013
:10CE4000202808D024B1002140F2CE70AFF300803A
:10CE5000707801F0EBFF24B1002140F2D370AFF302
:10CE600000800FB04046BDE8F08F0748002818BF8B
:10CE7000AFF3008062B6D3E704ED00E0582A00204B
:10CE8000000000005826002000000000D8290020E3
:10CE900000000000F00200202DE9F04F0646007867
:10CEA0008DB018B10DB00020BDE8F08F8C4800683F
:10CEB000C005C00D0ED0103840B20028B8BF00F039
:10CEC0000F0000F1E020ACBF90F8000490F8140DC2
:10CED0004009E7D0834D844C4FF0010B002725B16A
:10CEE000002140F2E550AFF3008094F831A084F8BF
:10CEF00029704FF0000925B1002140F2EA50AFF34C
:10CF000000807A482BEA0A0800EB8A1100EB8810AF
:10CF1000402206F030FD25B1002140F25E50AFF313
:10CF200000800AEB4A0108EB4800214420440A8CA7
:10CF3000028491F8221080F8221025B1002140F2DD
:10CF40006250AFF3008025B1002140F2EF50AFF303
:10CF5000008008A800F04CFFDDE90801CDE90A01D6
:10CF600043466A4631460AA8FFF7A2F825B10021D8
:10CF700040F2F550AFF3008094F8320020281AD028
:10CF8000E0680099091A0902CA1701EB1261091237
:10CF900011D50099814202D90299491C0291DDE91B
:10CFA0000021891A20F07F42084420F07F40CDE91B
:10CFB00000204FF0010925B1002140F2FF50AFF3EE
:10CFC000008000990A98019A091A101A21F07F41ED
:10CFD00020F07F40B1F5000F98BFB0F5000F09D8E1
:10CFE0004346694642480A9AFEF76CFB59EA00003C
:10CFF00029D142E00B98BDF80EA0029009AA07A91A
:10D000005046DDF8288000F083FD01F0A5FA00F01D
:10D0100063FD814694F8320020283BD0E068401D33
:10D0200020F07F400099814202D90299491C029167
:10D03000DDE90021891A0090084420F07F4001902A
:10D040001F208DF80C00009806F014FB411CBDF861
:10D050000E009DF80C2010440844C6E9040725B1D1
:10D06000002140F21A60AFF30080D6E90410214A93
:10D07000029BE3FB0210C6E9041094F829008DF826
:10D0800014009DF8140000287FF429AF0DB0012092
:10D09000BDE8F08F08F10908BAF1000F16D001F0D1
:10D0A00079FD98B901F030FCB0F5C67F08BF0D20BE
:10D0B0000BD0A0F54070563808BF1C2005D0A0F555
:10D0C00000709F3814BF384632208044079881454D
:10D0D00084BFA9EB0000804428F07F40A2E7000055
:10D0E00004ED00E000000000582A0020D8290020AC
:10D0F0000040420F0080841E2DE9F14F924D8CB00C
:10D1000095F8310000200890069001208F4CA5F181
:10D1100080094FF000080746079024B1002140F233
:10D12000E470AFF30080079800283CD085F8298090
:10D1300024B1002140F2E970AFF3008095F831A0EE
:10D14000402227EA0A0609EB861009EB8A1183467A
:10D1500006F011FC24B1002140F25E50AFF30080D4
:10D1600006EB46000AEB4A012844294400900A8C49
:10D17000028491F8221080F8221024B1002140F29C
:10D180006250AFF3008095F829008DF808009DF8F3
:10D19000080078B1002C1CBF002140F2EF70BCD019
:10D1A000AFF30080B9E76A48002818BFAFF30080EA
:10D1B00062B6BBE724B1002140F2F370AFF3008008
:10D1C0000C981BF8100003287ED1009A0C9992F855
:10D1D0002000884214BF4FF0000A4FF0010A02F10C
:10D1E000200C8346202209EB861303E0024603EB62
:10D1F00042004078884202D020280AD0F6E7202852
:10D2000007D0834507D103EB4B0040788CF8000032
:10D2100007E040460CE003EB400003EB420140789E
:10D22000487024B1002140F2C940AFF30080384675
:10D23000C34610EA0A0F18BFBB4600284ED024B1DF
:10D2400000214FF4FF60AFF30080324601200C99BB
:10D25000FFF742F924B1002140F60100AFF300804E
:10D260003C48002818BFAFF30080EFF3108072B67F
:10D27000079024B1002140F60600AFF3008095F836
:10D2800029008DF808009DF8080038B1002C1CBF5B
:10D29000002140F60A003FF440AF81E7BBF1000FE8
:10D2A00009D095F83200202805D131460220FFF739
:10D2B00045F90690F8B124B1002140F61E00AFF305
:10D2C000008095F8310000E008E027EA000085F8CA
:10D2D0003100FF2085F829000120089024B10021A9
:10D2E00040F62700AFF3008006981B4E022809D0B5
:10D2F000012810D014E09CB1002140F61900AFF3D2
:10D300000080ECE700F06EFDA968081A06F0B2F99B
:10D31000716821B904E071684FF0FF3001B18847AE
:10D32000079848B124B1002140F63C00AFF30080DB
:10D3300008980DB0BDE8F08F0548002818BFAFF37E
:10D34000008062B6EEE70000582A002000000000CE
:10D350000000000000000000F0020020202824BF90
:10D3600000207047C0EBC000034B43F8201003EBD4
:10D3700080004260012070475826002010B5202808
:10D3800011D20E4991F83130A1F1800202EB831CD9
:10D390001CF810303BB191F8313002EB831212F8D7
:10D3A0001020012A01D0002010BD91F83120014643
:10D3B0000020FFF791F8012010BD0000582A00203E
:10D3C0002DE9F84F864E804696F83100A6F1800789
:10D3D00007EB801010F81800002871D096F83190F3
:10D3E000804D25B1002140F6B930AFF3008007EB46
:10D3F000891414F81800012818D0C0B204281CBFE2
:10D400000528062861D02DB14FF0000140F6C53047
:10D41000AFF3008006F064FA25B1002140F6C93070
:10D42000AFF3008014F818000128E6D1012425B1DB
:10D4300000214FF43D60AFF30080002C4BD0002062
:10D4400086F8290025B1002140F6D530AFF30080E1
:10D4500096F831B0012020EA0B0907EB8B1107EB9E
:10D460008910402206F087FA25B1002140F25E5073
:10D47000AFF3008009EB490000EB060A0BEB4B0011
:10D480003044018CAAF8201090F822008AF822007B
:10D4900025B1002140F26250AFF3008096F82900D8
:10D4A0008DF800009DF80000E0B1002D1CBF0021A8
:10D4B00040F6DB30BBD000BFAFF30080B7E7FFE73B
:10D4C0004FF43B61702001F0DDFB4A4641460120EC
:10D4D000FFF702F8A0E74448002818BFAFF3008028
:10D4E00062B6ACE725B1002140F6DF30AFF3008033
:10D4F0009AF821300AF1210140461C464FF0200BDA
:10D5000007EB89120AF1220A04E0A34602EB4B0C56
:10D510009CF80140844202D0202C2BD0F5E7202C2F
:10D5200028D0A34204D102EB43004078087005E004
:10D5300002EB440002EB4B0140784870BAF1000F57
:10D5400011D025B1002140F2C140AFF300809AF81C
:10D550000000A04207D125B1002140F2C440AFF342
:10D5600000808AF800B05DB1002140F2C940AFF3FD
:10D57000008000E025B1002140F6E330AFF30080E9
:10D580001A48002818BFAFF30080EFF3108472B67A
:10D5900096F829008DF800009DF8000038B1002DA4
:10D5A0001CBF002140F6E9303FF441AF84E786F824
:10D5B0003190FF2086F8290054B1002D08BFBDE846
:10D5C000F88F002140F6F630AFF30080BDE8F88F09
:10D5D0000548002818BFAFF3008062B6EDE70000F1
:10D5E000582A002000000000000000000000000099
:10D5F00070B50D46064601F0BBFA0F4890F8312091
:10D600000024803800EB821010F8141029B1611C3E
:10D61000CCB2202CF8D3202070BD0848C4EBC40144
:10D6200040F8216000EB8100214645600120FEF7B3
:10D6300053FF204670BD0000582A002058260020C5
:10D640002DE9F04F83B000F0CDFB054600F0B0FEB1
:10D65000844C6068B0F1FF3F1CBF4FF0FF3060604A
:10D66000A07FDFF8049290B9D4E90210401A20F0AC
:10D670007F404FF40C7101F067FAE1680844281A02
:10D680000002C11700EB11600012C00F12D0607EC3
:10D6900020B394F827008DF800009DF80000E8B151
:10D6A00000F0E2FC94F82800F0B140F2F53170206F
:10D6B00001F0E8FA94F8320094F83210C0EBC000A0
:10D6C00009EB80004068C1EBC10159F82120082115
:10D6D000904740F2DD31702001F0D4FAE81C20F0D0
:10D6E0007F4000F0A5FBDDE7012084F8280094F8D6
:10D6F0003200202821D094F83280202084F8320093
:10D7000084F83300002084F8260084F82700206085
:10D7100000F028FF207794F8316006EB46000719E7
:10D7200097F82000202858D0C0EBC00009EB8009F2
:10D7300099F81A00012805D04FE04FF47E7170204F
:10D7400001F0A0FAB9F816B001AA6946584600F0EF
:10D75000DFF900F001FF00F0BFF994F83200202853
:10D7600004D0E068401D20F07F401DE005F1090A6B
:10D77000BBF1000F16D001F00DFA98B901F0C4F812
:10D78000B0F5C67F08BF0D200BD0A0F5407056380D
:10D7900008BF1C2005D0A0F500709F3814BF0020E2
:10D7A000322082442AF07F40D9F80820811A0902E9
:10D7B000CB1701EB1361091200290EDC09F10803F4
:10D7C000824202D29968491E9960D3E90021891AE0
:10D7D0001860084420F07F40586031460120FEF771
:10D7E000ADFE5FEA0009F8D0204800EB861010F883
:10D7F0001800022804D1324641460620FEF76CFE8E
:10D80000FF2084F8290097F82100194E20281CBF1A
:10D81000707801F00BFB207F20B100F07FFE00202C
:10D8200020776077B9F1020F11D0B9F1010F1CBF59
:10D8300003B0BDE8F08F4FF0FF307168002904BFDE
:10D8400003B0BDE8F08F03B0BDE8F04F0847A06813
:10D85000401B05F00FFF71680029F4D103B0BDE84B
:10D86000F08F0000582A002058260020D8290020D8
:10D87000F002002070B5424C054682B094F83200A8
:10D88000202808D06068B0F1FF3F09D040F6E421BD
:10D89000702001F0F7F940F6E321702001F0F2F971
:10D8A00094F832003749C0EBC00001EB8006B06845
:10D8B00005F0E0FE0246F08A317D334B0844401CFF
:10D8C00011189A4217D8314A90421BDCC2F1000C61
:10D8D00060451EDB56008E42DCBF01F5F701A1F169
:10D8E000F85105DD0029BCBFA1F5F70101F1F851A0
:10D8F0004819994204D940F29E51702001F0C2F9B2
:10D90000954204DD40F29F51702001F0BBF965455E
:10D9100004DA4FF4B461702001F0B4F98642DCBF40
:10D9200000F5F700A0F1F85005DD0028BCBFA0F518
:10D93000F70000F1F85001AA694600F0E9F89DF8F7
:10D9400004000F288CBF012000200099084420F01B
:10D950007F41616094F827008DF800009DF8000079
:10D96000002804BF02B070BD052000F0FBFB0028BA
:10D970001CBF02B070BD40F6EB21702001F082F9AF
:10D98000582A002058260020FF7F841E0040420FA6
:10D9900070B51C4C202184F8201084F8211084F8E4
:10D9A0002210002084F8310084F83210421EC4E9AD
:10D9B0000002A07784F8260084F82700207760779B
:10D9C00084F83310E26284F83000A4F1820110225E
:10D9D000887001F8040F521EFAD100F0CDFD0A4DF7
:10D9E000012684F82860FF202870084801F000FA1A
:10D9F000687001F06BFAA86000F048FD84F83460AC
:10DA000070BD0000582A0020F002002001C4000070
:10DA100000B583B0684600F0EBF9009805F02AFEE7
:10DA2000019A034B0021E2FB030103B000BD00009B
:10DA30000080841E70B5064682B01D46104605F073
:10DA400019FE0446684600F0D3F920490198A0FB6E
:10DA50000102301A44BFA0F5F70010F1F85004D5C8
:10DA600040F60B41702001F00DF9884204DB40F6CE
:10DA70000C41702001F006F9154A211A00238A1A78
:10DA800073F1000218D3DFF848C0021BB2EB0C0C94
:10DA900073F1000310D30F4B8B423EBFC0F59020B3
:10DAA00000F1F450011907D393420AD2C4F5902132
:10DAB00001F1F4510844414201F10F0002B0281A6B
:10DAC00070BD40F60531702001F0DCF80080841E46
:10DAD0000040420FFF7F841E410B48F237625143E2
:10DAE0000A0C094B510202FB03020848504300F59F
:10DAF00086306E30400D5B4210FB03F3B2EB532FC8
:10DB000088BF491C08447047F7C2FFFF6F0C010033
:10DB1000430B48F2376C03FB0CF330B41B0CDFF8FB
:10DB200044C05C0203FB0C030F4858434FEA505CAF
:10DB300004EB0C0043F609541CFB04F404F5807C50
:10DB400043F60855A3EB5C2C2C440CF0FF0CB3EB14
:10DB5000542F84BF4FF0000C401C086082F800C0B6
:10DB600030BC7047F7C2FFFF6F0C01002DE9F04198
:10DB70003B4DD5F80403DFF8EC8010F4803F4FF400
:10DB800000664FF0E0274FF0000419D036480068D7
:10DB9000B0B1C5F84041C7F88062D5F84005D8F863
:10DBA0000010401A20F07F40022802D3B0F5000F89
:10DBB00006D94FF48030C5F808030420FEF798FE1C
:10DBC000D5F8040310F4003F1AD028480068B8B113
:10DBD000C5F84441C7F880622548D0F84005D8F818
:10DBE0000010401A20F07F40022802D3B0F5000F49
:10DBF00006D94FF40030C5F808030520FEF778FE7B
:10DC0000D5F8040310F4802F1AD01A480068B8B170
:10DC1000C5F84841C7F880621748D0F84005D8F8E1
:10DC20000010401A20F07F40022802D3B0F5000F08
:10DC300006D94FF48020C5F808030620FEF758FEE9
:10DC4000D5F80401002808BFBDE8F081C5F80441FB
:10DC5000C7F880620948C168491CC160BDE8F0810D
:10DC600000B0004004B5004040B1004044B1004065
:10DC700004B0004048B1004008B00040FC02002061
:10DC80002DE9F041384D2878042868D0A81C0122DD
:10DC9000017859B1012908BF6A7002D0697800295A
:10DCA00058D002210170407800F012FB2F4CD4F8BC
:10DCB00004034FF0000810F4002F4FF480774FF06A
:10DCC000E0260AD02A48006838B1032000F000FBA3
:10DCD000C6F880720320FEF70BFED4F8040310F49C
:10DCE000802F0AD02348006838B1022000F0F0FAF3
:10DCF000C6F880720220FEF7FBFDD4F8040310F48E
:10DD0000003F0AD01C48006838B1012000F0E0FA5A
:10DD1000C6F880720120FEF7EBFDD4F8040310F47E
:10DD2000803F08BFBDE8F08114480068002808BFA4
:10DD3000BDE8F081002000F0CBFAC6F88072042024
:10DD40002870C5F80480C4F80082BDE8F0410020C6
:10DD5000FEF7CEBD4FF495616C2000F093FFBDE857
:10DD6000F0410720FEF7C4BDFC0200200080004007
:10DD70004C81004048810040448100404081004087
:10DD8000012211024FF0E0230020C3F8801103F5B7
:10DD9000C073BFF34F8FBFF36F8FC3F800110E49ED
:10DDA00041F8042F431EC1F80433C1F83C05C1F803
:10DDB0003C010A4BC3F84005C1F840011B1DC3F8E4
:10DDC0004005C1F844011B1DC3F84005C1F84801D6
:10DDD000CA600349487070470080004004800040DA
:10DDE000FC020020014800687047000004B50040B4
:10DDF00030B4EFF3108C72B600250B4B0B4A00BF0A
:10DE0000D3F80415D3F804412CB1D168491CD16072
:10DE1000C3F80451F4E7D268BCF1000F00D162B638
:10DE2000C0E9001230BC704700B00040FC02002086
:10DE30002DE9F047DFF834810546A8F1020698F88D
:10DE40000030B068012B04BFA842BDE8F0874FF056
:10DE50004041474A11604849464AC1F8082301F148
:10DE6000040C4FF00004002B55D0444AC1F848235D
:10DE7000CCF84045C1F84441D1F8482101274FF082
:10DE8000E029002A01BFD1F80421002A4FF40062E2
:10DE9000C9F880224FF0100A4FF48032C1F80823ED
:10DEA000C1F84823C1F84041354AD2F800C0A5EB7B
:10DEB0000C0C2CF07F4CBCF1020F37D3BCF5000FDB
:10DEC00034D8C1F840554FF4803CC1F844C32BB15D
:10DED0001168411A21F07F410229F9D3776034702B
:10DEE000FFF74EFF2748D0F8041564F30101C0F88E
:10DEF0000415D0F80825022161F30102C0F80825B5
:10DF00009AFAAAF1B1FA81F1092917D940F25531EB
:10DF10001DA000F08BFEC1F84823C1F84045C1F8B0
:10DF20004041CCF84045C1F84441A5E70020C1F884
:10DF300040054FF427716C2000F0A4FEC0F81015C6
:10DF4000C7607168C0F800124FF48070C9F8800291
:10DF5000C9F800010F49C00508600420B56088F8C1
:10DF6000010088F80070BDE8F0870000FE02002084
:10DF700008F50140FDFFFBFF00B00040FDFFFAFF88
:10DF800004B50040008000406E72665F74696D6584
:10DF9000722E680004F5014070B52A4CA1688142D8
:10DFA00014BF01220022DFF8A0C09CF80050022D0F
:10DFB00002D0002A34D002E0002A08BF70BD627887
:10DFC0009AB3224B4FF080421A60214B9213C3F850
:10DFD0000823C3F848230022C3F840211D4A1668CD
:10DFE000861B26F07F46022E24D3B6F5000F21D8DB
:10DFF000C3F840054FF48036C3F844632DB113686D
:10E00000CB1A23F07F43022BF9D3134B02214A078B
:10E010001A60A06004208CF801008CF8001070BD1C
:10E0200040F2AA216C2000F02DFE40F2AE216C20BF
:10E0300000F028FE0020C3F8400540F2BA216C2011
:10E0400000F020FEFC020020FE02002008F5014046
:10E0500000B0004004B5004004F50140014880686C
:10E0600070470000FC0200202DE9F0413648354A97
:10E07000C0F80823DFF8D4C0031D00219CF800403D
:10E0800084B1334AC0F84823C3F84015C0F844119E
:10E09000D0F848210123002A04BFD0F80401002849
:10E0A00011D10AE0C0F84823C0F84015C0F840116B
:10E0B000C3F84015C0F84411EAE74FF0E0224FF4EE
:10E0C0000060C2F88002022C04D040F2C6216C200D
:10E0D00000F0D8FD1F4E30681F4CC01C20F07F4060
:10E0E000A2681E4D90420BD03768D71B27F07F47A0
:10E0F000042F05D3B7F5000F02D8FFF799FE1BE0F8
:10E100003068101A20F07F40022813D3B0F5000FBA
:10E1100010D8134A4FF080401060636021706B602C
:10E12000EB604000111F086004208CF801008CF89F
:10E13000003001E0636021706068C5F80002BDE84E
:10E14000F0810000FDFFFBFF00B00040FE02002058
:10E15000FDFFFAFF04B50040FC02002000800040F3
:10E1600008F501402DE9F041544A0025012492F8B8
:10E1700000C053784FF4A07607287DD2DFE800F086
:10E1800004040404585858004D4A9768B7F1807F3A
:10E1900004BF5278002A03D0BCF1020F05D026E05C
:10E1A00040F256316C2000F06DFD1A1FD2B206EB22
:10E1B000820202F1804606F530460022BCF1010FD2
:10E1C00003D0BCF1020F08D00EE0042B24BF376847
:10E1D000002F08BF4FF0004206E0042B24BF376831
:10E1E000002F08BF42F0804212F0804FE5D1DFF8E7
:10E1F000D4C000F1100204FA02F2CCF808234FF068
:10E20000400303EB8003DBB263441C600CEB800033
:10E21000D0F84035A1EB030323F07F43032B26BF47
:10E22000C0F84015CCF80423C0F8405537D23CE084
:10E23000BCF1000F06D0834204D140F276316C204D
:10E2400000F020FD021FD3B2032B04D340F2D11102
:10E250006C2000F017FDDFF870C003F1100204FA23
:10E2600002F2CCF80823CCF8482306EB83034CF8E1
:10E270000350164B1B6800E01AE0001FCB1A23F076
:10E280007F43C0B20CEB8000022B0BD3B3F5000F21
:10E2900008D8C0F84015CCF80423CCF8442301205A
:10E2A000BDE8F0810021C0F840150020BDE8F081F4
:10E2B00040F27A316C2000F0E5FC0000FE02002004
:10E2C000FC0200200080004000B0004004B5004087
:10E2D0002DE9F843012600274FF4A078072851D2F2
:10E2E000DFE800F0040404041919190000F110011A
:10E2F00006FA01F22649C1F8082301EB8003002247
:10E30000C3F8402508EB80028F50224951F82000C5
:10E310000090BDE8F883204D011FCCB2297879B177
:10E320006A7882420CD11D4A4FF0404010600129AA
:10E3300008BFFFF725FD2F7019494FF080708860E6
:10E34000184904F1100006FA00F0C1F80803C1F8FA
:10E350004803A0000844D0F84005134A1268801A08
:10E3600020F07F40022807D301EB84020020C2F88E
:10E37000400508EB84000F500C4850F82400009032
:10E38000BDE8F88340F2FE316C2000F07BFC000019
:10E390000080004040810040FE02002008F501405E
:10E3A000FC02002000B0004004B5004040B1004035
:10E3B0002548244AC0F808232449031D91F800C0C9
:10E3C0000021BCF1000F10D0214AC0F84823C3F847
:10E3D0004015C0F8441100BFD0F84821002A04BFFE
:10E3E000D0F80401002811D10AE0C0F84823C0F891
:10E3F0004015C0F84011C3F84015C0F84411EBE7D0
:10E400004FF0E0224FF40060C2F8800211484FF054
:10E41000FF32C0F80823C0F84015C0F8401100F1E1
:10E420000402C2F84015C0F8441102F10402C2F817
:10E430004015C0F8481102F10402C2F84015C0F8B6
:10E440004C117047FDFFFBFF00B00040FE020020B2
:10E45000FDFFFAFF0080004010B507280DD2DFE86D
:10E4600000F00404040406060600064902E0001F4A
:10E470000549C0B201EB800010BD40F29E316C2016
:10E4800000F000FC4081004040B1004070B51F48E2
:10E49000002404210470801E01708905C46081601D
:10E4A000FFF76EFC01254FF0E02CEB02CCF8803139
:10E4B000BFF34F8FBFF36F8FCCF8803214484560A5
:10E4C000856014490A68002AFCD1511EC0F808135F
:10E4D000C0F84813C0F84045C0F840410E49C1F8A3
:10E4E0004045C0F84441091DC1F84045C0F84841C5
:10E4F000C0F80441CCF8003105604FF48271C0F8D7
:10E5000044130221C0F8041370BD0000FE02002075
:10E5100000B0004004B5004004B00040084890F945
:10E5200000000028B8BF704700F01F01012202FA66
:10E5300001F14009800000F1E020C0F800127047AE
:10E54000840300200348007803280CBF012000202A
:10E55000704700005C0300200148408870470000BD
:10E560005C03002003480078022816BF032801201E
:10E57000002070475C0300200248002101704180A8
:10E58000704700005C0300202DE9F041164C607AD2
:10E59000002827D04FF480718D05284605F095F8A6
:10E5A00080464FF48271284605F08FF80026074612
:10E5B000B8F1000F09D00120C5F80803207920B177
:10E5C0002671E06908B18047E66137B1C5F804619A
:10E5D0000220C5F8080300F075FA4046BDE8F04196
:10E5E00000F058B8BDE8F0810C03002010B505F02C
:10E5F00016F930B905F034F918B905F067F90028B3
:10E6000002D002490220086010BD0000340C004016
:10E6100070B500F09BF900F0BDFA094C4FF0804551
:10E6200030B1FFF7E3FF012028610420A07204E06D
:10E630000320A0720120C5F804030020E07170BD22
:10E640000C03002070B5124CA079E0B1E179401EB6
:10E65000814218DA00F09EFA054600F087FBA179A6
:10E66000012902D9E179491CE1710DB1616900E02C
:10E670002169411A022902DA11F1020F07DC0DB1FA
:10E68000606100E02061BDE87040FFF7C1BF70BD70
:10E690000C0300202DE9F04706464FF080454FF46B
:10E6A0008671284605F011F880464FF48871284697
:10E6B00005F00BF8274C8246277804F1080005F096
:10E6C00078F810B14FF4DB7116E04FF0010946B154
:10E6D000A07A032805D10420A072FFF787FFC5F8B0
:10E6E00010900026B8F1000F18D0C5F80C61A07A80
:10E6F000042804D04FF4E4716D2000F0C3FA05F053
:10E700008EF828B905F0ACF810B905F0DFF808B1BB
:10E71000114806600220A07200F0FCF8BAF1000F68
:10E7200008D0C5F81061A07A022801D1FFF78AFF4E
:10E73000C5F814903FB12670A07A022801D1FFF7E6
:10E7400067FF00F0E7F8BDE8F0470248083005F041
:10E7500047B800000C030020340C00402DE9F041C4
:10E76000494C00270646A761427881780078E0721C
:10E770006271A171E7714FF001084FF080450528E3
:10E7800025D2DFE800F0100306202200C4F818802C
:10E7900009E000F0DBF80121284604F09BFF002887
:10E7A000F9D00220A06104F0C1FFC0B100F00CFA62
:10E7B000217E01F00301884211D1B07960B10220BD
:10E7C000C5F8040344E03148ECE73148EAE740F299
:10E7D0003D316D2000F056FA00F0CAF938E0C5F876
:10E7E0000C80C5F80471A069C5F8180505F003F898
:10E7F00040B905F00AF828B905F01EF810B905F07F
:10E800002FF838B14FF08050D0F844022149C0F3BE
:10E810004230086004F0EFFF40B904F0F6FF28B979
:10E8200005F00AF810B905F01BF818B119491031B4
:10E83000C1F80080C5F808800220C5F80403B0794B
:10E8400030B900F029F80220C5F80803C5F80471B2
:10E85000A07970B1307860B900F09CF9064600F0FC
:10E8600085FA6FF0004116B1C4E9041001E0C4E973
:10E8700004010121284604F02DFF08B100F084F9BD
:10E88000A772BDE8F08100000C0300200100020027
:10E89000010003003C0500402DE9F0414FF08045A8
:10E8A000D5F8040310F0020F11D0164C2068C043B5
:10E8B00040F30016206840F0100020604FF482778B
:10E8C00039462846761C04F000FF28B10AE04FF4D0
:10E8D0003E716D2000F0D6F905F004F802E000BFAB
:10E8E00004F0FEFF3946284604F0EFFE0028F7D07A
:10E8F00000F03EF9002E03D1206820F010002060C7
:10E90000BDE8F08110ED00E00148C08970470000CB
:10E910000C03002010B5EFF3108472B60A4841785A
:10E9200029B14178491E4170417829B108E040F28F
:10E9300019116D2000F0A6F9807808B900F038F9B7
:10E94000002C00D162B610BD0C03002010B5EFF30F
:10E95000108472B606484178491C417040780128FD
:10E9600001D104F0CEFE002C00D162B610BD000033
:10E970000C030020054810B5C17821B100210171B8
:10E98000C170FFF7C7FF002010BD00000C0300207E
:10E9900070B50C4CE17861B90125E570E061FFF7D5
:10E9A000D5FF00F0F7F830B1E06910B180470020E2
:10E9B000E061002070BD4FF080402571C0F8045325
:10E9C000F7E700000C0300202DE9F04105006FF08F
:10E9D00015003FD0297804293CD8002969783BD01C
:10E9E000002937D1A978002934D1002004F05CFE39
:10E9F000002004F04CFE4FF080484FF0FF31C8F883
:10EA000008130026C8F80061C8F80461C8F80C6152
:10EA1000C8F81061144C6670A888A08104F068FEE4
:10EA2000012708B1E77067700121404604F052FEEB
:10EA300008B100F0A9F840F2F550E0812846FFF750
:10EA40008DFE6772002004F022FE4FF0E021304678
:10EA5000C1F80071BDE8F0810029FBD02029F9D868
:10EA6000A9782129C1D9F5E70C0300200148808944
:10EA7000704700000C03002010B50D4804F099FE0B
:10EA80000B49083948B1012008704FF0E021C1F866
:10EA90000002BDE81040FFF759BF887A022801D173
:10EAA000FFF7B6FDBDE81040014804F099BE000034
:10EAB000140300200248807A002800D0012070470B
:10EAC0000C030020F8B51F4DE87A00280FD1287EEE
:10EAD00000F0030004F01AFE002808D0EFF31081C4
:10EAE00072B6FFF7E7FF18B1002900D162B6F8BD92
:10EAF0000126AE7201B962B618204FF08044C4F806
:10EB00000803A6614FF42070ADF80000BDF80000C6
:10EB1000411EADF80010F9D20027C4F80C71C4F8FA
:10EB200010710848083004F057FE2F70FFF770FD91
:10EB30006661687900F07F00C4F838051820C4F8D1
:10EB40000403F8BD0C030020024610B50020002984
:10EB50000AD0002A08D0A2FB0101401E034A41F15D
:10EB6000FF3104F0C1FE401C10BD000040420F0008
:10EB700010B5044C207E00F0030004F0C7FD00280F
:10EB8000F8D010BD0C030020014901200870704727
:10EB9000850300204FF08040D0F8000118B90348E9
:10EBA0000078002800D00120704700008503002075
:10EBB0004FF08040012141600021C0F80011014860
:10EBC00001707047850300200248006800F00300D0
:10EBD000704700001C04004010B531B1012907D076
:10EBE00040F2023105A000F021F8D0F8140401E051
:10EBF000D0F8080400F0010010BD00006E72665FDE
:10EC0000636C6F636B2E6800BFF34F8F054801681C
:10EC1000054A01F4E06111430160BFF34F8F00BF6B
:10EC2000FDE700000CED00E00400FA0572B6034AAF
:10EC3000526802B19047FFF7E7FF00002C03002065
:10EC4000064810B50021016001210160084604F06A
:10EC500084FDBDE81040012004F072BDFC1F00409F
:10EC6000074810B501214160891EC0F808130C2027
:10EC700004F073FDBDE810400C2004F061BD0000FD
:10EC800000C000400EB572B60F4A5568D5B10022DB
:10EC900003466E460A2403E0B0FBF4F0521CD2B2E5
:10ECA0000028F9D1B05409E0B3FBF4F004FB1030B4
:10ECB000B3FBF4F3521ED2B23030B054002AF3D179
:10ECC0003046A847FFF7A0FF2C0300202DE9F041B4
:10ECD000184C0646174660780D4618B14FF0FF30C5
:10ECE000BDE8F081FCF752FA06B9134E6760257053
:10ECF000FFF7A6FFFFF7B4FF3046FFF765FE0600FB
:10ED0000EED1FEF745FEFFF7DDFE04F00DFC2846D0
:10ED100004F016FD0120002D09DB05F01F0100FAAB
:10ED200001F16A09920002F1E022C2F8001160705C
:10ED30003046D5E72C0300207C370100014840789D
:10ED4000704700002C030020074890F900000028BD
:10ED500009DB00F01F02012191404009800000F111
:10ED6000E020C0F8001270472C0300202DE9F0418C
:10ED700001264FF0E02231034FF000084046C2F870
:10ED80008011BFF34F8FBFF36F8F164CC4F8000193
:10ED90000C2004F001FD144D2868C04340F3001717
:10EDA000286840F010002860C4F8046326607F1CC7
:10EDB00002E000BF04F094FDD4F800010028F9D06F
:10EDC0001FB9286820F010002860084805686660B0
:10EDD000C4F80863C4F800810C2004F0DDFC284668
:10EDE000BDE8F08100C0004010ED00E008C5004023
:10EDF00010B5024605200C4904E000BF01EBC0033A
:10EE00001B7933B1401EC0B2F8D248216920FFF708
:10EE100039FF41F8302001EBC00100224A718A71AC
:10EE200001220A7110BD0000902A002010B50528AB
:10EE300001D3582106E00A4901EBC00001790129FC
:10EE400003D059216920FFF71DFF41798279491CC0
:10EE5000C9B28A4200D04171BDE81040FFF774BFCB
:10EE6000902A002010B5052803D34F216920FFF711
:10EE700009FF034A002102EBC000017110BD000030
:10EE8000902A002070B505250E4E0F4C16E0217813
:10EE900006EBC1000279012A08D1427983799A42AE
:10EEA00004D04279827156F8310080472078401CA6
:10EEB000C0B22070052801D3002020706D1EEDB275
:10EEC000E5D270BD902A00208603002000B504F032
:10EED00092FC40B904F099FC28B904F0ADFC10B9DB
:10EEE00004F0BEFC08B1024800BD024800BD0000AD
:10EEF0000C05004000E7014010B504F0B1FC30B350
:10EF0000EFF31080C8B1002172B61248026803689E
:10EF1000C2F3001243F0100303604FF0E023D3F874
:10EF20000042D3F804321C4300D040BF20BF00BFD2
:10EF300000BF00BF00BF12B105E00121E4E7026895
:10EF400022F010020260002900D062B610BD20BF7E
:10EF500010BD000010ED00E00149012088707047ED
:10EF600034030020433B01007B3B0100653B010073
:10EF7000533B01005F3B01004D3B0100413B010061
:10EF80003F3B0100773B01006B3B0100593B010017
:10EF9000473B0100393B0100313B0100353B01009B
:10EFA0002B3B01000148006800680047480300202F
:10EFB000014800684069004748030020014A126880
:10EFC000D26810474803002001490968C96A084708
:10EFD00048030020014800680069004748030020FA
:10EFE000014A1268926810474803002001490968E5
:10EFF000496A08474803002001490968896A0847A7
:10F000004803002030B4034C24686468A44630BC34
:10F010006047000048030020014800787047000066
:10F02000870300202DE9F04786468C460846089E57
:10F03000154674461946002B40F0C2808542B2FA4C
:10F0400082F245D94AB1C2F1200300FA02FC2EFA3D
:10F0500003F3954043EA0C0C94404FEA154EA8B2D6
:10F06000BCFBFEF8230C0EFB18CC08FB00F943EAAE
:10F070000C43994528D9EB1808F1FF3704D299457C
:10F0800002D9A8F102072B44A3EB0903A4B2B3FBF6
:10F09000FEFC0EFB1C330CFB00F044EA0344A042D0
:10F0A00014D92C190CF1FF3304D2A04202D9ACF1CF
:10F0B00002032C44241A43EA07401EB1D440002323
:10F0C00034607360BDE8F0874746DDE76346F1E7EB
:10F0D00092BB431B01214FEA154EAFB2B3FBFEFCBE
:10F0E000200C0EFB1C330CFB07F840EA0343984549
:10F0F00062D9EB180CF1FF3004D2984502D9ACF17B
:10F1000002002B44A3EB0803A4B2B3FBFEFC0EFBEE
:10F110001C330CFB07F744EA0344A7424ED92C19D1
:10F120000CF1FF3304D2A74202D9ACF102032C4404
:10F13000E41B43EA0040C0E7C2F1200320FA03F1D8
:10F14000954090402EFA03F303434FEA154EAFB2B9
:10F15000B1FBFEFC0EFB1C10190C0CFB07F841EA7E
:10F160000041884504FA02F422D969180CF1FF30F5
:10F1700004D2884502D9ACF102002944A1EB080170
:10F180009BB2B1FBFEFC0EFB1C110CFB07F743EA24
:10F1900001439F420ED9EB180CF1FF3104D29F427C
:10F1A00002D9ACF102012B44DB1B41EA004192E79A
:10F1B0006046E3E76146F7E76046A3E76346B7E7E3
:10F1C000834206D916B9002108467BE7C6E900E06C
:10F1D000F9E7B3FA83F78FB9834201D3724508D8B0
:10F1E000BEEB020460EB030301209C461EB9002124
:10F1F00068E73846FAE7C6E9004CF8E7C7F1200CA3
:10F20000BB4022FA0CF41C432EFA0CF120FA0CF34A
:10F21000B84001434FEA14490EFA07F5B3FBF9F879
:10F220001FFA84FE09FB18300B0C08FB0EFA43EAA8
:10F2300000439A4502FA07F240D9E31808F1FF307B
:10F2400004D29A4502D9A8F102002344A3EB0A0391
:10F2500089B2B3FBF9F809FB183308FB0EFE41EA4B
:10F2600003418E452CD9611808F1FF3304D28E4535
:10F2700002D9A8F10203214443EA0040A0FB02980E
:10F28000A1EB0E014145CE46434602D306D14D4582
:10F2900004D2B9EB020E68EB04030138002EA6D0AD
:10F2A000B5EB0E0261EB030101FA0CFC22FA07F345
:10F2B0004CEA0303F940C6E9003198E74046C5E748
:10F2C0004346D9E710F8012B11F8013B012A28BF6A
:10F2D0009A42F7D0D01A7047034613F8012B002A40
:10F2E000FBD1181A013870472DE9F84F0C468146BA
:10F2F000497800F103008DF8001020F00300A17898
:10F30000150006468DF8011000D000206946F4F77C
:10F31000ABFB06EB000A207861780027084400F078
:10F32000FF083E4608E0237AE279A179607900F08F
:10F33000ABFE761C0744F6B24645F4D30AF103004F
:10F3400020F00300064605B100203A464146F4F796
:10F350003FFD3044A1782E4659B1C01C20F0030077
:10F36000638AE2780546C9B206B10020F4F7E4FDED
:10F370002844C01D20F00700A0EB0900BDE8F88F6D
:10F3800030B50D468DB0144601461022684604F093
:10F39000F2FA1022294604A804F0EDFA684600F0BB
:10F3A000F8FF18B16FF015000DB030BD10222046E7
:10F3B00008A904F0E0FA0020F6E70EB50146684619
:10F3C00000F018F8684601F07FFC0EBD70B50C46E1
:10F3D0000546F4F7BFFA002802D03E2D01D00120E7
:10F3E00070BD122C04D02046BDE87040F4F7C4BABA
:10F3F000002070BD0A88C2F30B0282804A88C28056
:10F400004A789309002242724B78C3F301131BB16F
:10F41000012B05D0022B05D00272091D0160704737
:10F420000122F9E70222F7E710B50C4609790170CD
:10F43000417801F0F0014170A288C2F30322114328
:10F440004170A2798270E28801F0CF01120AC27085
:10F450004170227A41EA021101F03F014170627A63
:10F4600041EA821141702168021D914206D0E28872
:10F47000FB2A00D3FB22001D04F07DFAA079001DB9
:10F48000C0B210BD30B40A790270427802F0F002C6
:10F4900042708B88C3F303231A4342708B798370C5
:10F4A000C37802F0CF0203F0C003C370CC88C4F36A
:10F4B00005242343C37042700C7A04F0030442EA2B
:10F4C000041202F0BF0242704C7A42EA841202F047
:10F4D0007F02427003F03F02C2700B68021D93422C
:10F4E00005D0CA8830BC1946001D04F044BA30BCAF
:10F4F00070472DE9F0410D4604460F7800200C229C
:10F5000005233E26FF211E2F7DD2DFE807F0CE0F18
:10F510002628CE495364809395A0ABC6D0CECECEDC
:10F520002EB6B9D9F1F4EEEDECEBEAE922702879C8
:10F53000A0706879E070B5F80500000A2071E879DC
:10F540006071287AA0712889000AE071A87A207277
:10F550006889000A60720820A5E0102000E01A20E7
:10F5600020702879A07001209DE02920F4F704FA8A
:10F5700048B126702920A0702122291DE01C04F02A
:10F58000FAF922208FE00A20F4F7F6F9002829463C
:10F59000204602D000F05BF983E000F02FF980E014
:10F5A00026701420A0702879E070A888000A2071C5
:10F5B000A879BFE03E2222700422A2706868C4F8D5
:10F5C0000300A868C4F80700A889A4F80B00A87B6A
:10F5D00060730C2067E026700320A0702879E0702B
:10F5E000A8792071E888000A6071287AA0712889BA
:10F5F000000AE071A87A20726889000A6072287B8C
:10F60000A072A88900E050E0000AE072CFE0267006
:10F61000A3702879E070A888000A2071D5F8060048
:10F62000C4F80500D5F80A00C4F80900E889A4F870
:10F630000D00E1E011203BE023702879A07068798B
:10F64000E070B5F80500000A2071E87972E0082042
:10F6500020702879A070A879E070E888000A2071ED
:10F66000287A67E0302020702879A070A879E070AF
:10F67000E888000A2071032015E0267007205EE06C
:10F680002670A2702879E070A8792071E888000AB5
:10F690006071287AA071687A1FE0291D2046F4F76E
:10F6A0002BF9002801D06070801CBDE8F081572044
:10F6B00020702879A070A888000AE0700220F2E784
:10F6C00026701220A0702879E07068792071A879DE
:10F6D0006071E888000AA071287AE0710620E2E7EC
:10F6E00075E048E029E054E063E01BE003E0FFE759
:10F6F0002670202041E026702120A0702879E0703B
:10F7000068792071B5F80500000A6071E879A07188
:10F71000287AE071687A2072A87A6072E87AA0721A
:10F720000920C0E72170A120A0702879E0706879D5
:10F730002071002060710420B5E72170A220A07024
:10F740002879E070A888000A2071A8796071E8889B
:10F75000000AA071287AE0712889000A2072A87A2C
:10F7600060726889000AA072287BE072A889000A8A
:10F7700020730B2097E72170A320A0702879E070F8
:10F78000A888000A2071A8796071E879A071052025
:10F7900089E726701320A0702879E07068792071BD
:10F7A000D5F80600C4F805006889A4F809000A2005
:10F7B00079E72170A420A0702879E070A888000A59
:10F7C0002071A8796071E879A07107206BE721703A
:10F7D0008020A070A988A4F80310E988A4F8051077
:10F7E000297AE17169892181A9896181E989A181E8
:10F7F000297C01F00101A1730D2054E73E22027023
:10F80000012282700A79C27011F8052F02710A88EC
:10F81000120A42718A788271CA78C2714A6882601B
:10F820000A8982818A7D8273CA8A120AC2730A7E19
:10F8300002740A8B120A42748A7E82744A8B120AFC
:10F84000C274097F017513214170084670473E223A
:10F8500002700A2282700A79C27011F8052F0271B3
:10F860000A88120A42718A788271CA78C2714A681B
:10F8700082600A898281D1F80A20C0F80E20CA89E4
:10F8800042820A6942618A8A02838A7D8276CA8AB2
:10F89000120AC2760A7E02770A8B120A42778A7EA1
:10F8A00082774A8B120AC277097F80F820101F21C5
:10F8B0004170084670474A0901F01F0150F82200C4
:10F8C000C84000F00100704710B56FF0150420B17A
:10F8D000FFF773FD08B1002010BD204610BD10B524
:10F8E0000C4630B12CB1F3F7B7FF28B120700020DF
:10F8F00010BD6FF0150010BD6FF0220010BD03F0B9
:10F900009FB903F0BAB910B5F4F750F8002010BD54
:10F9100010B5F4F75DF8002010BD03F0CFB908B5BD
:10F9200000788DF80000684603F0ABF808BD0120B0
:10F930007047F9F7E5BE012070478178008803F031
:10F9400050B8007800B1012003F046B803F073B856
:10F9500010B50446FFF70AFAC11700EB917080104A
:10F960007F2801DD7F2004E06FF07E01884200DA0D
:10F9700008462070002010BD70B5054610220021F9
:10F9800004F073F81022002105F1100004F06DF866
:10F990004FF08054D4F88000401C0BD1D4F8840080
:10F9A000401C07D1D4F88800401C03D1D4F88C0047
:10F9B000401C0BD0D4F88020D4F88400D4F88810F0
:10F9C000D4F88C302A616861A961EB610020F4F7FA
:10F9D00013FD18B9D4F8A000C00718D1D4F89000CE
:10F9E000401C0BD1D4F89400401C07D1D4F89800E7
:10F9F000401C03D1D4F89C00401C08D054F8900F50
:10FA00006168A268E36828606960AA60EB60002012
:10FA100070BD38B54FF080550446D5F8A400401CA1
:10FA200005D1D5F8A800C0430004000C3ED0D5F89D
:10FA3000A000C0073AD0D5F8A400D5F8A810ADF8BA
:10FA40000010C4F80100BDF80000A4F80500A0797A
:10FA500040F0C000A071D5F89000401C0FD0D5F840
:10FA60009400401C0BD0D5F89800401C07D0D5F866
:10FA70009C00401C03D00020F4F7BEFC40B11022D3
:10FA80000021E01D03F0F1FF01202070002038BDAF
:10FA900055F8902F6968A868EB68C4F80720C4F887
:10FAA0000B10C4F80F00C4F81330EDE70020ECE7AA
:10FAB00002F0D6BF03F0D5B8F9F730BE02F012BDA0
:10FAC00002F0F5BC02F032BD02F023BD02F038BDF9
:10FAD00002880A8002F03DBD02880A8002F052BD11
:10FAE00002F07ABD02F07EBDF9F712BDF9F71ABD3A
:10FAF00002F0BCBD02F081BDF9F73CBD02F086BD4D
:10FB000002F0A0BDF9F75CBD02F0A0BD02F0CBBDD4
:10FB100002F0B0BD02F0DCBD02F0E8BD02F0FBBDBA
:10FB200002F02CBE02F0BFBE02F0DDBEF9F752BDFE
:10FB300010B5F3F729FF002010BD02F0E1BE02F07E
:10FB4000F8BE02F00CBF02F018BF02F01FBF02F0B7
:10FB500032BF02F05EBCF9F7EBBD70B50B88C47C18
:10FB600000F11805C3F30E0602883544641D2D8884
:10FB7000224492B22544541E2C4494FBF2F402FB1E
:10FB80000462408892B2904203D903F400401043CB
:10FB900002E04FF400409843088070BD4204B2EB8D
:10FBA000414F07D100F4004001F40041884201D0E8
:10FBB00001207047002070478188C088884201D1A9
:10FBC00001207047002070472DE9F0410F460446A0
:10FBD00000F1180180880026C0F30E0045183E6031
:10FBE000E089002816D06189084480B260812988A4
:10FBF000884205D940F251114FF01400F3F732FD5D
:10FC000006D104F104012046FFF7A7FF66813D609D
:10FC1000E6810120BDE8F0812DE9F041044600F1C4
:10FC20001803C0880E46C0F30E07208AD91908B100
:10FC3000B04202D20020BDE8F081A089002540B189
:10FC4000B1F800C0604506D04FF401711420F3F7FD
:10FC500009FD0D800EE094F813C018440CF1050C5A
:10FC6000BC446044B4F814C020F803CC94F816C027
:10FC700000F801CCA0893044A08108883044088075
:10FC80002AB1A11D2046FFF768FFA5810AE0E07CAC
:10FC9000A189401D38441944084430F8031DA1824D
:10FCA0008078A07525820120C5E7801C704710B5BB
:10FCB0000446C088A188814203D0608908B9E089E0
:10FCC00008B1002010BD211D2046FFF746FF00208F
:10FCD000E081012010BD10B5044600F11802C08873
:10FCE000C0F30E0002442088452800D245208842F7
:10FCF00004D24FF482711420F3F7B4FCA07C0028E6
:10FD000003D01088884201D2002010BD1180A11DAF
:10FD10002046FFF722FF0020A074012010BD10B57F
:10FD2000C4888388014600F11802C3F30E00104412
:10FD3000A34202D04989002900D0002010BD0388C9
:10FD4000452B00D245231380C288C2F30E0300F175
:10FD500018021A440A6080897047C07C401D08441C
:10FD6000C01E1060088870472DE9F0410E46C1881A
:10FD70000289044600F118080088C1F30E05C2F399
:10FD80000E07452800D24520B04203D2C6211420D8
:10FD9000F3F768FC1046FFF701FF10B10020BDE843
:10FDA000F081AF4208D9E17C781B401A401F86429F
:10FDB00002DD0020A074F1E708EB050001210680B8
:10FDC000A174ECE738B5C488818800F11802C1F34A
:10FDD0000E031A44A14210D04389C58912882B44CE
:10FDE000934208D3ADF800106946FFF7B6FEBDF8A0
:10FDF0000000A04201D0012038BD002038BD70B500
:10FE0000C6888588034600F11804C5F30E00204417
:10FE1000B54202D10020D88170BD04885D89DE7CA6
:10FE2000641B354428440D88A4B2801CA54200D927
:10FE30000C805C8924B1002414700988D98170BDBC
:10FE40000124F9E72DE9F0411D461646069F0B46B1
:10FE500004463A462946304600F039F8834201D23A
:10FE60009E2112E0A00701D09F210EE01822002160
:10FE7000204603F0FAFDA819401D784380B2E574CE
:10FE80006080B0F5004F03D9A4211420F3F7EAFBFA
:10FE90002680BDE8F08170B50B46044600F11801DC
:10FEA00002898088C2F30E050D44824201D10020F0
:10FEB00070BD23B1E27CA91C184603F05CFD2D88BF
:10FEC00004F108012046FFF748FE284670BD0144B2
:10FED000491D51438AB20021452802D2C0F1450094
:10FEE00081B21832501880B270472DE9F047884629
:10FEF000C18804460089C1F30E0604F11805C0F359
:10FF00000E0705EB0609FFF749FE002298B9208885
:10FF1000452800D24520B74206D9E37CB91BC91A4F
:10FF2000491F814200DA0846A18911B1B9F80030B1
:10FF3000C01A404503DA22820020BDE8F087E07C49
:10FF40002944401D30440844A4F81080C01EF4E742
:10FF500070B50023A1F108024FF6F774A24204D352
:10FF600040F2CD111520F3F77DFB02680AB91EE0BF
:10FF70001046026893888B4202D01368002BF7D199
:10FF8000948813468C4201D111680DE001F10805F7
:10FF9000AEB20025B44209D3641A11440D608C80BE
:10FFA0000268126802600A60016000E000231846DF
:10FFB00070BD10B50C0004D0082C07D240F295118A
:10FFC0000AE008B100210160002010BD58B1B4F56D
:10FFD000803F04D340F2A7111520F3F743FBA1B2F1
:10FFE000006800F014F8201D10BD0021026803E035
:10FFF00093881268194489B2002AF9D100F007B831
:020000040001F9
:1000000000230B608A8002680A6001607047002349
:100010004360021D0181026070471CB50446002048
:10002000019000908DF806400AE0BDF804002146DA
:10003000F3F79EFD20B14FF429711720F3F712FB5F
:100040006846F3F74DFD0028EFD01CBDA0F57F42B8
:10005000FF3A01D0022901D300207047F3F7BABD5F
:10006000A0F57F42FF3A01D0022901D3002070475A
:10007000F3F7D8BD10B50446F3F720FEA04201D92E
:10008000012010BD002010BD70B50E461D46114662
:1000900000F013F804462946304600F004F82044E6
:1000A000001D80B270BD10B50A460921FFF70FFF91
:1000B0004FF6FC71C01C084010BD10B50A460A215D
:1000C000FFF705FF4FF6FC71C01C084010BD09B1D9
:1000D000002100E0022143181A7D022A08D05B7D2E
:1000E000022B09D0032A03D0032B05D00020704730
:1000F00000EB4100008B704700EB4100408B7047E4
:1001000009B1002100E0022100EB4100018B11B98F
:10011000408B002800D00120704738B583788DF8D7
:100120000030009B00939DF800305BB900240AB1B9
:10013000002300E00223C218157D022D04D0527D59
:10014000022A04D0002038BD1A465B1C00E05A1C6D
:1001500079B1C51800EB43032C751C830323841865
:10016000237500EB820300EB42005B680B60008BA1
:100170008880012038BD10B509B1002100E00221BE
:1001800043181C7D944203D100EB4100008B10BD4D
:100190005B7D934203D100EB4100408B10BD0020FA
:1001A00010BDB0F5FF7F01D2410800E0FF21401AE9
:1001B00040F27261884200DB084680B2704701213C
:1001C000FFF785BF2DE9F041064642F380074878E6
:1001D0000C4622F004057F1C00B10DB9284304D160
:1001E00045B100212046F3F767FEFF20A0701FB144
:1001F000002002E00121F5E702202118097D0329F2
:1002000002D1022D00D0401C22180121117504EBEF
:100210004001002204EB80000A834068A27031464E
:1002200062F30F01C6E90001BDE8F0812DE9F0415C
:100230001E461346044609B1002000E00220FF21BB
:10024000A17021180A7D012A03D0497D01290CD112
:10025000401C04EB40050027298BB5F820C08A1903
:10026000624505D920442F8307750020BDE8F08141
:1002700004EB8000324640680844194603F07BFBDB
:10028000288B30442883A7700120EFE710B50121A7
:10029000FFF736FF002800D0012010BD0122FFF734
:1002A0003CBF0022FFF739BF10B50021FFF728FF40
:1002B000002800D0012010BD70B509B1002300E076
:1002C0000223FF218170C11802240D7D012D07D06A
:1002D0004D7D012D09D04FF48B710920F3F7C2F940
:1002E00000EB43031A830C7503E000EB43035A83CE
:1002F0004C750021817070BD012101707047012291
:100300001146FFF738BF01220021FFF734BF00215B
:10031000FFF7DDBE002809DB00F01F02012191403C
:100320004009800000F1E020C0F8801270470028EA
:100330000DDB00F01F02012191404009800000F117
:10034000E020C0F88011BFF34F8FBFF36F8F70476D
:1003500010B50E20FFF7EBFF0E20FFF7DBFF0F209D
:10036000FFF7E5FFBDE810400F20FFF7D3BF0028DF
:1003700009DB00F01F02012191404009800000F1DB
:10038000E020C0F8801270474058002800D00120BB
:10039000704710B504462046F3F796FE1128FAD0B0
:1003A00010BD10B5FFF7F5FF002803D0A0211D20D8
:1003B000F3F758F910BDF3F7E5BFF3F7D3BF10B566
:1003C00050400A781C78624010444A785C78624059
:1003D00010448A789C7862401044CA78DC78624085
:1003E00010440A791C794979624010445A79514085
:1003F000C14201D1012010BD002010BD10B500295F
:1004000004464FF0060102D0F3F7CCF901E0F3F710
:10041000D7F9607900F03F00607110BD704730B5CA
:100420000C4605468DB04FF0030104F1030012B1F4
:10043000F3F7B8F901E0F3F7C3F960790D2200F0A2
:100440003F0040F040006071002104A803F00DFB64
:10045000E0788DF81F0020798DF81E0060798DF806
:100460001D0010222946684603F085FA6846FFF70A
:1004700098FF9DF82F0020709DF82E0060709DF869
:100480002D00A0700DB030BDF4F7F4BAC10701D053
:1004900001207047800701D5022070470020704777
:1004A00010B5012808D0022804D040F222410620CD
:1004B000F3F7D8F8012010BD002010BD002904D0AA
:1004C000012803D0012901D0022070470120704784
:1004D000FFF795BC0121F4F76DBE10B502F0FDFEEB
:1004E00018B1BDE81040F9F7E1BCFF2010BD10B510
:1004F000F4F7A8FE102803D0F4F774FE102800D1FA
:10050000082010BD10B5F4F79DFE102807D0F4F7B1
:1005100069FE102803D0F4F7F3FE012010BD00207F
:1005200010BD10B5F4F78EFE102803D0F4F730FF9D
:10053000012010BD002010BD70B50E468CB01446D1
:1005400001461D461022684600F038F91022314657
:1005500004A800F033F96846FFF723FF08A94FF01D
:10056000100228461CB100F029F90CB070BD03F050
:1005700002FAFAE710B50C460021FFF771FD606042
:1005800018B101202070002010BD022010BD40F2E3
:10059000E2414843704740F2E241B0FBF1F080B2E3
:1005A000704770B5044690420BD2101B652800D2EC
:1005B000652025188D4203D80321FCF791F808B176
:1005C000204670BD284670BD10B5A2F110030D295C
:1005D0004DD2DFE801F007090E151A1D21292C4E16
:1005E0002F364800F2B342E0062A3ED0072A3CD01C
:1005F0003DE00B2A39D00C2A37D00A2A35D036E014
:100600000D2A32D00E2A30D031E00C2B2DD92EE01D
:10061000113A0B2A29D92AE0032B26D990F85C003D
:10062000F8B11C2A21D922E0042A1ED01FE0012A99
:100630001BD01CE01D2A18D01E2A16D01F2A14D049
:1006400015E0202A11D0212A0FD0222A0DD0232AEA
:100650000BD0242A09D0252A07D0262A05D02E2AF5
:1006600003D004E001E0282A01D1012010BD0020C0
:1006700010BD0F2AFBD1F8E70B2819D00C2817D092
:100680000A2815D00D2813D00E2811D020280FD0FD
:1006900021280DD022280BD0232809D0242807D0C8
:1006A000252805D0262803D02E2801D00020704709
:1006B0000120704711F00C0F18D04A074FF4167143
:1006C000002A02DA4FF0100201E04FF0400201DA96
:1006D0004FF0960101F5BC71A0EB0103884203D9EC
:1006E00093FBF2F080B2704700207047022908D0D7
:1006F0007028F9D97038C11700EB5170C0F3CF00E2
:1007000070473C28F0D93C38C11700EB9170C0F31A
:100710008F0070470968C0F866107047C10701D0A4
:1007200001207047810701D502207047400701D59D
:10073000082070470020704710B540F6C412012908
:1007400006D0022905D040F2A1312920F2F78AFF14
:1007500008B1104610BD40F2E24010BD2DE9F04155
:1007600007460E46D7E90454FCF796FB98B11EB332
:10077000D7E90401401B002361EB04011A461B1A50
:100780008A4119DA421C71F1000107DB40F21B219A
:100790002920F2F767FF40F21121F9E73044401EAB
:1007A000B0FBF6F101FB06F0281844F10004C7E99C
:1007B00004040846BDE8F0810020FBE730B513468D
:1007C00006E0CC18D51A14F8014C5B1E4455DBB278
:1007D000002BF6D130BD00230364A0F8482040F27E
:1007E00071235A4301EB0212521EB2FBF1F1416434
:1007F00070472DE9F05F074690468B460126084674
:1008000000F0E1F98246584600F0DFF98146FFF733
:1008100085FF04465046FFF781FF054654EA050070
:1008200000D10026F9F7C4FA10EA090F00D100241C
:10083000F9F7BEFA10EA0A0F00D1002597F86A000E
:10084000A04200D1002488F8004097F86B00A8422D
:1008500000D1002588F8015074B96DB9584600F0F0
:10086000A0F9B7F89410401A00B247F6FE7188421A
:1008700001DC002800DC00263046BDE8F09F40F295
:10088000E2414843704740F2712110FB01F04FF6FE
:10089000FF7101EA4000704710B500231A4603E0DB
:1008A000845C2343521CD2B28A42F9D30BB100209C
:1008B00010BD012010BD0144142901DD1420704732
:1008C0006FF07E008142FADB48B2704770B5054692
:1008D00081EA114086B21046EC7A314600F063F8A6
:1008E00070402521B0FBF1F201FB120105EBD102B2
:1008F00001F00703527801269E40324201D008469B
:1009000070BD4443210C2846BDE87040F4F748BE52
:1009100010B5044690F8300008B1252801D91220FE
:1009200010BD32B194F8250028B1012809D01F204C
:1009300010BD002010BD2046BDE810401146F4F760
:10094000E7BDA28A496904F12500FFF7BFFF84F8DB
:100950003300EEE770B50446401C884204D00868B6
:10096000C4F8010008796071607900F01F006071BF
:100970000020E07205466619707800F04AFBB071FD
:10098000E17A6D1C0844EDB2E072052DF3D370BD21
:10099000C1B291FAA1F1000A090E90FAA0F0000E7E
:1009A00041EA0020704770B50D4648400024FFF72B
:1009B000EFFF00EB0010641C2844E4B280B2032C6B
:1009C000F5D370BD027802F00F02032A03D0052A86
:1009D00004D100F02EB940780C2801D000207047D7
:1009E0000120704770B5144605461F2A03D9EE2131
:1009F0002A20F2F737FE05F1090002F0BCFFA41D22
:100A00006C7070BD10B5027801F00F0302F0F002B7
:100A10001A43027007290CD2DFE801F0040604062D
:100A200004080400062102E00C2100E022214170AC
:100A300010BDA8212A20F2F715FE0A6840F8092FF8
:100A4000898881807047027802F07F0242EAC112F1
:100A5000027070470A6840F8032F898881807047C8
:100A60000278402302F0BF0203EA81110A430270B8
:100A7000704770B5144605461F2A04D94FF4887193
:100A80002A20F2F7EFFD05F1090002F074FFA41D22
:100A90006C7070BD42680A60007A08717047B0F8E7
:100AA0000900704770B5B0F80720B0F8094030F879
:100AB000055F10F8013CC08831B1B2F5506F03D921
:100AC00040F607518A420BD9911F40F67A46B1424F
:100AD00010D87BB1082B0DD893420BD2954209D880
:100AE000B4F5FA7F06D240F676410A38884201D83A
:100AF000012070BD002070BDB0F807007047B0F84D
:100B000009007047B0F80B00704710B5FB2904D9F5
:100B100040F2A9612A20F2F7A5FD417010BD80893D
:100B200008807047D0F816000860704742680A6075
:100B300080684860704750F80E2F0A60406848602F
:100B400070470968C16070470A68426049688160FF
:100B50007047007800F00300704780887047C088B5
:100B60007047008970474089704701891B290CD361
:100B700041894FF4A472914207D381881B2904D381
:100B8000C088904201D3012070470020704701794E
:100B9000490704D04079400701D001207047002068
:100BA0007047C08870470179407901F007014A1EFB
:100BB00000F007001140421E1040014301D0002008
:100BC000704701207047007970474079704700797D
:100BD000704701717047407970474171704710B597
:100BE0001B2A04D940F27F412A20F2F73BFD4270D4
:100BF000BDE81040C01C02F0BEBE027801F0030147
:100C000002F0FC020A43027070470171090A417147
:100C100070478171090AC17170470172090A4172F6
:100C200070478172090AC172704700797047007974
:100C3000704770B5D0F81F2090F8233012F0FF0FE6
:100C400003F0E00308D1C2F307242CB9C2F3074430
:100C500014B9120E00D14BB34678B0F81920B0F891
:100C60001B40B0F81750837D222E1FD131B1B2F551
:100C7000506F03D940F607518A420BD9911F40F6B5
:100C80007A46B14212D88BB1082B0FD893420DD2BD
:100C900095420BD8B4F5FA7F08D2B0F81D0040F6A3
:100CA00076410A38884201D8012070BD002070BD0D
:100CB0004168002291F82A32002B04D081F82A22C0
:100CC000406800F070BD704710B5017A19B1012974
:100CD00006D0002010BDC28803688088022103E08E
:100CE000C288036880880121F4F7C4FC08B9F4F7CE
:100CF00011FD012010BD08B5037A8DF80030009B6E
:100D000000939DF8003023B140F217311020F2F724
:100D1000A9FCBDE80840F4F771BEF4F79DBE037A64
:100D200082B08DF80030009B00939DF80030002BBE
:100D300002D102B0F4F762BE02B0704700204870E2
:100D40000320087001200871704710B58C880A894B
:100D50004B88C988A0F84830A0F84C10A0F84A4049
:100D6000A0F84E2010BD70B515460C4600F01AF9DB
:100D700096302844A04201D8201A70BD002070BDD2
:100D80002DE9F0470446C78E468FB0F84C50B0F8B6
:100D90004000854200D30546204694F86B1000F0D1
:100DA0009CF80146E5866187A28F04F12C00E38F51
:100DB0008046AA4200D22A468B4200D20B460282CB
:100DC000A8F81230BD4201D1B14201D0012000E0AB
:100DD00000208146B4F84850B4F84200A78E268F10
:100DE000854200D3054694F86A10204600F07DF84D
:100DF00094F86010022908D1AF4200D23D468642E5
:100E000000D23046002184F86010A8F80850A8F8F5
:100E10000C00BD4201D1B04201D0012000E0002011
:100E200040EA0900BDE8F087406870472DE9F041CD
:100E300016460F46044600F0B5F805463A462169C5
:100E4000E06A00F045F8A919814200D30846206302
:100E5000BDE8F0811B2202848283C28282824281A9
:100E60000282028142858285828400290AD14FF460
:100E7000A4714184C18341830183C1814182818105
:100E8000C18501867047006801F19C02904203D938
:100E9000401A9C38400870470020704710B5029CEB
:100EA0008182C2820383448310BD001D10B580B2CD
:100EB000012906D0022907D040F226210620F2F7A8
:100EC000D1FBC000503001E080002C3080B210BD5A
:100ED000884200D30846801A7047B0F84E10B0F828
:100EE0004400814200D208467047B0F84A10B0F87A
:100EF0004600814200D20846704738B50022A0F172
:100F00001803132402724A700C70D3F822504D60FB
:100F1000D3F826508D60D3F82A50CD60057A8DF82D
:100F20000050009D00959DF80050002DEAD138BD7D
:100F3000F0B587B00D460446F4F788FB002628B3C9
:100F4000A4F5BC702672078803A9384601F065FD38
:100F500008B1FD2117E0ADF80070BDF81200ADF842
:100F60000200BDF81400ADF80400BDF80E00ADF8A5
:100F70000600BDF81000ADF80800684601F089FDD4
:100F800020B14FF483712C20F2F76CFB1B202870EA
:100F90006E7054F80A0F68606068A8602089A881A4
:100FA00007B0F0BD962190F86B3090F86A2000F001
:100FB00000B82DE9F0410D46064698461746808E4A
:100FC0001146FFF772FF044639463046FFF78DFFA2
:100FD000A04200D20446B08F4146FFF766FF0746A5
:100FE00041463046FFF779FFB84200D338462044E7
:100FF0002844801DBDE8F08110B504460821204634
:10100000F2F7DEFB2068002802D160680028F5D0E6
:1010100010BD00F05501552202EA5000084400F0CE
:101020003301332202EA9000084400F00F0101EB83
:101030001010704710B5A0F1340230F8B44C002005
:1010400048700A230B700871A1F8054092F83D0022
:10105000C8712046F2F702FFFEF7AEFD40B1204610
:10106000FFF7A9F92046BDE810400021F2F780BD46
:1010700060216320F2F7F6FA38B500224A700723A0
:101080000B70A0F17404A0F5DF730272DA84D4F857
:101090007E504D60D4F882508D60B4F886508D81BA
:1010A0000A71057A8DF80050009D00959DF800505A
:1010B000002DEAD138BD00224A700B220A7000F1DF
:1010C0000A02837AA0F20A200B710088C880107986
:1010D0000872704700224A700C220A70827AA0F2CD
:1010E0000A200A710088C880704700224A700822CE
:1010F0000A70A0F5377212888A80C268C1F806208B
:101100000269C1F80A20808AC881704710B5446816
:101110000378002194F89D2080342046FFF754FA8C
:1011200010B10420607710BDAA211C20F2F79AFAB2
:1011300010B5416891F88C20D2070BD011F8DA2F46
:10114000521E52B20A704068002A05DAB9211C20EA
:10115000F2F788FAB721FAE750F88C1F21F0010165
:10116000016010BD00224A7006220A7050F8092F53
:101170004A6042688A6002898A81807A88737047EF
:1011800000224A700E22A0F5AC700A700088888098
:10119000704738B500244C7001250D70A0F15E0237
:1011A000A0F1DE030C7104721D88A1F8055092F8BD
:1011B0006750CD71B2F868500D81B2F86A504D8118
:1011C000057A8DF80050009D00959DF80050002D87
:1011D000E9D138BD70B503784068002500F180047E
:1011E00090F8DD1000F5987089070ED4627F002119
:1011F0002046FFF7E9F930B10120607784F8560006
:10120000A4F8525070BD6E210BE0217B89070FD5E9
:1012100094F85A10491E49B284F85A10002903DA8A
:1012200080214020F2F71EFAE16821F00201E1601E
:10123000857470BD00224A7019220A70D0F80A0025
:101240004860704710B504466FF00042D4E90010C2
:10125000504070EA010108D0FCF7DAFBD4E9002322
:10126000801A994101D3012010BD002010BD012832
:1012700002D14879800901D00020704701207047D1
:10128000012806D148790121B1EB901F01D101203D
:10129000704700207047022803D0032801D00020A7
:1012A00070470120704710B50446007CFFF7F3FF3C
:1012B00048B194F8570004F15801FFF718F90828CD
:1012C00001D0012010BD207C18B1022801D0E07DA2
:1012D00010BDBDE810400020F3F78EB808B590F8B7
:1012E00074108DF80010009900919DF8001041B91C
:1012F00090F8AE108DF80010009900919DF8001044
:1013000009B1012008BD90F89E008DF800000098FA
:1013100000909DF80000002008BDFF200870486B79
:10132000FEF7EABF7CB50D4604464FF48C720021EF
:1013300002F09BFBFF2020707F2084F82E001320FA
:10134000608042F210706084F2F746FE01466063EE
:1013500000226846FEF736FF00220121606BFEF78F
:10136000ABFF04226846616BFEF72CFF002211469A
:10137000606BFEF7A1FFA57304F12800BDE87C4077
:1013800000F06BB98078C0F3800008B1002070478E
:101390001F207047F5F702BB806870470120704737
:1013A00010B50446283000F018F96188BDE81040F7
:1013B0002822F5F7C3BC0022028643881D2B01D0EA
:1013C000417370474273704710B50024406BFEF7BD
:1013D0006BFF844384F0010010BD002070478078CB
:1013E00000F0010070478078C0F3C0007047012012
:1013F00070478078C0F34000704790F90E00704746
:101400000078FF2801D0012070470020704700F8C5
:10141000201F427070470A6840F8112F8988818028
:10142000012181717047007B704701207047C161C5
:1014300090F850204A72D0F85120C1F80A20B0F834
:101440005500C881704780F868107047C07B00283D
:1014500000D0012070470278202302F0DF0203EA67
:1014600041110A430270704710B5FFF740F8044677
:10147000F3F714FE38B12046F3F748FD18B11021F8
:10148000FFF70AFA08B1002010BD012010BD0121AC
:10149000F4F7F4BE0121F4F7F1BE00224A700522F0
:1014A0000A70D0F80A004860704710B50C46002159
:1014B00061701221217000F109012122201D02F02A
:1014C0005AFA0120E0712079002815D0B4F80540BF
:1014D00000212046FEF7C4FD00280DD00088FEF74D
:1014E0006AFF00212046F2F743FB002804D04FF4A6
:1014F00014712D20F2F7B6F810BD00224A701A229E
:101500000A7050F8092F4A6042688A60007A0873AE
:1015100070472DE9F04104460F46407EF3F7B6FCD4
:101520000646207E04F1510520B11EB1607EF3F71E
:10153000A1FCA0B194F86A00002824D0A07E002865
:1015400021D094F850002946FFF79AFEA8B1F3F78E
:101550008DFC3A462946BDE8F041FEF760BF012008
:1015600084F850003A4629463046FEF758FF617E1F
:101570002846BDE8F041F3F795BC39462846BDE85A
:10158000F041FEF73BBFBDE8F08110B504460846C8
:10159000F9F7B2F92179BDE810402520F9F782B9B1
:1015A00070B514461D460646FCF732FA001969412B
:1015B000C6E9000170BD70B50170427014460D4659
:1015C000807800F07FF810FB05F06043FF2803D31C
:1015D0005C212E20F2F746F870BD10B504468078E5
:1015E00000F070F86178227811FB02F14843C0B234
:1015F00010BD10B5044600F04DF86179491CC9B220
:101600006171627891420BD100226271E1780143ED
:10161000E170A378994203D1E2702179491C2171CC
:10162000BDE8104000F025B88170704770B50446E1
:10163000807800F047F8617811FB00F5E07800F061
:1016400041F86178627910FB012021782279891AAA
:1016500011FB05F1081AC0B270BD00210160818044
:1016600001214170017070470021C1704171017109
:10167000704710B5012807D0022807D0042807D0EA
:1016800039212E20F1F7EEFF252010BD262010BDB8
:10169000272010BD014600208A78D30702D0CB78DE
:1016A000DB0706D0930706D5CB789B0703D402202F
:1016B0007047012070475207FCD5C9784907F9D413
:1016C00004207047C0F38001C0F34002114400F0D1
:1016D00001000844704740F25A314843704740F2D5
:1016E000EF2070470E021C043006600C5A03B4064B
:1016F000C505F50B2512A301B103BF05EF0249068D
:10170000A30910B590F8101109B1002010BD90F890
:10171000D01031B1D0E935128A4202D9F4F796FDE2
:10172000F3E7012010BD10B531B1012908D040F216
:101730007A713020F1F796FFBDE8104000F0B7B99C
:10174000002180F8D010BDE8104000F013B910B5AA
:10175000044690F8E000002819D0012084F8100118
:1017600001462046FFF76FFE94F8E00070B114F8D0
:10177000C80FFBF7C1FC2078FBF722FE14F8C8095C
:10178000FBF7FCFD20B1002084F8E000002010BD34
:1017900040F205213020F1F765FFD0F8CC0070470A
:1017A00090F8E00070477CB5044690F82B020028C2
:1017B0005FD194F85C0203285BD1FCF729F9D4F8D7
:1017C0009032D4F89422C01A61EB020100231A4629
:1017D0001B1A8A414DDA421C71F1000102DB4FF401
:1017E000B86136E0216911B1B0FBF1F000E00020F2
:1017F000B4F89410401C0844A4F86C02B4F86C02CD
:10180000B4F82412081A00B2002832DD94F8A402B9
:10181000FBF772FC00282CD0FF2084F87102B4F88A
:10182000CE00B4F8CC1001AE401AB4F89410401EAB
:10183000084485B217E00096B4F86C120023012228
:101840002046F5F70FFD002813D0012804D040F200
:10185000F9513020F1F706FFB4F86C02BDF804101E
:101860000844A4F86C02B4F86C02281A00B20028EC
:10187000E1DA7CBD0020704770B5044600F0F0F856
:10188000A4F8F000002084F8E8000146012504F1E6
:10189000E80084F8F3500646FEF760FFB4F8000154
:1018A000401C0A2801D2A4F80001D4F8CC0038B1B9
:1018B000B4F80001401C0A2802D384F8F25002E078
:1018C000022084F8F200204600F022F820B12046E1
:1018D000BDE8704000F00DB894F8C800314600F043
:1018E000BDF8002804D140F28E613020F1F7BAFE35
:1018F00070BD10B5044614F8C80FFBF73FFD00207B
:10190000207610BD10B5FFF74BFD00F5887010BDB7
:1019100070B5054690F8100108B1012070BDD5E9F9
:1019200042106FF00042504070EA010112D00024D2
:1019300021462846FFF7E6FFF5E93E1240185441DC
:10194000D5E90421F83D101AA14103D52846F4F742
:101950007DFCE2E7002070BD10B5044690F86B00F6
:1019600000F0EFF902462046BDE8104040F21B119E
:10197000FFF75CBA10B5F8F7F1FDBDE81040FBF7D2
:101980005FBE2DE9F047044690F87202002851D05E
:1019900094F85C0203284DD194F86B9001F035FC6B
:1019A000054694F81B02F5F77FFB284486B294F8AD
:1019B0001B02F5F779FB00F5C8601FFA80F848466E
:1019C000F8F78AFED4F8AC120D1A4846F8F7B0FEC4
:1019D0004FF47A7A00F2E730B0FBFAF02D1A48465D
:1019E000F8F77AFED4F830120F1A4846F8F7A0FE3E
:1019F0004AF2A1310144B1FBFAF0391AA1F16000B9
:101A00007043B0FBF8F2292000EB51006032A0EBEC
:101A1000520100EB5200A94201D8854201D9FDF7DD
:101A20002BF831462069FDF78FF80021C4F86402D5
:101A300084F87212BDE8F08770B50C460546F8F7D9
:101A400077FE4AF2A13108444FF47A71B0FBF1F607
:101A50002846F8F741FE3044204470BDFBF72EB80D
:101A60007CB50446FFF7C3FCF8B12046FFF7B7FC8E
:101A700018B92046FFF7BDFC40B155246846FDF774
:101A8000BBFA9DF8000018B1012502E05024F5E7EB
:101A9000002501A8FDF798FA9DF8040000B1012087
:101AA000054300D00A3420467CBD61207CBD70B562
:101AB0000446408C002530B1F4F760F8618CB0FB2F
:101AC000F1F201FB12052046FFF766FCD4E93E2146
:101AD0002844E8340025821845EB0100C4E90420BD
:101AE00004F80B5B012004F80109022004F8F20954
:101AF0002046FFF7B5FFA4F8F0002046FFF708FFE7
:101B000030B994F8C80004F1E801FFF7A7FF28B145
:101B1000A4F80051BDE87040FFF72CBF40F2D4613B
:101B20003020F1F79FFD10B50446002084F85C02D8
:101B300094F8A402FBF722FC202084F8A40210BD34
:101B40002DE9F8430446002580F8D050D4E93E67DB
:101B5000894680F8E0504FF0010880F8E180D0F825
:101B6000CC004146C834F3F721FC6068C0F89062AD
:101B7000C0F894726168207881F8A4026168C1F8A5
:101B8000A8926068C0E9A667646884F85C52002384
:101B9000A4F8A0521A46194620460095F5F762FBB4
:101BA00020B140F219213020F1F75CFDC4F8585201
:101BB000C4F8505284F85C82A4F86E52A4F86C52B7
:101BC000943484F8DD512088401E2080A4F80E5201
:101BD000BDE8F843FFF7CEBE70B540B1092949D240
:101BE000DFE801F007153C3C38482A404400CB218F
:101BF0003DE00446F4F7FAFA10B140F2752136E000
